:020000040800F2
:10000000F8FF012061A40908FDA40908916E050804
:10001000FDA40908FDA40908FDA4090800000000CA
:10002000000000000000000000000000FDA409081E
:10003000FDA4090800000000FDA4090839610408B6
:10004000FDA40908FDA40908FDA40908FDA40908E8
:10005000FDA40908FDA40908052D04082D2D040898
:10006000552D04087D2D0408A52D04084903000022
:100070005D03000071030000850300009903000088
:10008000AD030000C1030000FDA40908FDA4090898
:10009000FDA40908FDA40908FDA40908CD2D040844
:1000A000FDA40908F5450408FDA40908E545040870
:1000B000054604081546040825460408C51A040820
:1000C000B91A0408F91A0408ED1A0408FDA409086D
:1000D000FDA40908C1300000113200007D3300008A
:1000E0000D2E0408FDA4090800000000E1460408E4
:1000F000B9460408F1460408A9460408D5030000DF
:10010000FDA40908FDA4090835460408FDA4090852
:10011000ED3400005D3600004546040865D7080848
:10012000E9030000FD0300001104000025040000A5
:1001300039040000FDA40908FDA40908FDA409086C
:1001400000000000000000000000000000000000AF
:100150004D0400006104000075040000CD3700006C
:100160002D1B0408211B0408FDA40908FDA409088F
:10017000FDA40908FDA40908FDA409080000000069
:10018000FDA40908FDA409083D390000AD3A0000AE
:10019000FDA40908FDA40908FDA40908FDA4090897
:1001A000FDA40908FDA40908FDA40908FDA4090887
:1001B000FDA40908FDA40908FDA40908611B0408A1
:1001C000551B0408FDA40908FDA40908FDA409089D
:1001D000FDA40908A5CD0808FDA40908FDA4090887
:1001E000FDA40908FDA40908FDA40908FDA4090847
:1001F000FDA40908FDA40908FDA40908FDA4090837
:10020000FDA40908FDA40908FDA40908FDA4090826
:10021000014704081147040821470408FDA4090800
:10022000FDA40908FDA40908FDA4090800000000B8
:10023000FDA40908FDA4090800000000FDA40908A8
:10024000FDA40908FDA40908FDA40908FDA40908E6
:10025000FDA40908FDA40908FDA40908FDA40908D6
:10026000FDA40908FDA40908FDA40908FDA40908C6
:10027000FDA40908FDA409081D3C000000000000C1
:10028000FDA4090800000000FDA40908000000000A
:0802900000000000FDA40908B4
:020000040804EE
:10000000114A037A0168D35C10B4CC58CA1824F0A2
:100010000104CC501368DB07FCD4037D1F2B09D9E6
:10002000203B20225DF8044B02FA03F343F018034F
:10003000CB60704720225DF8044B02FA03F343F0D3
:1000400018038B60704700BFE8420A084368426D9E
:1000500030B49A61EFF31182502383F31288416820
:10006000D2B2856C0B68046D23EA050323430B6051
:1000700082F31188436981681A68096822F00102D5
:10008000D0E908541A60826A1D605C615A60D0E948
:100090000B429C60DA600023B0F86C2030BCCA626E
:1000A00003777047002A4FEA014C034630B508BF7A
:1000B000E64600F1C00514BF8E468C460024196840
:1000C0000C3353F8042C43F8084C41EA0C0142EA83
:1000D0000E02AB4243F80C1C43F8042CEFD1D0F8CD
:1000E000C03043EA0E03C0E93144C0F8C03030BD2F
:1000F00010B40C4C6368002B11DD002004F1080CD7
:100100000146DCF8AC3003F1C00259600C33934275
:10011000FBD1013063680CF5867C8342F1DC5DF82D
:10012000044B704704000020F0B5404C04EB401332
:1001300093F8543403B9F0BD3D4B42011D7893F858
:1001400001C065450CD00CEB4C0E03EBCE0E9EF8B7
:1001500004604FEA4C0E771E012F5AD9032E52D05D
:100160002244A2F83814EFF31181902383F312880C
:1001700092F83A34C9B2B2F8380443EA4003002096
:100180009BB282F83A0481F311881909207881EA38
:1001900013215940D8B1C9431B01D2F8505401244E
:1001A000D2F83C049BB201F00F01D5F8AC2084409A
:1001B0000B4302F1C000590013F4004F8BB202D17F
:1001C0005168214351600C329042F4D1F0BDD2F815
:1001D0003C041B01D2F8502401F00F0110309BB2F7
:1001E0000124D2F8AC200B43844002F1C000590036
:1001F00013F4004F8BB202D15168214351600C328D
:100200009042F4D1F0BD0CF1010606F00306AE42B7
:10021000A6D0E64403EBCE030344597C00299FD0CB
:10022000A318012083F83A049AE700BF04000020D5
:10023000F01A0024704700BF024B03EB401393F801
:100240005504704704000020D0E90920131A5842D1
:100250005841704790F8573830B53BB990F8551869
:10026000012490F85638DAB2914200D830BD04FA31
:1002700003F2B0F85E5801332A43A0F85E28F2E793
:100280000379024613F0010006D0D2E90731D268A3
:100290005B1A013A03EA0200704710B5037904467D
:1002A00013F001030ED0FFF7EBFF034650B1226AB3
:1002B0006369E1689B5C0132B2FBF1F0DBB201FBE8
:1002C00010222262184610BD03799B070AD5436AA3
:1002D0008269D154436A02690133B3FBF2F102FB34
:1002E00011334362704770470171704703790146CB
:1002F00013F0020007D00B69D1E90921013B521A22
:100300001A40D2B2981A70470C4B4FF0E02C10B440
:100310005A6EDCF81800596E8A42F9D1996E8842FB
:10032000F6D8DC6E4FF47A7101FB04F31B1AB3FBB1
:10033000F4F35DF8044B01FB02307047F01A00241F
:100340002DE9F04F4C484FF0010A4C494FF002099B
:100350004B4B4FF0040808271026202540244FF06F
:10036000800EDFF820C130F8022F12F0010F03D009
:100370001960083323F804AC12F0020F03D019609F
:10038000083323F8049C12F0040F03D019600833DB
:1003900023F8048C12F0080F03D01960083323F8F7
:1003A000047C12F0100F03D01960083323F8046C9A
:1003B00012F0200F03D01960083323F8045C12F008
:1003C000400F03D01960083323F8044C12F0800F5B
:1003D00003D01960083323F804EC12F4807F05D0B1
:1003E0004FF4807B1960083323F804BC12F4007FBB
:1003F00005D04FF4007B1960083323F804BC12F4D5
:10040000806F05D04FF4806B1960083323F804BC6B
:1004100012F4006F05D04FF4006B1960083323F815
:1004200004BC12F4805F05D04FF4805B1960083380
:1004300023F804BC12F4005F05D04FF4005B196090
:10044000083323F804BC12F4804F05D04FF4804BDE
:100450001960083323F804BCD20B05D04FF40042D6
:100460001960083323F8042C01F5806161457FF49D
:100470007AAFBDE8F08F00BF76C2090800000258CD
:10048000601B00240024025810B584464FEA810EF8
:10049000102312F4004F4FEA420214BF0E24072427
:1004A000013B92B2CCF80040F444F2D100EB81124F
:1004B0008C010351122042F8213010BD10B5844642
:1004C0004FEA810E0424130B013C4FEA021203EBA6
:1004D000430392B203F11803CCF80030F444F2D194
:1004E00000EB01130A018450062043F8214010BD9F
:1004F000704700BF704700BF00EB4000024B03EBAA
:10050000C00393F84905704704000020064B93F898
:10051000F825824206D900EB400003EBC003D3F874
:100520004C05704700207047040000201D4B93F8D5
:10053000FC25AAB3D3F8381509B100200860012AB8
:100540002ED0D3F8501509B100200860022A27D018
:10055000D3F8681509B100200860032A20D0D3F829
:10056000801509B100200860042A19D0D3F8981525
:1005700009B100200860052A12D0D3F8B01509B1DE
:1005800000200860062A0BD0D3F8C81509B1002056
:100590000860072A04D0D3F8E0350BB100221A60B6
:1005A000704700BF040000201D4B93F8FC25AAB340
:1005B000D3F8381509B100200860012A2ED0D3F8ED
:1005C000501509B100200860022A27D0D3F8681519
:1005D00009B100200860032A20D0D3F8801509B1A2
:1005E00000200860042A19D0D3F8981509B100201A
:1005F0000860052A12D0D3F8B01509B100200860B0
:10060000062A0BD0D3F8C81509B100200860072AC4
:1006100004D0D3F8E0350BB100221A60704700BF58
:1006200004000020C44B1B78002B40F04F81C34BCB
:1006300093F8FC25002A00F0498193F8481530B55D
:1006400000294ED1D3F838150020012A086047D977
:1006500093F86015002966D1D3F850150020022ABE
:1006600008603DD993F87815002940F0CB80D3F885
:1006700068150020032A086032D993F890150029E4
:1006800040F0E280D3F880150020042A086027D9C2
:1006900093F8A815002940F0F880D3F898150020A9
:1006A000052A08601CD993F8C015002940F00F8175
:1006B000D3F8B0150020062A086011D993F8D81590
:1006C000002959D1D3F8C8150020072A086007D996
:1006D00093F8F025002A73D1D3F8E03500221A6090
:1006E00030BDD3F83C25910AA1F58011522940F282
:1006F0000F814FF0FE0CEFF31181502080F3128830
:100700008F4C4FF02C0E556AC9B250690EFB0C4C41
:10071000013540F00100CCF81855506181F3118883
:1007200093F8FC258EE7D3F85425910AA1F58011A2
:10073000522940F2F2804FF0FE0CEFF3118150206D
:1007400080F312884FF02C0E556A7D4CC9B2506967
:1007500001350EFB0C4440F00100C4F818555061FF
:1007600081F3118893F8FC250020D3F85015022A54
:1007700008603FF677AFB3E7D3F8CC25910AA1F52F
:100780008011522900F2EA806E48014491F814C0A9
:10079000EFF31181502080F312884FF02C0E556A30
:1007A000674CC9B2506901350EFB0C4440F00100A2
:1007B000C4F81855506181F3118893F8FC2581E73E
:1007C000D3F8E425910AA1F58011522900F2C980DD
:1007D0005C48014491F814C0EFF31181502080F37C
:1007E00012884FF02C0E556A554CC9B2506901352C
:1007F0000EFB0C4440F00100C4F81855506181F321
:10080000118869E7D3F86C25910AA1F58011522966
:1008100040F288804FF0FE0EEFF31181502080F3FC
:1008200012884FF02C0C556A454CC9B250690135FD
:100830000CFB0E4440F00100C4F81855506181F3E0
:10084000118893F8FC2512E7D3F88425910AA1F5C5
:10085000801152296BD94FF0FE0CEFF3118150201B
:1008600080F312884FF02C0E556A354CC9B250698E
:1008700001350EFB0C4440F00100C4F818555061DE
:1008800081F3118893F8FC25FCE6D3F89C25910AA6
:10089000A1F58011522957D94FF0FE0CEFF31181C9
:1008A000502080F312884FF02C0E556A244CC9B2A8
:1008B000506901350EFB0C4440F00100C4F8185596
:1008C000506181F3118893F8FC25E6E67047D3F870
:1008D000B425910AA1F5801152293AD94FF0FE0CA6
:1008E000EFF31181502080F312884FF02C0E556ADF
:1008F000134CC9B2506901350EFB0C4440F00100A5
:10090000C4F81855506181F3118893F8FC25CFE69F
:100910000C48014491F814C0EDE60A48014491F8EE
:1009200014C00AE70748014491F814E074E7054849
:10093000014491F814C090E7000000240400002056
:10094000F01A002478C209080748014491F814C03D
:10095000A4E70548014491F814C0C1E74FF0FE0C2C
:1009600016E74FF0FE0C37E778C2090800EE100AD0
:10097000B8EE400A704700BFBCEEC00A10EE103A55
:1009800098B2704707280AD84FF4B472054B02FB9F
:100990000033B3F80006B0FA80F040097047002039
:1009A000704700BF04000020072807D8044B4FF40D
:1009B000B471012201FB003383F80226704700BFA7
:1009C00004000020072808D8044B03EB401393F8D9
:1009D000542412B1012283F83A2470470400002005
:1009E000072808D8054B03EB4013B3F83804B0FAD6
:1009F00080F0400970470020704700BF04000020CD
:100A0000054B93F8F825824204D903EB4013D3F841
:100A10004404704700207047040000200346012270
:100A200000205A77704700BF826908B50346006B03
:100A3000D96A02449A6101B18847002008BD00BF0D
:100A4000436A02461B681B6A5B685B7813F001000F
:100A500008BF5077704700BFC2628161704700BF16
:100A6000704700BF043070470C4B93F88827D3F8C9
:100A7000841702440144D2B2C3F8841783F888274C
:100A800093F88827120605D593F8882782F080020C
:100A900083F88827024B01225A707047F01A00240D
:100AA000000000242DE9F84F164FD7F88C57ED0AB7
:100AB00023D00026DFF850A007F5F269B04674197C
:100AC000D7F890174FF01003524648BF0134D1F8C1
:100AD00028B04846C7F8BC876410E102D8470F2801
:100AE0000BDD094B03F1100153F8042B013207D140
:100AF0008B42F9D12546B542E1DCE802BDE8F88F2A
:100B0000661CF8E7F01A002440E60024194B596EE1
:100B1000D3F8C4278A1A322A05DCD3F8D8278A1AD0
:100B2000002A11DC7047D3F8C81749B193F8D427CD
:100B3000888802F001020968120100FA02F28A6153
:100B40000022C3F8D8277047D3F8C8276AB11068C5
:100B50003231928810B44469C3F8D81722425DF844
:100B6000044B18BF1204826170473231C3F8D817A2
:100B7000704700BFF01A0024074AD2F8C8374BB1BB
:100B800092F8D4279988186802F001031B0101FA32
:100B900003F3836100207047F01A0024044B4FF4E4
:100BA000007C0020D3F8E837A2F800C00B60704743
:100BB000F01A002400207047012070470120704780
:100BC000002070472DE9F0414FF425728EB00021CE
:100BD00073485AF0D9FF734B734D4FF00008D3F8A8
:100BE000F02040F27D27A5F1680605F6F41442F0E6
:100BF0000102C3F8F020D3F8F02002F001020092C5
:100C0000009AD3F8E82042F00102C3F8E820D3F8B4
:100C1000E82002F001020192019AD3F8E82042F0A4
:100C20000202C3F8E820D3F8E82002F002020292A0
:100C3000029AD3F8E82042F00402C3F8E820D3F87F
:100C4000E82002F004020392039AD3F8E82042F06D
:100C50000802C3F8E820D3F8E82002F00802049262
:100C6000049AD3F8E82042F01002C3F8E820D3F841
:100C7000E82002F010020592059AD3F8E82042F02D
:100C80002002C3F8E820D3F8E82002F02002069200
:100C9000069AD3F8F02042F00202C3F8F020D3F80D
:100CA000F02002F002020792079AD3F8E82042F0FF
:100CB0004002C3F8E820D3F8E82002F0400208928E
:100CC000089AD3F8E82042F08002C3F8E820D3F86D
:100CD000E82002F080020992099AD3F8E82042F451
:100CE0008072C3F8E820D3F8E82002F480720A92F8
:100CF0000A9AD3F8F02042F48032C3F8F020D3F8F7
:100D0000F02002F480320B920B9AD3F8F02042F4D8
:100D10000032C3F8F020D3F8F02002F400320C9235
:100D20000C9AD3F8F02042F48022C3F8F020D3F8D4
:100D3000F03003F480230D930D9B55F82810002309
:100D400054F83320914226D001330E2BF8D10020E5
:100D500008F1070852F0B0FBB845EED14FF000089B
:100D600040F27D2755F82810002354F83320914293
:100D70000CD001330E2BF8D1002008F1070852F0F7
:100D80009BFBB845EED10EB0BDE8F08106EBC30386
:100D9000B3F8600AF1E706EBC303B3F8600AD7E7DC
:100DA000E01F002400440258E0C2090810B50446C0
:100DB0005AF0B4F90146204689B2BDE81040FFF769
:100DC000B3B900BF38B50B4D00EB400005F5A76384
:100DD000C40003EBC003254493ED027AD3ED037AFC
:100DE000E7EE007AB0EE670A5AF098F9D5F8383590
:100DF000186038BD0400002002692DE9F843C3687B
:100E000012EA030828D005460E464FF00047B8FA0C
:100E100088F327FA03F21B3BD24308EA02082A614F
:100E2000042B16D8DFE803F03B30251A0300B36A21
:100E3000002B3FD003F1FF3900231FFA89F9B36279
:100E4000746A34B123682046494698476468002C88
:100E5000F8D1B8F1000FDAD1BDE8F8837068002846
:100E6000F7D0696B036889B29847B8F1000FCED10B
:100E7000F2E7B0680028ECD0A96B036889B2984704
:100E8000B8F1000FC3D1E7E7F0680028E1D0E96BC3
:100E9000036889B29847B8F1000FB8D1DCE7306930
:100EA0000028D6D0296C036889B29847B8F1000FA2
:100EB000ADD1D1E7EB6A1FFA83F9C1E72DE9F04321
:100EC000144C83B0DFF85090DFF8508004F5906642
:100ED00002E00834B44219D094F90650002DF8D13C
:100EE0002768083407EB08039B0A09EB4303B3F8B0
:100EF000CC0A52F0E1FA34F8041C01232A463846A1
:100F0000CDE9005555F04AFBB442E5D103B0BDE848
:100F1000F08300BF601B002478C209080000FEA710
:100F20008069B43049F0DABAF8B5A0F507642379DE
:100F3000DB0725D5657994F8543805F001073D465F
:100F4000FBB1D4F848341A68D36A5B08536294F84A
:100F5000583823B1B4F862380133A4F8623885F008
:100F60000101606C50F0B2FC012384F85738002373
:100F700084F8553884F85638A4F85E3884F8543824
:100F8000F8BD94F85768012E03D194F8553884F8C9
:100F900056382046FFF75EF94EB9012385EA030172
:100FA00084F85738606CBDE8F84050F08FBC0023DF
:100FB000394684F85738F5E738B54AF01DFF0D4932
:100FC0000D4CD1F8FC20A4FB00400C4D42F0807287
:100FD0000B4B800CC1F8FC204FF060420949E866D9
:100FE000C2F8B01F00225A601A6842F001021A606B
:100FF00038BD00BF00ED00E083DE1B43F01A002483
:10100000001000E055CEACC51B481C4AC1681C4B03
:1010100010B44FF6FF0485B021401A4C0A43C26059
:10102000D3F8D010D3F8DC20C4F8681842F000528E
:10103000C3F8DC20D3F8DC2002F000520192019AC0
:10104000D3F8DC2042F08042C3F8DC20D3F8DC2067
:1010500002F080420292029AD3F8DC2042F0004271
:10106000C3F8DC20D3F8DC3003F000430393039B88
:1010700005B05DF8044B9FE700ED00E00005FA05C0
:1010800000440258F01A002401302DE9F84F7E4C3C
:1010900001F1FF387D4D10265FFA80FB012750F0EB
:1010A0006DF84FF4FA794FF0E0214FF47A7C6B68D9
:1010B000C3F30803002B40F0C080EFF31183002B33
:1010C00040F0BB80636E8869626E9342FAD1A26E73
:1010D0009042F7D8E26E0CFB02FEAEEB000EBEFBB8
:1010E000F2FE0CFB03EE6B68C3F30803002B40F029
:1010F0008680EFF31183002B40F08180636E886956
:10110000626E9342FAD1A26E9042F7D8D4F86CA0E6
:101110000CFB0AF2121AB2FBFAF20CFB0323A3EB4C
:101120000E03B3F57A7FDED3B9F10109BFD14FF4D5
:101130007A79584650F0F4F94FF0E021CC466B68CC
:10114000C3F30803002B40F08B80EFF31183002BD7
:1011500040F08680636E8869626E9342FAD1A26E17
:101160009042F7D8E26E0CFB02FEAEEB000EBEFB27
:10117000F2FE0CFB03EE6B68C3F308030BBBEFF34B
:101180001183F3B9636E8869626E9342FAD1A26EDD
:101190009042F7D8D4F86CA00CFB0AF2121AB2FBFA
:1011A000FAF20CFB0323A3EB0E03B3F57A7FE2D331
:1011B000B9F10109C3D1B8F10108BFF470AFBDE8BE
:1011C000F88FEFF3118386F31288D1F818A00A691B
:1011D000D20303D5C4F86C78D1F818A0606EDBB2E6
:1011E000D4F86C2883F311880244E06E0CFB00F302
:1011F000A3EB0A03B3FBF0F30CFB0233D3E7EFF3EB
:10120000118386F31288D1F818A00A69D20303D596
:10121000C4F86C78D1F818A0606EDBB2D4F86C28F2
:1012200083F311880244E06E0CFB00F3A3EB0A0386
:10123000B3FBF0F30CFB023371E7EFF3118286F39B
:10124000128888690B69DB0302D5C4F86C78886959
:10125000636ED2B2D4F86CE882F31188734439E734
:10126000EFF3118286F3128888690B69DB0302D5DC
:10127000C4F86C788869636ED2B2D4F86CE882F3F3
:10128000118873446EE700BFF01A002400ED00E0FF
:1012900070B505460A26084C013E00D170BD94F990
:1012A000000019F00BFC031E04DB6178EA18517290
:1012B000A278EA540434EFE756CD090838B590F81F
:1012C00028300446012B06D0407F08B9012038BDE4
:1012D0000023637738BD406A03681A7B9AB9637F3D
:1012E000002BF3D00A4D022305F1200205F1400145
:1012F00044F006FE95F82130D84303F0010300F0D6
:1013000001006377E6E71B6A002BE8D0002038BDB8
:1013100040E6002438B5044694F82830012B07D065
:10132000637F0BB100236377012038BD1B6A23B1B3
:10133000606A03681A7B002AF8D1637F002BF3D020
:10134000074D022305F1200205F1400144F0D8FDCC
:1013500095F8213003F00102DB076277E4D5DBE783
:1013600040E60024F0B5002395B0224E04460693D3
:1013700002200B9306F180021093139311930092B5
:1013800006F1A002277F1C4D0192626A04950D466A
:101390000290CDE90E3301238DF80C3007938DF8C0
:1013A00020308DF834308DF8483006F1C0030593B5
:1013B000124B099306F160030A933B1D10680C93CE
:1013C00056F096FD9FB12A0E06F1620386F8612061
:1013D0002A0A9D70280C69465A701870606A44F099
:1013E000D5FD636A186856F083FD15B0F0BD06F1AF
:1013F0006103EDE740E60024410A04081D0A0408E1
:1014000010B594B004465022064968465AF05EFB77
:101410006946606A44F0BAFD636A186856F068FD70
:1014200014B010BD7CCD09082DE9F8431F46436A6E
:10143000044688461868914656F05AFD237FA069F5
:10144000002B3BD0254E020E052386F8E120E23624
:10145000234D012FB0706B634FEA10434FEA102009
:10146000337070704FF00000D8F800302B64D9F85A
:101470000030AB642363A86523D0022F1CD1D9F8B8
:10148000042028651344D8F8041085F84C00EA6558
:10149000012269652363134B85F860206B66124B4C
:1014A000627FA3F11401606A002A08BF194644F064
:1014B0006DFDE36A63B1206BBDE8F88304230B4E36
:1014C000C6E7084B85F84C706865E8652B65E6E76C
:1014D000636A186856F00CFDEDE700BF40E6002493
:1014E00000000024290A04081800002421E7002431
:1014F00000B583B08161019201A9049A0093012390
:10150000C2626A46FFF790FF03B05DF804FB00BFBC
:101510002DE9F843DDF820800F46164600212022F1
:1015200004461D465AF030FBB8F1000F0CD0D8F835
:101530000030B8F80A20E3811B0C2382D8F804306D
:101540006282E3821B0C2383384658F0A1FAF3062B
:1015500019D4431EB8B107EB000C01E0013B12D3D4
:101560001CF801EDBEF12E0FF8D1C01A03F10109EC
:10157000421EB944032AA8BF0322082BA8BF082390
:1015800090461A4606E008280246B9464FF0000881
:10159000A8BF08224FF020333946204623606360FD
:1015A0005AF094FA164B04F108004246494623814A
:1015B00083705AF08BFA611EE21D11F801CFACF175
:1015C0006103ACF1200C192B98BF81F800C0914247
:1015D000F3D104F10A0011F8013FA3F16102203BAD
:1015E000192A98BF0B708142F5D1182365832D0C01
:1015F000E6722373099BA582E361BDE8F88300BF0F
:10160000202020002DE9F04FDFF8589485B0D9F85C
:101610006400C9F8C407002B60D00C46154601F5DC
:10162000FE7603EB020B1FE0002D64D0D9F8F437EF
:10163000AB4200F0C780D9F8F037AB4200F0F98038
:10164000D9F8F837D9F8FC17AB424BD88D42C0F027
:101650007481691A20464FF01DFA013504F50074B3
:1016600006F500765D4539D0D9F80028AA42DBD8C6
:10167000AA1AD9F81078D308396B02F00708023398
:101680008B4202D3BA6B93420BD939461846039367
:101690004FF0D0F9039B0746002800F06E81C9F88F
:1016A00010083A79002A40F01F81D7F828A0BAF133
:1016B000000F00F05B813A6B013520464FF400715A
:1016C0009B1AFA6804F5007406F5007608EBC30867
:1016D0003B4602EB4822D0475D45C5D1002005B00E
:1016E000BDE8F08F8D42B4D24FF400720021204645
:1016F0005AF04AFAB1E74FF40072294620465AF0F0
:1017000043FA8023CB4A84F8BE310C2384F8C231DB
:10171000D9F8F017D9F8E8379142C4F8C611C4F8DF
:10172000CA3100F30F81C44A013BC44F82FB01025E
:10173000C81787FB01C70A44C0EB6212C0EB273011
:10174000BF4F87FB02C7C2EB821C84F8C101801027
:10175000A1EB0C01174420F03F0001310843D117E1
:10176000C1EBE71184F8C0010A4484F8BF21B14AF3
:10177000934200F3F380B04AB04882FB0312D917BA
:1017800080FB03701A44C1EB6212C1EB2031AC48FC
:1017900080FB0270C2EB821784F8C5118910DB1B35
:1017A000104421F03F0101331943D317C3EBE01379
:1017B00084F8C4111A4484F8C3214AF65523A4F8C6
:1017C000FE314AE74FF0FF3300274FF4F072201D3F
:1017D00084F8EC31394684F8ED3184F8EE3184F840
:1017E000EF315223237063706123A37084F8E731D3
:1017F0004123E37084F8E631722384F8E43184F8FD
:10180000E531D9F80838C4F8E8315AF0BDF9552364
:10181000C4F8F07184F8FE316FF05503C4F8F47128
:10182000C4F8F87184F8FC7184F8FD7184F8FF3114
:1018300013E74FF40072002120465AF0A5F9814BBE
:10184000022203CB45F6EB032274227323809023FC
:10185000A273A370F82384F82C200822C4F8030094
:101860006273C4F807106375D9F8F017D9F8E83730
:101870005B1AD9F8F8172362D9F8FC375B1A4AF6D5
:10188000552163620023E372E3736377A377E37701
:1018900084F82D3084F82E3084F82F3084F83130DD
:1018A000694BA3613E232377012384F830308023E2
:1018B00084F84030654BC4F84230654B84F84620CC
:1018C000A4F8FE11634A03CBC4F84B101988C4F87E
:1018D00047009B78A4F84F1084F8513003CAC4F82D
:1018E0005200C4F85610B8E64FF4007200212046AA
:1018F0005AF04AF93B6CB8F1000F45D104F1200AC7
:10190000002B00F081803B6B112253492046CDE92A
:101910000088FFF7FDFD3B6C1A6C002A00F0818007
:101920001B6B504611224D49CDE90088FFF7F0FDB1
:1019300004F1400A4FF4E07871E0E91A20464FF0D4
:10194000A9F88AE6FF22013B84F8C1214FF6FF7215
:10195000A4F8BF21374A93427FF70DAFFF2384F8E5
:10196000C5314FF6FF73A4F8C33126E751464FF453
:10197000007220465AF008F96FE6231F384A43F8F0
:10198000042F9E42FBD168E6002B7F6C14BF02231C
:101990000123C3EB0813002F3FF45FAE013BBF6C84
:1019A000002B01DD002FF9D1A2464FF40078002F63
:1019B0003FF453AE0AEB080303959A460BE000256B
:1019C000A8F12008CDE900E5FFF7A2FDBF6CCFB17B
:1019D000B8F11F0F16D93D7907F11C0E1122396895
:1019E0003B6BAAEB0800002DE9D17A79A8F1200819
:1019F0003D6942F02102CDE900E5FFF789FDBF6CAA
:101A0000002FE5D1039D28E6CDE9008843464FF439
:101A1000F0780822D9F8EC172046FFF779FD7F6CA3
:101A2000C5E75046434611220C49CDE90088FFF72F
:101A30006FFD7DE7FF03FB0083200882975545413A
:101A40008180808020420A083F00FF0029940E0D0B
:101A50002C420A0838420A0818420A081C420A089E
:101A6000DEADBEEFF01A002430B40D4CBFF34F8F43
:101A70000C4BC3F85C42BFF34F8FBFF36F8F0A4B21
:101A80000A4D03F13000DA792AB1597934F811207E
:101A900092B225F811200C338342F4D130BC704748
:101AA000A0EA002400ED00E06023002400EA002406
:101AB00000207047704700BF014849F059BE00BF81
:101AC000CC230024084810B4D0F8DC38D0F81049F2
:101AD00099691A682CB1234600F6DC005DF8044BC6
:101AE00018475DF8044B7047F01A0024014849F08C
:101AF0003FBE00BF30240024084810B4D0F840395D
:101B0000D0F8744999691A682CB1234600F514601D
:101B10005DF8044B18475DF8044B7047F01A002439
:101B2000014849F025BE00BF94240024084810B4A1
:101B3000D0F8A439D0F8D84999691A682CB123464D
:101B400000F6A4105DF8044B18475DF8044B70478D
:101B5000F01A0024014849F00BBE00BFF82400240D
:101B6000084810B4D0F8083AD0F83C4A99691A6885
:101B70002CB1234600F608205DF8044B18475DF8A9
:101B8000044B7047F01A0024B0F1FF3F00F062826E
:101B900003282DE9F04F054683B000F32B81642024
:101BA000BE4C05FB00F004EB000CDCF8DC080CF686
:101BB000DC0B002800F01E81FF2A4FEA41077ED08F
:101BC0009CF81D19202940F00F819CF81C1901294F
:101BD00000F00A810121D4F8548A8CF81C1906E01F
:101BE000D4F8541AA1EB0801192900F20781816980
:101BF00011F40049F4D14FF0640A0C99CDF800803B
:101C000058460AFB054ACAF800192221CAF8109959
:101C10008AF81D1940218AF81E193946CAF82099F8
:101C2000AAF806390A2351F06BF8002840F0028127
:101C3000BAF806399BB2FF2B40F2E581DAF8DC18DE
:101C4000FF239748AAF804394B68964A03403B4360
:101C50001A434A604FF0640909FB054906E0D4F8CD
:101C6000543AA3EB08030A2B00F23C818A6912F074
:101C70000402F4D04A6AD9F800391A70B9F8063962
:101C8000D9F80029013B01329BB2C9F80029A9F813
:101C90000639B9F80439B9F80629013B92B29BB26A
:101CA000A9F8043912B1002B00F05481B9F80639B3
:101CB0009BB2002B00F0B981D9F8DC18D6E79CF86C
:101CC0001D29202A40F090809CF81C29012A00F050
:101CD0008B8001228CF81C29D4F854CA06E0D4F871
:101CE000542AA2EB0C02192A00F28880826912F4AD
:101CF0000042F4D164214FF0220E0C9E01FB0541FD
:101D000081F81DE94FF0100EC1F8006981F81EE955
:101D1000C1F82029A1F80639B1F80639C1F810290F
:101D20009BB2FF2B7BD8B1F8063942689BB2A1F871
:101D30000439DBB25A4947EA03430A4013435A4A7B
:101D40001A4342604FF0640808FB0548B8F80639AA
:101D50009BB2002B00F03B81D8F8DC180BE08B69BC
:101D600013F0200340F0CE80D4F8542AA2EB0C02EA
:101D70000A2A00F2E1808B695B076ED48B69DB066F
:101D8000EDD58B6913F0200309D1D4F8542AA2EBC6
:101D90000C020A2A51D88B6913F02003F5D02023B6
:101DA0001022CA61CB618B699E0701D500238B622B
:101DB0008B69D80703D48B6943F001038B614A68B0
:101DC00064233A4E002003FB0543324020264A603C
:101DD000D3F8202983F81C0942F00402C3F8202913
:101DE00083F81D6983F81E09B4F8583A01339BB291
:101DF000A4F8583A002003B0BDE8F08F64232020F7
:101E0000002103FB0543D3F8202983F81C19024362
:101E1000C3F8202983F81D0983F81E19E4E74368F5
:101E20001F4A13401F4A3B431A43FF23A1F80439BA
:101E3000426087E78AF81C99D6E76422202002FBDB
:101E40000542D2F8201982F81C390143C2F8201942
:101E500082F81D0982F81E39C6E74A6AD8F80039A7
:101E60001A70B8F80639D8F80029013B01329BB244
:101E7000C8F80029A8F80639B8F80439B8F80629CE
:101E8000013B92B29BB2A8F80439002A3FF45EAF3E
:101E9000002B7FF45BAFD8F8DC180FE0F01A0024B9
:101EA000009800FC0024FF810024008200E800FE6E
:101EB000D4F8543AA3EB0C030A2B13D88A6912F016
:101EC0008002F5D0B8F806399BB2FF2B5FD94B687A
:101ED000614A1340614A3B431A43FF23A8F804397F
:101EE0004A6033E76423202003FB0543D3F820191D
:101EF00083F81C290143C3F8201983F81D0983F8CE
:101F00001E2971E78B695A0703D5B8F80439002BED
:101F1000A3D12020524AC8614B68134000224B6075
:101F2000642303FB0543C3F8202983F81C2983F8A5
:101F30001D0983F81E2957E76422202002FB054271
:101F4000D2F8201982F81C390143C2F8201982F80E
:101F50001D0949E7D9F8DC1805E0D4F8543AA3EB99
:101F600008030A2BBED88A6912F08002F5D0B9F8AE
:101F700006399BB2FF2B1AD94B68374A1340374AB0
:101F80003B431A43FF23A9F804394A608EE6B8F8A8
:101F9000063931489BB24A68A8F80439DBB20240DE
:101FA00047EA0343134343F000734B60CEE6B9F8AE
:101FB000063929489BB24A68A9F80439DBB20240C5
:101FC00047EA0343134343F000734B606EE66146F8
:101FD000584650F0CDFE034600287FF405AFD8F8F0
:101FE000DC2820201E4ED06151683140516088F8B5
:101FF0001D0988F81E3964220023012002FB0544D4
:1020000084F81C39F7E6BAF80639DAF8DC189BB21E
:1020100014484A68AAF80439DBB2024047EA03438D
:102020001343114A1A434A6014E64146584650F099
:102030009FFE034600287FF4D7AED9F8DC28202085
:10204000074ED06151683140516089F81D0989F807
:102050001E39D0E700207047009C00FC0000FF0103
:1020600000E800FE009800FC002400822DE9F04109
:102070000468D4E90435A8611A7D1F681F2A49D96C
:10208000203A20212E6801FA02F242F01802FA608A
:102090002A7D1F2A48D9203A202101FA02F242F073
:1020A0001802F2606A6800215868016038461160C1
:1020B000116841F01001116093F80880A26941464F
:1020C00053F02EFA2D7AE2693046294653F028FA69
:1020D000226A63689468184A12F80800515D5A68C9
:1020E0006FF30F0222435A603A5842F001023A500D
:1020F000725842F0010272509A6842F440429A606B
:102100001A6842F001021A601A6842F400721A60FA
:10211000BDE8F08120212E6801FA02F242F0180297
:10212000BA602A7D1F2AB6D8202101FA02F242F0B5
:102130001802B260B6E700BFE8420A08D3B20F2B1C
:1021400021D8124B00B503F17E0E02E00333734534
:1021500016D093F800C08445F8D193F801C08C459F
:10216000F4D102EB42020A48997800EB82037C30FA
:10217000C3F8841000EB820083F87C105DF804FB48
:1021800000205DF804FB0020704700BFCCCD09089B
:102190000000002410B40C4C002304F65C2C01E079
:1021A000152B0CD003EB430201331CF802108142C3
:1021B000F6D1144494F95E0A5DF8044B70474FF071
:1021C000FF305DF8044B7047F01A002430B5124D13
:1021D000002305F6D43C02E001331A2B1AD05CF838
:1021E00033408442F8D10CEBC30EDC009EF804E0CF
:1021F0008E45F1D102EB4202084B254403EB8201EC
:102200007C3395F8D94B03EB8200C1F8844081F808
:102210007C4030BD002030BD78C209080000002499
:10222000F0B1002310B504460E4894F804E000F61F
:102230005C2C01E0152B11D003EB430201331CF899
:1022400002107145F6D183186179206893F95E2AEE
:10225000D3B20F2B02D8BDE81040B7E7002010BD65
:1022600000207047F01A002401380E4B0E4A00EB94
:10227000C000D2F8D81003EB800310B4D3F83C317F
:1022800083B00A4CA34214BF022301231943C2F8AE
:10229000D810D2F8D82013400193019B03B05DF809
:1022A000044B704700000024004402580000024024
:1022B0000138F8B500EBC000124C1D46124B04EB80
:1022C000800417460E46D4F83C01984214BFA12062
:1022D000A02051F0F1F8B4F95201B909C4F84C61E9
:1022E000C4F8545150F04CFCB4F95231002B07DBC8
:1022F00003F01F0001225B090449824041F82320BA
:10230000F8BD00BF000000240000024000E100E032
:102310002DE9F04F002385B0DFF800A34FF001094D
:102320000193B94B0AF1F00BB84FA3F17C080BE015
:10233000019B09F101090AF1280A0BF1050B013390
:10234000062B019300F0F1809AF80030022BEFD1B8
:102350009BF90320511C00F0EB80D2B2944602EBB3
:102360004204A94B9DF8041003EB84040F2A5ED8A5
:10237000A74802E00330B84259D00378002BF9D1C6
:1023800045788D42F6D18578D8F840616068A560BF
:10239000B042257000F04481D8F86461B04200F08A
:1023A0005E81D8F88861B04200F06281D8F8AC61F3
:1023B000B04200F06281D8F8D061B04200F06C8188
:1023C000D8F8F461B04200F08081D8F81862B042C9
:1023D00000F07681D8F83C62B04200F08081D8F8F5
:1023E0006062B04200F07681D8F88432984200F002
:1023F0008C81D8F8A832984200F08181D8F8CC328C
:10240000984200F0A581D8F8F032984200F09A8105
:10241000D8F81433984200F0A781D8F8383398429E
:1024200000F0A881D8F85C33984200F0978101321F
:102430000C34D2B2624599D9002303939BF904204E
:10244000531C79D0D2B2964602EB42046E4B9DF8F3
:10245000041003EB84040F2A5DD86D4802E00330BA
:10246000B84258D00378012BF9D145788D42F6D186
:102470008578D8F840616068A560B04225705FD06B
:10248000D8F86461B04200F0EF80D8F88861B042BB
:1024900000F0F880D8F8AC61B04200F0F880D8F8CD
:1024A000D061B04200F0FD80D8F8F461B04200F095
:1024B0000281D8F81862B04200F0F880D8F83C6287
:1024C000B04200F01781D8F86062B04200F00C8191
:1024D000D8F88462B04200F02481D8F8A83298423B
:1024E00000F01981D8F8CC32984200F02581D8F854
:1024F000F032984200F01A81D8F81433984200F074
:102500004B81D8F83833984200F04081D8F85C33DA
:10251000984200F0358101320C34D2B296459AD2FD
:1025200000220023CAE9042302E705B0BDE8F08FCA
:102530004FF00F0C002212E74FF00F0E002283E73E
:1025400000231E46029306EBC600013608EB80000E
:1025500090F958C1BCF1000FDDD1624680F84431DA
:10256000AC462C4B1546029AC0F848C1134480F87B
:102570005991CAF81430132380F858313046FFF7C8
:1025800073FE039B002BCBD0DAF814402046FDF7F6
:1025900037FDDAF81000FDF733FDDAF81830C168BE
:1025A000DAF80420596240215D60996002F120014F
:1025B0009D631960C3E90355C3E90555C3E9075590
:1025C000C3E90A55C3E90C55A4B1DAF81C3030321E
:1025D000E1681D625962C3E900254FF48032C3E906
:1025E0000255C3E90455C3E90655C3E90B55C3E9D0
:1025F0000D559A620023304607491A46FFF758FEE8
:1026000001238AF80C3093E67C0000244ACE0908A6
:10261000CCCD09083C010024C50900009025002408
:102620001846029300EBC00E013008EB8E0E9EF9A7
:102630005861002E7FF4FBAE029A8EF84431594B5C
:10264000CEF8485113448EF85991CAF8103014232B
:102650008EF85831FFF708FE01230393EEE624209D
:10266000012302901846DDE724201E4602906AE707
:102670004820022302901846D4E76C2003230290DE
:102680001846CFE7022348201E4602905BE703234B
:102690006C201E46029056E79020042302901846B4
:1026A000C0E7042390201E4602904CE70623D82062
:1026B0001E46029047E70523B4201E46029042E7DB
:1026C000D820062302901846ACE7B42005230290D8
:1026D0001846A7E74FF4907002900820A2E7FC206C
:1026E0000723029018469DE74FF490730826029343
:1026F000002328E70723FC201E46029023E74FF41F
:10270000B470022302900A208CE74FF4A2730920D0
:102710000293012386E74FF4B47002230A26029045
:1027200011E74FF4A270092602900CE74FF4D8731A
:102730000C260293042306E74FF4C6730B2602937C
:10274000032300E74FF4D8730C200293042369E7B6
:102750004FF4C6730B200293032363E74FF4077310
:102760000F20029307235DE74FF4EA730D200293D5
:10277000052357E74FF4FC730E200293062351E71D
:102780004FF407730F2602930723DCE64FF4FC7324
:102790000E2602930623D6E64FF4EA730D26029323
:1027A0000523D0E63C010024234B5B68C3F30803F8
:1027B00010B4DBB9EFF31183C3B9204B4FF0E02C19
:1027C0005A6EDCF81800596E8A42F9D1996E884227
:1027D000F6D8DC6E4FF47A7101FB04F3181AB0FBE3
:1027E000F4F05DF8044B01FB02007047EFF3118138
:1027F000102383F312884FF0E0229469136913F4D5
:10280000803F0E4B03D00120C3F86C089469586ECA
:10281000C9B2D3F86C2881F31188D96E4FF47A735A
:10282000024403FB01F0001B5DF8044BB0FBF1F028
:1028300003FB0200704700BF00ED00E0F01A002427
:10284000BE4803780BB90120704743682DE9F04F6B
:10285000002BDFF8109387B0D9F8646018DD00F121
:1028600008050024B649D5F8F430BFF34F8F03F5BF
:102870009072C1F85C3220339342FAD1BFF34F8F8C
:10288000BFF36F8F0134436805F586759C42EADB20
:1028900090F8F815AB4A0491A2FB0612AA4BAB4E76
:1028A0005209DFF8C4A2A3FB0213DB0803EB830386
:1028B000A2EB4303DAB206EB830B06F538730592FD
:1028C000009300239846049B984500F01481DAF8A1
:1028D0001830DAF80470D3E93D45FFF765FF9C49ED
:1028E00099F8AFEB012269180190BEF1540F99F8E5
:1028F000AE0B02FA07F204EB410104EB400301D1F5
:10290000A9F8B60B994240F26A811F88174200F07D
:102910005F815F88174200F070819F88174200F046
:102920006E81DF8808331742ECD11C1B99424FEAB5
:10293000640440F25481281B452828BF452003EB3E
:102940004000834280F04F8100251F46AC46294657
:10295000CDE9028EB3F800E00EEA020E8E451CD1DE
:10296000B3F802E00EEA020E714540F01A81B3F8A6
:1029700004E00EEA020E714540F01581B3F80680BE
:10298000083308EA0208414508D1984209D9B3F84A
:1029900000E00EEA020E8E45E2D00233984200F2C9
:1029A000E580BCF1110FDDE9028E40F21C81DCF103
:1029B000150200F118816749D9F8C00BD1F87C33B2
:1029C0009C4238BFC1F87C43019C231A002B14DBC6
:1029D000614B03449C4201D923460533C9F8C03BEF
:1029E000D1F87C33052B40F20C81053BDBB289F832
:1029F000AE3B4FF0FF33C1F87C333AB105FA02F237
:102A0000CCF1140C012505FA0CF51543534BC5F315
:102A1000C43203EB8202D2F8A40C05F01F0203EBD0
:102A20008202D2F8A41CC5F34412C5F3842503EB3B
:102A3000820241EA0031D2F8A42C03EB850341EA7B
:102A40000211D3F8A43C41EA0321454B81EA11224B
:102A5000D3F81C3A82EA1212013302F00F020F2A55
:102A600040F0A380B1F5803F80F09F80BEF1540F0D
:102A70004FEA111147D03A4AB1F5606FC2F81C3ADB
:102A80004DD0009B998196F858300598834210D01C
:102A9000DBF8082033689B1A33607368DBF830205A
:102AA0009B1A73600023CBF80830CBF8303086F8DF
:102AB0005800336801333360DBF808300133CBF85A
:102AC00008304FF6FF73994207D173680133736082
:102AD000DBF830300133CBF83030009B08F10108CF
:102AE0005C360BF15C0B1433B8F1080F0AF1200AC5
:102AF00000937FF4E8AE0123194A012082F8183BC5
:102B000007B0BDE8F08FB9F8B02BB1F5606F02F1F6
:102B10000102A9F8B02B124AC2F81C3AB1D199F8B7
:102B2000013003EB430309EBC30343445B7C0D2BF0
:102B3000A7D18023009A9377A5E700BF0400002067
:102B400000ED00E01F85EB51CDCCCCCC301800203F
:102B5000C7FFFF7F0000002420A1070078C20908FA
:102B6000FC100020F01A00243C040020A3EB070E08
:102B7000254F33F8021C4FEA6E0E11400EF1010E84
:102B800087FB0E87A7EBEE774FF0010E012FB8BF42
:102B90000127BD40BC44013F0EFA07F73D431F46E5
:102BA000D8E60433FAE60633F8E6BEF1540F04D152
:102BB000B9F8B02B0132A9F8B02B144A4FF6FF71C7
:102BC000C2F81C3AD2F8183A0133C2F8183A5AE758
:102BD00002331C1B99424FEA64043FF6ACAE10B1BD
:102BE000013889F8AE0BBEF1540F7FF476AFB9F817
:102BF000B23B0133A9F8B23B6FE7043395E60633E5
:102C000093E60023F3E600BF56555555FC1000200F
:102C1000264B70B51A785B789A4242D1244E73687D
:102C2000002B22DD06F108000025224CD0F8AC3044
:102C3000BFF34F8F03F1E002C4F8683220339342B0
:102C4000FAD1BFF34F8FBFF36F8F337813B1037F88
:102C5000012B20D042690135716800F58670136838
:102C6000A94243F001031360E0DCFFF79DFD124B26
:102C7000D3F81C4B002C0DDD03F5326303EBC404C9
:102C80001968083333F8042CC8689C4242EA0002F1
:102C9000CA60F5D170BD002380F8FC30FDF7D6F98D
:102CA000D8E756F0CDF80028B8D170BDF01A00244E
:102CB0000400002000ED00E0FC100020800AA0F5D8
:102CC0008010522807D8054B03441B7D0D2B02D8DA
:102CD000034AD05670470020704700BF78C20908E9
:102CE000D8420A0860B182884FF0B0414FF00043EB
:102CF000B2FA82F2D1F88000D3400343C1F88030A9
:102D0000704700BF4FF0B042D2F88030D2F8881040
:102D10000B4003F00103C2F8883023B1024BD3F813
:102D2000C40B036818477047F01A00244FF0B042F4
:102D3000D2F88030D2F888100B4003F00203C2F8BA
:102D4000883023B1024BD3F8C80B0368184770478B
:102D5000F01A00244FF0B042D2F88030D2F8881038
:102D60000B4003F00403C2F8883023B1024BD3F8C0
:102D7000CC0B036818477047F01A00244FF0B0429C
:102D8000D2F88030D2F888100B4003F00803C2F864
:102D9000883023B1024BD3F8D00B03681847704733
:102DA000F01A00244FF0B042D2F88030D2F88810E8
:102DB0000B4003F01003C2F8883023B1024BD3F864
:102DC000D40B036818477047F01A0024F8B54FF089
:102DD000B043D3F88050D3F88820154005F47875B7
:102DE000C3F888507DB1084F0126B5FA85F4C4F1C7
:102DF0001F0407EB840306FA04F4D3F8C40B03683A
:102E00009847A543F1D1F8BDF01A0024F8B54FF06A
:102E1000B043D3F88050D3F88820154005F47C45A2
:102E2000C3F888507DB1084F0126B5FA85F4C4F186
:102E30001F0407EB840306FA04F4D3F8C40B0368F9
:102E40009847A543F1D1F8BDF01A002430B10368CA
:102E500082881B691A4214BF01200020704700BFFE
:102E600010B1036882889A61704700BF18B18388E7
:102E700002681B049361704770B50D4682B004462A
:102E8000164640B101680C4B0C4A0B449B0A02EBFE
:102E90004303B3F8CC0A50F00FFBC5F38101C5F32F
:102EA000411305F01302CDE90016A188206853F004
:102EB00075FB02B070BD00BF0000FEA778C2090814
:102EC00000B1D9E770472DE9F84FC44F6423044699
:102ED00003FB0073D3F8C468002E00F06981D3F8B7
:102EE000CC88B8F1000F04D098F90630002B40F0E0
:102EF0005F81642303FB0473D3F8D05825B195F99F
:102F00000630002B40F05481631CDBB2B8F1000F97
:102F100004D0152288F8073088F8062015B116224B
:102F2000EB71AA714FF0640A308D50F0C5FA294652
:102F30000AFB04FA404655F011FF404607EB0A0928
:102F4000DFF8BC8299F8D63899F8D428002B0CBF4A
:102F50004FF01E0B4FF03E0B5946FFF7B1FF2846CE
:102F60009F4D594699F8D5285544FFF7A9FF4C22A3
:102F70000021284658F008FED9F8C438994A5B6801
:102F80009342C9F8DC38DFF87C9240F0138148F0B6
:102F900055FFD9F82030C3F30213434493F8243D7E
:102FA00003F01F039FED907A9FED905AB0EE084A10
:102FB000D8406423F7EE003A4FF0000C07EE900A79
:102FC00003FB047340F21458F8EE677AB3F8D8A8FC
:102FD000C7EE275A07EE90AA9FED857AF8EEE77ABA
:102FE000C7EE274ADFED837AB0EE007AE5EE877A06
:102FF000A5EE875A25EE844A37EE856A74EEE72AF5
:10300000BAF5C87F0CF1010ED5BF4FF49672782245
:103010006423322307EE90EAD8BF4FF416791344A5
:10302000A2F13202F8EEE76AC8BF4FF4827907EEE8
:10303000903AD4BF41464FF4FA7166EEA56AB8EEF5
:10304000E77AC7EE267A07EE102A01EB0902B8EEFE
:10305000C77A37EE447A77EEE37AFCEEE77A17EE3A
:10306000903AC7EE267AFCEEE77A17EE900A07EE62
:10307000909AB8EEE73A07EE902AF8EEE77A23EE58
:10308000243A83EE277A37EE453A32EEC77AC3EE1A
:10309000267A77EEE37AFCEEE77A17EE901AC7EE1F
:1030A000267A77EEE37AFCEEE77A17EE902A02F1C1
:1030B000020909EB010BB0EE467A07EE90BAF8EE82
:1030C000677AA6EEA77AF4EEC74AF1EE10FA7DDC35
:1030D00043EA00095FFA89F9B9F10F0F78D841EA9C
:1030E00002091FFA89F9B9F1FF0F71D81B05000415
:1030F00003F07F6392B200F47F0003433E4843EA4B
:103100000C7300EA01210B4313436422284602FB9F
:1031100004740027C4F8E0380123C4F8E478C4F844
:10312000E838C4F8EC78C4F8F078C4F8F878C4F853
:10313000FC7853F0E5F994F81D39202BD9B21AD157
:1031400094F81C39012B16D0242384F81D39D4F8A7
:10315000DC381A6822F001021A601A6822F48052E0
:103160001A601A681A601A6842F001021A6084F83C
:103170001D1984F81C79002196F82B004FF000FDF2
:1031800096F82B3001241D4D5A0903F01F0300212E
:1031900004FA03F345F8223096F82A004FF0F0FCC9
:1031A00096F82A305A0903F01F039C4045F8224044
:1031B000BDE8F88F48F042FED9F81C30C3F3021383
:1031C000984498F8243DEBE6F44619E7013170E79E
:1031D000BEF10F0FF8D1002397E700BFF01A0024CB
:1031E000CC230024001C0058286B6E4E00001643B0
:1031F000002474490000704200FFFF0000E100E07D
:1032000078C209080044025808B1002234E6704729
:1032100070B50E4C94F8F865AEB104F587640025DE
:1032200003E001352034B5420DD0237F002BF8D0C8
:10323000E06800220028F4D00135217DFFF71CFE54
:103240002034B542F1D1012070BD00BF0400002040
:1032500070B590F8EE311C09013C082C0DD8194EC0
:10326000054603F00F0336F8140040FA03F2D207C4
:1032700003D595F8F121012A01D0012070BD9A40B3
:103280002644013A104058F02FFE96F8343D0E4A7D
:10329000034402EBC30452F83320A388106918409A
:1032A000ECD0002395F8EF210221204685F8F1317A
:1032B000FFF7E2FDD5F85021136843F008031360CF
:1032C000DBE700BF78C20908601B002438B5BFF3F4
:1032D0004F8F6A4A6A49A2F50353C1F86832203316
:1032E0009342FAD1BFF34F8FBFF36F8F654C94F8C1
:1032F0005528B4F86438022A11D094F85528012AC8
:1033000000F08D80D4F818580C2B0CD8DFE803F0AF
:10331000110B0B0B300B0B0B4D0B0B0B6A0000232F
:1033200084F8663838BD00236B62012384F8553871
:1033300038BDD4F83C08544B544AC36490F8343038
:10334000C263012B00F09780012290F83530934240
:1033500080F8342000F0858000234FF4006280F86C
:10336000343042656B62EB6843F40073EB60DCE77A
:10337000D4F84008444B454AC36490F83430C263E3
:10338000012B61D0012290F83530934280F834202F
:1033900053D000234FF4006280F8343042656B62F2
:1033A000EB6843F48063EB60BFE7D4F84408364B26
:1033B000364AC36490F83430C263012B4ED00122E8
:1033C00090F83530934280F8342040D000234FF4F9
:1033D000006280F8343042656B62EB6843F400634E
:1033E000EB60A2E7D4F84808274B284AC36490F85A
:1033F0003430C263012B1DD0012290F83530934246
:1034000080F834200FD000234FF4006280F834306D
:1034100042656B62EB6843F48053EB6085E7022200
:1034200084F855286EE740F62A0305F14002184952
:1034300047F040FD00236B62ECE740F62A0305F1FC
:103440003802134947F036FD00236B62A8E740F6C7
:103450002A0305F13C020E4947F02CFD00236B6264
:10346000BBE740F62A0305F13402094947F022FD83
:1034700000236B6277E700236B6274E740550124F9
:1034800000ED00E0F01A0024257808087D7808088F
:1034900080340124014B53F82000704750400058FD
:1034A000014B43F8201070475040005819481A4B00
:1034B00001681A4A41F4807130B482B00160D3F8D7
:1034C000F410FF24CA2041F48031C3F8F410D3F87B
:1034D000F41001F4803101915321019D5462506236
:1034E0005162D3F8D030DB010CD40C4B00220C49D4
:1034F0005A659A65DA651A665A669A66196502B05F
:1035000030BC7047126D064B9A42EED102B030BC0F
:10351000704700BF0048025800440258004000585D
:10352000316665422DE9F84FD0F85C710446534B83
:1035300000F59676FDB227F0FF09826800F1E00AF7
:10354000103D4846D2F80080A3FB05352D092946D9
:1035500052F042F8D4F81C210023B2F5807F84F8A1
:1035600020317FD00DD8102A00F084805DD8012A48
:1035700046D0042A16BF6FF400616FF008013C23A7
:103580000EE0B2F5805F71D0B2F5803F3BD0B2F56E
:10359000806F15BF6FF400616FF008013C230423B6
:1035A000324608F11806404656F803C001EA0C01FD
:1035B000F150D4F81CB1594651F0BCFCBBF5807FEA
:1035C0002ED024D8BBF1100F3FD037D8BBF1010F5C
:1035D00002D0BBF1040F34D14FF0080C33685246CF
:1035E0002946484643EA0C0333604023C4F8E830D8
:1035F00051F096FF3B6843F010033B60BDE8F88F45
:103600006FF00801CCE76FF008013C23C8E7BBF579
:10361000805F22D0BBF5803F1AD0BBF5806F10D100
:1036200008F11C064FF0080CD8E7402A15BF6FF4CC
:1036300000616FF008013C230023B1E7BBF1400FAC
:10364000CAD03C364FF4006CC8E74FF4006CC5E7B5
:1036500008F154064FF0080CC0E708F11C064FF4BF
:10366000006CBBE76FF00801042399E76FF4006179
:10367000042395E76FF4006192E700BFABAAAAAA02
:103680002DE9F04F474D85B02B781BB9012005B0CF
:10369000BDE8F08F444B5C6EFFF786F895F8F8357F
:1036A0000193002B00F0C781404B05F5C065404EEB
:1036B0000027A3FB042300955B09A6FB03263D4AD4
:1036C000F60802F2347806EB8606A3EB4606D2F83B
:1036D000483BC11A1346F2B203F6142A08EB8606D9
:1036E00089460392B9F1000F05DB009BD3F8243122
:1036F0004B4500F387814FF4B4732A4A03FB072339
:1037000093F82037002B00F0BF80009D2A48D5F8A1
:103710005C11AB681A68CBB221F0FF01103BA0FB33
:10372000030326481B09C35C0B44A9895C68D36862
:10373000A4B223EA0103C4F11604D360072C40F2BB
:10374000A3801C4A0121D5F86451D2F81C3A8B465B
:10375000AE4602970133C2F81C3A0022286894460C
:1037600014E0BCF1140F2BDC13F1080748BF03F180
:1037700017073B110CEB271C5F1E013102FA03F304
:103780000BFA07F78C4247EA030219D303468C422F
:103790005EF8040FA0EB0303E3D8CCF115034FF060
:1037A000150CE9E704000020F01A00241F85EB51F6
:1037B000CDCCCCCCFC100020ABAAAAAAE8420A08C7
:1037C000BCF1150F029F40F013819F48C2F3842380
:1037D000C2F3441100EB830300EB8101D3F8403DB9
:1037E000D1F8401D1B0243EA011302F01F01C2F38E
:1037F000C43200EB810100EB8202D1F8401DD2F807
:10380000402D0B4343EA023383EA132282EA121269
:1038100002F00F020F2A40F0EB80C3F30F134FF6B4
:10382000FF72934200F0E480B3F5606F00F0EE8029
:10383000AAF80C3098F858200398824210D0B1684A
:10384000D8F80020521AC8F80020D8F80420316BAC
:10385000521AC8F804200022B260326388F8580077
:10386000D8F800200132C8F80020B2680132B260F6
:103870004FF6FF72934207D1D8F804300133C8F8ED
:103880000430336B01333363009C013708F15C086B
:103890005C3620460AF1140AFFF744FE04F5B473BF
:1038A0000093019BBB427FF41DAF684901220023B6
:1038B00081F8182BC1F8483B6549D1F8083691F8D2
:1038C000D8261B6812F0020FD1F81C171A6A0CBF19
:1038D0000A4342EA81021A62019B012B3FF4D6AEF1
:1038E0005B49D1F8703791F840281B6812F0020F3D
:1038F000D1F884181A6A0CBF0A4342EA81021A629C
:10390000019B022B3FF4C2AE5149D1F8D83891F84F
:10391000A8291B6812F0020FD1F8EC191A6A0CBF23
:103920000A4342EA81021A62019B032B3FF4AEAEC6
:103930004749D1F8403A91F8102B1B6812F0020F5A
:10394000D1F8541B1A6A0CBF0A4342EA81021A6278
:10395000019B042B3FF49AAE3D49D1F8A83B91F866
:10396000782C1B6812F0020FD1F8BC1C1A6A0CBF2D
:103970000A4342EA81021A62019B052B3FF486AE9C
:103980003349D1F8103D91F8E02D1B6812F0020F79
:10399000D1F8241E1A6A0CBF0A4342EA81021A6255
:1039A000019B062B3FF472AE2949D1F8783E91F87D
:1039B000482F1B6812F0020FD1F88C1F1A6A0CBF37
:1039C0000A4342EA81021A62019B082B7FF45EAE31
:1039D000204A52F8203C92F8B0001B68D2F8F4104C
:1039E00080071A6A4CBF42EA81020A431A624DE616
:1039F000164AD2F8183A0133C2F8183AAFB14FF666
:103A0000FF7317E7002005B0BDE8F08F12494A7830
:103A100002EB420201EBC2023A44527C0D2A7FF4CF
:103A200007AF80228AF81E2004E7294658220B4857
:103A300058F04CF8E3E719460122044BC3F8481B41
:103A400083F8182B22E600BF78C20908FC1000207A
:103A50000400002004100020F01A0024BC1B0020E9
:103A60002DE9F8432422D0F8505100238168C0F892
:103A7000D02104462A6800F5A87622F001022A60C7
:103A80002B606B60AB604279C0F8D83180F8CC31E4
:103A9000C0F8D031C0F86831C0F8D431C0F8703106
:103AA0009302C0F8541103F48053BC49C0F8583154
:103AB00013038D4203F40053C0F85C314FEA022334
:103AC00003F48063C0F8603100F0AB812379D8073C
:103AD00003F0020100F14081002940F07181C4F837
:103AE000641194F8F0314BB1D4F8783143F0080305
:103AF000C4F878314FF40043C4F8883112F008025A
:103B0000D4F8D03100F06E81002B00F0AD81242379
:103B10003046C4F8D0312B6823F001032B6048F005
:103B200021FD012817D0D4F87831002B40F09F8177
:103B30006B68304623F490436B60AB6823F022033C
:103B4000AB60AB6843F00803AB602B6843F0010344
:103B50002B6051F003FE94F8048018F0010F6FD031
:103B6000D4F82C71002F00F06C8100234FF4807C7E
:103B700004F13C09E7632366E3664846C4E9113370
:103B8000C4E91433C4E91933D4F83431C4F8B83073
:103B90004FF48063E3644FF48033C4E916C353F0F9
:103BA00093F8484646F0E6FFD4F8D431C4F8C891FB
:103BB000202B666741D1E368626998B2EAB3B0FA34
:103BC00080F14909C8B394F8CCC1BCF1010F34D0DD
:103BD0004FF0220CC4F8D811A4F8AC010120C4F8AD
:103BE000D4C1DFF8D0C1C4F8A821C4F878C0DFF888
:103BF000C8C1C4F88C10C4F87CC0DFF8C0C184F818
:103C0000CC01C4F888C094F870C084450CD084F806
:103C1000700094F87100012800F031814FF40063C6
:103C200084F87010C4F890301023C4F8D831002301
:103C300084F8CC312023C4F8D0317B68C4F84431F7
:103C400018F0020F00F08680D4F83051002D00F0FB
:103C5000EC80D4F83821002304F1B407C4F8C03054
:103C60003846C4F8C830C4E92D524022C4F8BC20FC
:103C70004FF48062C4F8C4204FF48032C4E9333377
:103C8000C4E93633C4E93833C4F8D42053F01CF8FF
:103C9000384646F06FFF002840F0A380404B414972
:103CA000414A8D4218BF9D42404801F16001C4F86D
:103CB000C4710CBF01230023C4F8EC60954208BF17
:103CC00043F001033032854208BF43F00103603006
:103CD000954208BF43F0010330328D4208BF43F0E4
:103CE000010301F56871954208BF43F0010302F535
:103CF0005C72854208BF43F0010300F5687095428D
:103D000008BF43F0010330328D4208BF43F0010386
:103D10006031954208BF43F001033032854208BF4D
:103D200043F00103954208BF43F0010330328D4256
:103D300008BF43F00103954208BF43F001033BB9BC
:103D40001B4BEB1AB3FA83F35B09002B00F0AF8037
:103D500000236B60BDE8F8830423C4F8643171B1BB
:103D60000C23C4F86431D3077FF5BBAED4F87831A7
:103D70004FF4803143F00203C4F8801128E0D307E8
:103D80007FF5AFAED4F8783143F00203C4F8783150
:103D90004FF48033C4F88031A3E600BF000C005814
:103DA000100002402800024040000240580002403B
:103DB000B804024005790808397908083D790808EF
:103DC0000823D107C4F864317FF58BAED4F878317D
:103DD00043F00103C4F878314FF40033C4F87C3168
:103DE0007FE6FEE70BB194F8CC21242384F8CC21A4
:103DF0003046C4F8D0312B6823F001032B6048F023
:103E0000B1FB01283FF4A7AED4F87831002B32D1B2
:103E10006B68304623F490436B60AB6823F02A0351
:103E200092E60423C0F8743150E6D4F8DC311A6805
:103E300042F080021A601A6842F040021A60BDE83F
:103E4000F883D4F8DC311A6842F480721A609A68F8
:103E500042F001029A601A6842F020021A601A6861
:103E600042F010021A60EBE684F8CC314FE630469F
:103E700048F076FD5CE6304648F072FDC8E79BB23C
:103E8000484605F1240147F015F800287FF4CCAE30
:103E900084F8CC012B6843F480732B60AB6843F04B
:103EA0000103AB60AB6843F04003AB60C5E66B60F9
:103EB00050E700BF38B50409013C082C18D80E4D56
:103EC00000F00F0335F8140040FA03F212F001027B
:103ED00010D00122254402FA03F3013B184058F0A8
:103EE00003F895F8343D054A034402EBC30038BD9E
:103EF000002038BD104638BD78C20908601B002478
:103F00002DE9F047984D05EB0013D3F8044C002C35
:103F100000F08F80B3F80E7C06464FEA0019384651
:103F20004FF0CAFA01227B0907F01F07023BBA4093
:103F3000082B0FD8DFE813F0BF00C700CF00D70071
:103F4000DF000900E700EF00B7008849CB6F23EAE4
:103F50000203CB6705EB0903013693F8080CF6B2B0
:103F6000FFF7A8FF074610B11223C671837105EB56
:103F7000090393F8090CFFF79DFF824610B1132344
:103F8000C671837105EB090393F80A0CFFF792FFE2
:103F9000804610B11423C67183714D4450462E21C2
:103FA00095F80C2CFEF78CFF95F80D2C40460E2151
:103FB000FEF786FF95F80B2C2E213846FEF780FF82
:103FC00023686B4A23F001039442236033D0694B8A
:103FD0009C423ED1654BD3F8902042F48042C3F816
:103FE0009020D3F8902022F48042C3F89020E36818
:103FF00043F00043E360A36823F4F073A3602368F5
:10400000DA0716D4A1685C4A5C4B0A401343A360EC
:10401000E368DB0042D5E268594B134043F0E863A4
:10402000E360236823F400632360236D23F001031E
:104030002365BDE8F0874D4BD3F8982042F48052B9
:10404000C3F89820D3F8982022F48052C3F898201F
:10405000CDE74C4B9C4213D04B4B9C4263D04B4B17
:104060009C426ED1414BD3F8982042F48012C3F8A1
:104070009820D3F8982022F48012C3F89820B6E74D
:104080003A4BD3F8902042F40042C3F89020D3F882
:10409000902022F40042C3F89020A8E7236843F45C
:1040A00080532360B7E73149D1F89C3023EA0203FB
:1040B000C1F89C304EE72D49D1F8983023EA02032D
:1040C000C1F8983046E72949D1F8903023EA020335
:1040D000C1F890303EE72549D1F8943023EA020335
:1040E000C1F8943036E72149D1F8803023EA020341
:1040F000C1F880302EE71D49D1F8843023EA02034D
:10410000C1F8843026E71949D1F88C3023EA02033C
:10411000C1F88C301EE71549D1F8883023EA020334
:10412000C1F8883016E7114BD3F8982042F40052BA
:10413000C3F89820D3F8982022F40052C3F89820AE
:1041400055E7134B9C427FF452AF03F50C33D3F881
:104150009C2042F02002C3F89C20D3F89C2022F03F
:104160002002C3F89C2042E7F01A002400440258C1
:104170000030014000380040E0FFBF8F0700002002
:10418000FFFF39D8003C004000340140005001409E
:104190000014005808B51D20FFF78CFE10B190F9EF
:1041A000063053B11E20FFF785FE10B190F906309E
:1041B00003B108BD5523C38008BD5523C380F1E773
:1041C000F8B50E4C94F8F875A7B104F5C064C7F1C2
:1041D00009070925013D0FD0A6683079FFF76AFE6F
:1041E00094F8DC10F27908B1FEF746FEAF4204F510
:1041F000B474EFD10120F8BDAB68FFDE04000020ED
:1042000008B549F001FC1B20FFF754FE08B1292333
:10421000C3801C20FFF74EFE08B12923C38052F053
:1042200009FB0B484FF0B8FA0A4B93F8692C012AA6
:1042300001D0012008BD084AD3F8480FC3F8442F25
:1042400052F006F90023054A184682F8233008BDCB
:1042500080030024F01A0024B803002400ED00E0DD
:10426000F8B50446EFF31185502383F31288D0F894
:1042700030311B6803F001031BB1EDB285F31188E7
:10428000F8BDD0F8D021D0F8D4110A4302F02102B1
:10429000212AF2D0D0E90912914250D090B24BD8E5
:1042A000194623691B1A9BB2A162002184F8E01110
:1042B000D4F8D0112029E0D1A1698918DDD0B3FA52
:1042C00083F25209002BD8D094F8CC010128D4D025
:1042D0002120A4F8A6314FF0010CC4F8D821C4F86D
:1042E000D001D4F8C401D4F85061C4F8A011A4F8E6
:1042F000A43184F8CCC160B31B4F90F834E0C7639D
:104300001A4FE64502650764194FC7640AD090F852
:10431000357080F834C0674515D04FF4006380F8DD
:1043200034204365102100222023C4F8D81184F8DA
:10433000CC21C4F8D031A0E7081A83B2B4E7012336
:1043400080F8E03199E706F1280246F0B3FD002835
:10435000E8D100234022326284F8CC31B36843F0C4
:104360008003B36089E700BFDD7808080179080899
:104370003D790808BFF34F8F0549064BCA6802F420
:10438000E0621343CB60BFF34F8F00BFFDE700BF78
:1043900000ED00E00400FA050021032008B5FFF756
:1043A0007FF872B6FFF7E6FF08B51D480023C0F896
:1043B0008430BFF34F8F436923F480334361BFF3ED
:1043C0004F8FD0F8803043F6E074C3F34E3CC3F314
:1043D000C90E4FEA4C1C0CEA0401734641EA837291
:1043E000013BC0F874225A1CF8D1ACF1200C1CF12E
:1043F000200FF0D1BFF34F8FBFF36F8FBFF34F8FFD
:10440000BFF36F8F4369002223F400334361C0F888
:104410005022BFF34F8FBFF36F8F72B6FFF7AAFF23
:1044200000ED00E0800AA0F5801052280CD8074B60
:1044300003441B7D0D2B07D803EBC302044803EB99
:10444000420300EB830070470020704778C20908E0
:104450003C2A002403689B0AA3F58013522B57D8EB
:1044600070B5384C23441B7D0D2B50D840794FF04C
:104470004C0C354C4FF0020E86080CFB034C03EB42
:1044800083000EFA06FEDCF84C5F03EB400030447C
:10449000EE68002942D004EB800C46EA0E06CCF808
:1044A000F414CCF80425EE60EFF31186502282F369
:1044B00012882C2101FB0340D0F8F0244AB3111DCF
:1044C000C0F81425214A03EB8300214D03EB400083
:1044D000800005441030024452F8040F08B108600F
:1044E000011DAA42F8D10022F6B20A6086F31188B3
:1044F0002C2202FB0342D2F81425CAB14C2202FB43
:104500000343D3F84C2FD36843F00103D36070BD4D
:1045100070470E4A01FB03212431D4E726EA0E0638
:10452000EE6004EB8005C5F8F414C5F80425BBE77C
:104530004C2202FB0344D4F84C2FD36823F0010330
:10454000D36070BD78C20908F01A0024E01F00246F
:104550000020002403689B0AA3F58013522B00D986
:1045600070470F4A13441B7D0D2BF9D84FF04C0CAC
:1045700010B40C4C42790CFB03400223D0F84C0FD2
:10458000DA409340C26829B922EA03035DF8044B7C
:10459000C360704713435DF8044BC360704700BFAE
:1045A00078C20908F01A002403689B0AA3F5801357
:1045B000522B11D8094A13441A7D0D2A0CD8407980
:1045C000022307494FF04C0CD8400CFB02128340E9
:1045D000D2F84C2FDB431361704700BF78C2090843
:1045E000F01A002401490248FCF706BCE01F002431
:1045F0000000014001490248FCF7FEBBE01F002417
:104600000000014002494FF08040FCF7F5BB00BFBD
:104610000C20002401490248FCF7EEBB382000249E
:104620000004004001490248FCF7E6BB6420002476
:104630000008004001490248FCF7DEBB902000243E
:10464000000C0040F8B5164D164E2A69EB681A406A
:104650004FF00040B2FA82F3EAB120FA03F3012AE4
:104660006FEA030302EA03012B610A46F2D1D6F88E
:10467000F4758FB1013F0023BFB2C6F8F435D6F808
:10468000F04534B123682046394698476468002CC9
:10469000F8D10022DCE7F8BDEF6ABFB2EFE700BF58
:1046A00000100040F01A002401490248FCF7A4BBA6
:1046B000142100240004014010B5064C064804F201
:1046C0002461FCF799FB04F27C610448BDE81040CA
:1046D000FCF792BBF01A002400040140001C0040CB
:1046E00001490248FCF788BB402100240018004023
:1046F00001490248FCF780BB9821002400200040BB
:1047000001490248FCF778BBC42100240040014065
:1047100001490248FCF770BBF0210024004401402D
:1047200001490248FCF768BB1C22002400480140F4
:10473000800AA0F5801052280ED8084B03441A7D39
:104740000D2A09D8064B4C2101FB0233D3F84C2F1C
:10475000136843F001031360704700BF78C2090873
:10476000F01A00241F4B984210B50ED003F5806359
:1047700098420AD01C4A03F58043984218BF9042E1
:1047800003D003F5806398421BD147F057FB174BCA
:104790001749DC69DA69C4F3022CC2F3022201EB87
:1047A0000C0393F8243D03F01F03D8400F4B11492D
:1047B0001B69C3F3C03342EAC303CB5C03FB00F0C5
:1047C00010BD47F03BFB094B0949DC69DA69C4F3CA
:1047D0000214C2F302120B1993F8243D03F01F03D5
:1047E000D840E3E700000140004001400044025887
:1047F00078C20908C4420A082DE9F04F002391B09D
:10480000AE4C0093AE4BAF4FA3F55E66AC4D4FF090
:104810000009AD4BD5F800A093F8DA224FEA9A23AD
:10482000A3F58013522B00F2D08033441B7D0D2B57
:1048300000F2CB80012A17F903B000F01181022A9F
:1048400002D1BBF1080F3CD14FF000084146584659
:1048500011F026FD11F0ACFD90F900C0BCF1000F85
:1048600018BFBCF1540F14BF4FF0010C4FF0000CF7
:1048700040F0EA8008F104081FFA88F8B8F1100F38
:10488000E4D1009B002B00F0AB808C4A0BE033445A
:104890001B7D0D2B0ED8FB565B450ED002F58672A4
:1048A000944200F0998091680B689B0AA3F58013ED
:1048B000522BECD900235B45F0D14B7969799942B1
:1048C000ECD109F101091C35B9F1080FA1D1009B08
:1048D00004F586740133042B009397D17B4A4FF083
:1048E000010B92F8F83502F5876901330393039BB6
:1048F0005B4567D0744B99F81020D9F80C6093F899
:10490000EE320092002E5DD0704AD6F800A05568B5
:104910006F48B288002D504401924FEA902040F336
:10492000AE80664A002405E0013402F58672AC428E
:1049300000F0A28011688142F6D1604B4FF486727C
:10494000019D02FB0434009B0322C9F80C6089F826
:104950001030019BC9F81840B3FA83F7C7F11F0361
:104960005800C9F80430B27186F807B002FA00F6B0
:10497000A16C0122D4F854C0314302FA00F002FACB
:1049800003F3A164216D0143D4F8AC0021654F49C4
:104990000E7899B2002E00F04E8143EA0C03636555
:1049A000CAF81850FBF77EFB0BF1010B2046FBF712
:1049B0004DFB09F1200940F20113BBF1090F29F861
:1049C000043C94D111B0BDE8F08F013A012A7FF682
:1049D00078AF4FF0000B37E7BCF1000F7FF471AFF9
:1049E000A86800223B4904E001320C31102A00F093
:1049F00088834B689842F7D152B269795046FDF7E7
:104A0000E5FB354A4068002351680133884208D0ED
:104A1000102B02F124023FF454AF51680133884255
:104A2000F6D1DBB22D4A013B03EBC30302EB830358
:104A300093F95831002B7FF444AFC9EBC909204BDF
:104A400003EB8903A36042E7009B002B7FF41DAFBB
:104A500009F101091C35B9F1080F7FF4DAAE36E728
:104A6000BBF1010F3FF4F0AE09F101091C35B9F1BA
:104A7000080F7FF4CEAE2AE7042C00F049824FF4F1
:104A80008671124A01FB052211690491002900F088
:104A90000483906001304FF054019C46C4B20D482D
:104AA00082F8101182F811416A1C08494A60049A80
:104AB0001168976802915179002216E00C000020DD
:104AC00058D00908D8420A08E82B00240400002026
:104AD0000000FEA77C0000243C010024000000240C
:104AE00001320C30102A00F00C8343689F42F7D14A
:104AF00052B20298CDF814C0FDF768FB944B4FF406
:104B00008672DFF87C8202FB05310022059B0132B0
:104B1000D0E90170C1E9077041464868874208D072
:104B2000102A01F124013FF44DAF48680132874259
:104B3000F6D1D2B28749013A02EBC20201EB8202FE
:104B400092F9581100297FF43DAF4FF4867182F835
:104B500059410693542401FB05F37F4882F85841DC
:104B60009A107E49059300FB02F201F560747848C3
:104B7000C2EBC20C02EBC202184401EB4C1104EB75
:104B80004212C0F80CA0C0F8B410C0F8FC203322C8
:104B9000C0F8B8208C22C0F80021714A0298D418BD
:104BA000FFF7E0FD069B062B00F0B981072B6D494E
:104BB0006D4B6E4A18BF1A466D4B18BF0B464FF42B
:104BC0008671DDF808A0B0FBF3F3B0FBF2F2013B15
:104BD0005F48013A01FB05019BB2A1F8BC20A1F896
:104BE00074302366059B03F1580100F10803504619
:104BF00019440023A4F858306366E36550F018FBAD
:104C0000DAF8003043F08003CAF80030049B5B7987
:104C10001A4606930C2A1CD8DFE812F003021B0088
:104C20001B001B00DD011B001B001B00BB011B0048
:104C30001B001B009601C7F12F072D0402FA07F392
:104C4000324643EA0C036365CAF81850FBF72AFAA8
:104C5000AAE63F4A4FF4867302984FF0000A03FB1E
:104C600005230222CDF828A059690368079123F093
:104C70000103CDF834A0CDF83CA003606023089375
:104C80004FF480730E93012309930A23CDE90B326D
:104C900008AA50F04FF90799B1F5807F00F02882FB
:104CA00040F24081B1F5805F00F00E82B1F5803FA7
:104CB00000F00482B1F5806F15BF4FF40063082344
:104CC0004FF03C0A4FF0040A029A183252F80A10C8
:104CD0000B4342F80A30049B1879002840F0CB813E
:104CE000029A136843F0010313600023D8F80420EC
:104CF0000133974200F0BC81102B08F12408F5D154
:104D00004FF0FF330027134A03EBC30302EB830387
:104D1000D3F83C01174B984214BFA120A0204EF0BD
:104D2000CBFB069A0C2A00F2A081134B03EB420343
:104D3000B3F8C0CE4FF48673054A104803FB052331
:104D4000DDF808E000F53261A3F818C0002320E088
:104D500004000020000000246B4CA407802C0124D8
:104D60000C000020D0DD06004495080010552200FC
:104D700040771B000000024078C20908FC100020A8
:104D80003C010024964500F09D810133042B00F086
:104D9000BB8151F83320002AF4D1D0F81C2B01320A
:104DA000C0F81C2B00EBC300029ADB00C0F8202BDC
:104DB00019443846234690228F884CEA070C002776
:104DC000A1F804C0C349FDF773FA4FF48673C24AD1
:104DD00040214FF4403CC14803FB052A4FF4805268
:104DE000DAF81C502B6843F010032B602B6843F05B
:104DF00014032B60C4E91F77C4E92777C4E9297736
:104E0000DAF82030A167E9B2C4F89430069310397B
:104E10004FF48063C4F898C0A0FB01014FF4804CAC
:104E2000C4F88430DAF8B8000909059BC4F890008A
:104E300025F0FF00DAF80C80C4F8882008F1180289
:104E40000491029008F11008226703F17002A44B4C
:104E50001A44DAF8B430C4F88CC0636750F060FBD1
:104E6000D5F800C0059BC4F820C0D5F814C003F1E4
:104E7000B8029B4BC4F824C0D5F804C01A44069B62
:104E8000C4F828C0D5F808C00499C4F82CC0D5F8D7
:104E90000CC0C4F8DC304FF48063C4F8C870C4F8A8
:104EA000CC304FF40033C4F830C0C4F8E03002987E
:104EB000C4E93077C4E93977C4E93B774FF4006738
:104EC000DAF80031C4F8B880C4F8D0704FF48047E5
:104ED000C4F8D830DAF8FC30C4F8D470C4F8BC3068
:104EE00050F01EFB2B68D6F800A063636B69A363C8
:104EF0006B68E363AB682364EB6863642B6843F01F
:104F000010032B602B6843F014032B60B5881AE55F
:104F10000323744A82F8EF3211B0BDE8F08F724A71
:104F2000724B4CE6102900F0E98000F2BD800129A7
:104F300000F0E280042915BF4FF4006308234FF00E
:104F40003C0A4FF0000ABFE602984FF486726249AD
:104F50004FF0020A036802FB05124FF4805123F060
:104F60000103516108AA036000230A930D930F9374
:104F7000602308934FF480730E93012309930A234F
:104F8000CDE90B3A4FF0D6FF4FF0040A4FF400631F
:104F90009AE602984FF486724F494FF0020C03686C
:104FA0004FF0040A02FB05124FF4807123F0010355
:104FB00051616022036000230E910A930D930F93B9
:104FC0000123CDE908230A2308AACDE90B3C4FF0C1
:104FD000B1FF082378E602984FF486723E494FF0FD
:104FE000000A03684FF0020E02FB0512102123F0A5
:104FF0000103CDF828A0516108AA03606023CDF811
:1050000034A008934FF48073CDF83CA00E93012395
:1050100009930A23CDE90B3E4FF08CFF4FF4006358
:1050200052E602984FF486722B494FF0000A03684B
:105030004FF0020E02FB0512012123F00103CDF80F
:1050400028A0516108AA03606023099108934FF4D6
:105050008073CDF834A00E930A23CDF83CA0CDE99F
:105060000B3E4FF067FF08232EE64FF0000C61E681
:10507000DFB27B1E47E6FEF71DFF824638B1049B78
:105080000221DA79FDF7F8FE5423AAF80630029AD5
:10509000536C43F40043536422E60223114A82F81E
:1050A000EF3211B0BDE8F08F402915BF4FF4006317
:1050B00008234FF03C0A4FF0000A05E608234FF0A2
:1050C0003C0A01E6DB0073E64FF400634FF0040A8C
:1050D000FAE500BF0100000004000020ABAAAAAA64
:1050E0000C000020E82B0024882A1100A0BB0D0032
:1050F00008234FF0040AE7E50823E5E54FF40063D1
:10510000E2E500235B68FFDE00239B88FFDE00BF33
:105110002DE9F04FB04D8FB095F8F082B8F1000F47
:1051200003D100200FB0BDE8F08F00222F214046B0
:1051300011F094F906460028F3D090F80590A74F97
:10514000D0F800A0A7F86498FDF76AF80028E8D026
:10515000D0E901430193002CE3D0DFF8B8B200227C
:10516000594601E0102ADCD04B68013224319C42C0
:10517000F8D1D2B29A4B013A02EBC20203EB82029F
:1051800092F95831002BCCD12F2150460293A2F82E
:105190005811C7F818A8FFF7E5FA924A029B904207
:1051A00080F0FA801A460123039350460292FFF7DB
:1051B000D9FA029A039BC7F81C288B49B0FBF3F27B
:1051C000120A8A48A1FB02210022C7F82828C7F842
:1051D00020280A090909A0FB0202C7F8241852086E
:1051E000A5F8F4225200A5F8F22297F8552802F00B
:1051F000FF01002A00F0DE80022250467C4987F839
:10520000552847F0F1F80122404687F8602887F8D2
:10521000562887F8572887F8582887F8592887F894
:105220005A2887F85B2887F85C2887F85D2887F874
:105230005E2887F85F2887F85528FEF73BFEC5F8FB
:10524000F80228B12F21C1804E21F279FDF714FE1A
:10525000684A0021019B4FF4806CC5F80813B9F12E
:105260000C0FC5F81813C5F82013C5E9BF43C5E9ED
:10527000CA11D2F8D80040F00100C2F8D800D2F824
:10528000D80000F0010004900498D2F8D80040F053
:105290000200C2F8D800D2F8D82002F0020205922B
:1052A000059A4FF04002C5F804234FF48052C5E937
:1052B000C3C24FF48042C5F814234FF40032C5F83E
:1052C0001C234FF00302C5F8242376D84A4A02EB88
:1052D0004902B2F8DC8EC246484A08F1080848493B
:1052E000C5F8342307EB8802C2F818185946002283
:1052F0004B68013224319C4262D0102AF8D14FF021
:10530000FF32374B02EBC20203EB8202D2F83C01C0
:105310003C4A904214BFA120A0204EF0CDF80022BC
:10532000DBF8043001320BF1240B9C424BD0102AE5
:10533000F6D1002007EB8807534660223249FCF77C
:10534000B7FFD7F8180845F015FC00287FF4E9AE40
:10535000B479002760260C9063004A4606A92748C6
:1053600003F002030893E300CDE9066703F00803A6
:10537000002600270993CDE90A674DF075F800284B
:105380007FF4CFAEA30749461C481ED547F0A0F8CE
:10539000B0FA80F04009C5E65046FFF7E3F91B4A32
:1053A0001B490244A1FB0212920D531E9AB2531CD8
:1053B0000393FAE687F854181EE78A4688468BE777
:1053C000D2B2013A9DE7D0B2B4E746F081FFB0FA1D
:1053D00080F04009A6E600BFE82B0024F01A002464
:1053E00000000024006CDC02598B4F01ABAAAAAA72
:1053F0000C2300240044025878C209080823002422
:10540000E42E002400000240D502000000366E01A8
:10541000819F5E163C010024830AA3F58013522B62
:1054200000D970472DE9F0410F4C23441E7D0D2E0D
:1054300018D80E4C4FF04C080139154608FB0647AA
:1054400089B2C7F8581FFFF78DF907F57561B0FBF2
:10545000F5F2013AD7F84C0FC7F8502FBDE8F041EC
:1054600046F0C2BFBDE8F08178C20908F01A0024F6
:10547000830AA3F58013522B70D82DE9F043734DA6
:1054800085B02B441E7D0D2E65D84C23704F904661
:10549000044603FB06F907EB0905D5F84C2F8242B9
:1054A00059D00139C5F84C0F89B2C5F8581FFFF71C
:1054B00059F909F1080307F64C7100220B44C5F8AD
:1054C000542FB0FBF8F00138C5F8500FC3E90222A1
:1054D00095F8893F03F0FF02002B40D04C250223B2
:1054E00005FB061105FB06750431D5F84C8F85F8D0
:1054F000893F404646F078FF012385F8943F85F8C0
:105500008A3F85F88B3F85F88C3F85F88D3F85F87D
:105510008E3F85F88F3F85F8903F85F8913F85F85D
:10552000923F85F8933F85F8893F4A4B9C4219D0BA
:10553000B4F1804F16D0A3F57C439C4212D003F502
:1055400080639C420ED003F580639C4260D003F5DB
:1055500078439C425CD005B0BDE8F083704785F885
:10556000882FBBE74C2303FB067393F8882F012A8F
:10557000F1D0022283F8892F374AD8F808100A4060
:10558000C8F80820012283F8892F002283F8882F89
:1055900000224C232F4903FB067303928845CDE973
:1055A00001224FF0020283F8892FD8F80420D8F89E
:1055B000083028D001F58061884524D022F070029F
:1055C000C8F80420254A90450DD0B8F1804F0AD084
:1055D000234902F50062904518BF884503D002F5C3
:1055E0004062904503D123F08003C8F808304C2373
:1055F0000121002203FB067383F8891F83F8882F9B
:1056000005B0BDE8F08317491140C8F80410EAE777
:105610004C2303FB067393F8882F012A9BD00222A8
:1056200083F8892F0C4AD8F808100A40C8F80820D7
:10563000012283F8892F002283F8882F0A4B9C428D
:10564000A6D003F578439C42A2D084E778C209082B
:10565000F01A0024000001408800CEFF0004004042
:10566000000800408FFF0FFF000C00402DE9F041C3
:105670000468A30AA3F58013522B04D82D4D2B44A4
:105680001E7D0D2E01D9BDE8F0812046FFF7F0FE0A
:105690004C22294B02FB063393F8892F012A10D0A4
:1056A0000023264951F8332094421CD001330E2B9D
:1056B000F8D1012100204DF063FA214B01221A603C
:1056C000E1E70221D3F84C2F83F8891F1D4B916825
:1056D0000B40062BE4D0B3F5803FE1D0136843F0D4
:1056E00001031360DCE705EBC3050126144F95F8B1
:1056F000624A314604F01F0520464DF041FA1B2C4A
:105700004FEA541806FA05F547F8285009D02E2C10
:10571000B9D131462C204DF033FA4FF480537B60E1
:10572000B1E7314619204DF02BFA4FF000733B6082
:10573000A9E700BF78C20908F01A0024D4CC0908F0
:1057400000E100E00700010037B590F86738044633
:10575000032B2FD10023204D8DF807309DF8073003
:1057600094F868289A4201D803B030BD9DF80730FC
:1057700005EBC30393F878338BB181F0010383B158
:105780009DF8073005EBC303D3F87403FDF768FBFE
:105790009DF807300133DBB28DF80730DEE70B46AA
:1057A000EDE79DF8073005EBC303D3F87403FDF76D
:1057B0005DFBEDE7D0E910039B7903F0010399420B
:1057C00004D003B0BDE83040FDF74ABB03B0BDE8EC
:1057D0003040FDF74BBB00BFE82B002438B5044632
:1057E00000790D4650B1FEF765FB08B10323C38075
:1057F000E2792946BDE83840FDF762BB38BD10B5F7
:1058000004462221FFF7EAFF2046FEF7CDFE2046A0
:105810000121BDE81040FEF79DBE10B504460121F0
:10582000FFF7DCFF00212046BDE81040FEF792BEE6
:1058300038B510F8133CA0F66C041BBB94F858382C
:105840008BBBD4E909239A421CD05A1CA169A262DD
:10585000CB5C21695B008A4228BF002243F40073BD
:10586000A262A4F85C380A2384F85A38012384F829
:10587000583894F86738012B01D0042B02D1606CA2
:10588000FFF7CBFF94F85438002B6DD194F85538BE
:105890000133DBB2092B84F8553825D12046BDE809
:1058A0003840FAF7D7BC94F95A586DB1B4F85C187F
:1058B000013D20464B0801F00101A4F85C38FFF7D8
:1058C00043FF84F85A58DDE7D4E9092384F858588F
:1058D0009A42D7D194F86738012B01D0042BD1D14B
:1058E000606CFFF78CFFCDE70A2B3DD194F8573859
:1058F0002BB9B4F85E3843F00103A4F85E3823797D
:10590000D9070AD5B4F85E08820501D4C30718D4B4
:10591000B4F864380133A4F864380122002384F811
:10592000542894F8572884F85538012A1CD16179F5
:10593000606C84F8573801F00101BDE838404BF045
:10594000C5BFE36AC0F3470013B1216B9847E4E792
:10595000E3696269D054E369E2680133B3FBF2F1B1
:1059600002FB1133E361D8E738BD00BF2DE9F043F6
:10597000BFB0BFF35F8FA24A0020516A03460446BE
:1059800021F4803151620146C2F89400C2F8983087
:105990000133C2F89C10112BC2F8A010F6D10523D8
:1059A000C2F89430536A43F480335362BFF34F8F8D
:1059B000BFF36F8F9348944A9449121A56F086F8B1
:1059C0009348944A9449121A56F080F8934BDA6D32
:1059D000042A00F0FB8005D8012A00F07283022A15
:1059E00000F08583864A00238D4C0120D2F8881070
:1059F0008C4E41F470018C4DC2F8881020602361F8
:105A0000216841F080012160216801432160216803
:105A100041F480312160216841F480512160A3610B
:105A2000E3612362A362E36223636363A363E363CB
:105A300023646364216821F4802121607B4923660B
:105A4000C1F808014FF000614FF6FF00784B9160FC
:105A5000D16801400B43D36046F0CEF9A3690246FA
:105A60000F20C3F30323A169334493F8243D03F0CB
:105A70001F0322FA03F3C5F8003444F0F9FC6D4A21
:105A8000D36813F0040FD36840F0A2806A4B002162
:105A9000684A0591D96A21F00101D962DB6A03F0F5
:105AA00001030593936943F440439361936903F4BD
:105AB00040430593059B93699B04FCD54C22002130
:105AC0000EA85E4C56F060F85D4A42F2030312687D
:105AD000B3EB124F4FF000030893A4F1140308BF77
:105AE0001C46E268002A4DD0534B5249D86A20F038
:105AF0000100D862DB6A03F0010308938B6923F489
:105B0000404313438B618B6903F440430893089B24
:105B1000484A93699F04FCD5414B4FF440374948AC
:105B20000321D3F8E02042F08002C3F8E0200122F4
:105B3000D3F8E03003F080030793079B87610D9B48
:105B400000910193002350F029FD022322690EA841
:105B5000CDE91733A3781E9201221993A3881A93D3
:105B6000A3791B93E3791C93237A1D9300231F933E
:105B70004FF48033CDE90E2345F086FE03283BD059
:105B800098B1FEE72B4A2C4B916941F44041916159
:105B9000926902F440420892DA6A42F00102DA6243
:105BA000DB6A03F001030893B1E7274B1A6812F090
:105BB0000E0F4DD11A6822F00F0242F002021A6055
:105BC0001B6803F00F03022B42D0FEE7DC6509E7F8
:105BD00023F007031D4C43F00203D360D4F8541A9A
:105BE00006E0D4F8543A5B1AB3F57A7F3FF64EAF2D
:105BF00053689804F5D549E772B6FEF7BBFB00BFC2
:105C000000ED00E000000000683E00005CD30A08E0
:105C100000000020040000204E370B080040005810
:105C20000044025878C20908000000240080005196
:105C30000003FA050048025800040058EC03002451
:105C40000010005C001C025800200052F01A0024D2
:105C50006E4A936903F070033F2B05D8936923F0D4
:105C6000700343F040039361684AD36903F0700303
:105C70003F2B05D8D36923F0700343F04003D36171
:105C8000624AD36903F4E063B3F5806F05D2D36948
:105C900023F4E06343F48063D3615C4A136A03F046
:105CA00070033F2B05D8136A23F0700343F04003C1
:105CB0001362564B9A69100705D49A6922F00F02B5
:105CC00042F008029A61514A936923F47063936128
:105CD000136899017FF579AF136941F288304C4C14
:105CE00023F0070343F003031361D4F8541A05E0CB
:105CF000D4F8543A5B1A834200F29B81136903F093
:105D00003803182BF4D1936903F00F03082B05D93E
:105D1000936923F00F0343F0080393613D4A13682E
:105D200003F00F03022B0BD9136823F00F0343F08A
:105D300002031360136803F00F03022B7FF445AFD7
:105D4000324A936903F07003402B05D9936923F01D
:105D5000700343F0400393612C4AD36903F070034E
:105D6000402B05D9D36923F0700343F04003D3617E
:105D7000264AD36903F4E063B3F5806F05D9D3698C
:105D800023F4E06343F48063D361204A136A03F091
:105D90007003402B00F245811C4F46F02DF803465E
:105DA000D5F80404BA69B969C2F30322164496F817
:105DB000242D02F01F02D340C5F8003444F058FBF4
:105DC000002840F07D811023159017900EA80E93A7
:105DD00045F05AFD002840F023813B680E4A43F00D
:105DE00080033B60D7F8F43043F00203C7F8F43087
:105DF000D7F8F43003F002030493049B136A43F0D2
:105E000001031362054BD4F8541A0CE00044025805
:105E1000F01A0024002000520004005800E20400A0
:105E2000013B3FF4E9AED4F8542A9142F8D0D4F8BB
:105E3000542AD4F8543A9B1A0A2BFAD9AF4C4FF48F
:105E400080224FF440130EA80E924FF000082F93BB
:105E50004FF05AFDD4F8EC3041F20302A849032672
:105E600043F002030EA8C4F8EC30D4F8EC3003F091
:105E700002030393039BD4F8943043F00203C4F865
:105E80009430D4F8943023F00203C4F894300B68B3
:105E90009C49B2EB134F9C4B9C4A28BF0A465A6060
:105EA0001A6822F47C5242F400521A601A6842F0D6
:105EB00060021A600E96CDE92B884FF025FD4FF455
:105EC000E0430EA8CDF8E4800E93CDE925884FF08D
:105ED0001BFD18230EA8CDF8B8800E93CDF8CC800A
:105EE0004FF012FD4FF400230EA80E934FF4003331
:105EF00036934FF009FDD4F8E0304FF480718448B8
:105F000043F00103C4F8E030D4F8E03003F00103BB
:105F100009934346099A0222CDE9006850F03EFBFE
:105F200023694FF400717B4823F0FE7343F08873BC
:105F30002361D4F8E03043F00403C4F8E030434672
:105F4000D4F8E02002F004020692069A0222CDE97B
:105F5000006850F023FB236923F07E4343F0FC43A9
:105F6000236145F049FF6C4B6C4A4146C5F800047B
:105F70001846D21A55F008FE69486A4A6A49121A48
:105F800055F0A4FDBFF35F8F684D4646684C01276E
:105F90006B6A23F480336B62C5F8948023E0002998
:105FA00046D0D4F80090637A103414F8060C1B061F
:105FB00043EA007343EA410314F8051C43EA8143B2
:105FC00014F8041C43EA414314F8031CC5F8986014
:105FD000013643EA0143C5F89C90032E43F00103C8
:105FE000C5F8A03026D06368217A002BD7D0D4F82A
:105FF00000900029D7D129F01F01A3EB0108B8F1C7
:10600000200F38BF4FF02008404655F09DFD431E3D
:10601000014607FA03F0804508BF1946C9B2C2E736
:10602000FEE7136A23F0700343F040031362B3E604
:10603000FEE7CAE50523C5F894306B6A43F4803364
:106040006B62BFF34F8FBFF36F8FBFF34F8FBFF301
:106050006F8F0022C5F85022BFF34F8FBFF36F8FB1
:106060006B6943F400336B61BFF34F8FBFF36F8FE6
:10607000C5F88420BFF34F8FD5F8805043F6E07603
:106080002A49C5F34E34C5F3C905640104EA060084
:106090002B4640EA8372013BC1F86022F9D2203CD2
:1060A00014F1200FF2D1BFF34F8F4B6943F48033CB
:1060B0004B61BFF34F8FBFF36F8F3FB0BDE8F083ED
:1060C00083E50E4A02201B49D865D2F8F430034319
:1060D000C2F8F430D2F8F43003400E930E9AD1F89F
:1060E000003883F30888D1F804389847FEE7042184
:1060F0000320FDF7D5F972B6FEF73CF900440258CB
:106100000010005C7FBB2200008400407FBB223077
:10611000000002580008025800EA0024A0EA002407
:1061200040E6002400EA002452370B0800ED00E0AE
:10613000080400240090F01F10B4EFF31182102324
:1061400083F312880B4B4FF0E0200024D2B2596E3B
:106150000131596681699966C3F86C48016982F317
:106160001188D3F8542A5DF8044B0132C3F8542A3D
:10617000704700BFF01A002410B4EFF31181102310
:1061800083F312884FF0E0229469136913F4803F7F
:106190000C4B03D00120C3F86C089469586EC9B247
:1061A000D3F86C2881F311880244D96E4FF47A70C9
:1061B00000FB01F31B1B5DF8044BB3FBF1F300FB89
:1061C00002307047F01A00242DE9F047DFF8908084
:1061D000FCF7EAFA4FF4867900210646D8F8045015
:1061E0001D4F002D2DDD00231C4609FB03820133CA
:1061F00092F80521AB4244EA0204F6D121435FFA4A
:1062000081FA7B68C3F30803C3B9EFF31183ABB919
:10621000FAF77AF8801BB0F5FA6FCCBF002104F0D2
:1062200001010029DDD1BAF1000F04D00B4B93F826
:10623000AF2B542A08D05046BDE8F087FFF79CFFEB
:10624000E8E78A460024DCE7B3F8B42B5046013275
:10625000A3F8B42BBDE8F08700ED00E0F01A0024AD
:10626000040000202DE9F8430546254EFCF79CFA72
:106270001027244B04464FF0E02C4FF47A7E4FF069
:1062800001087268C2F30802CAB9EFF31182B2B909
:106290005A6EDCF81800596E8A42F9D1996E88421C
:1062A000F6D8D3F86C900EFB09F1091AB1FBF9F19D
:1062B0000EFB0212121BAA42E3D3BDE8F883EFF3F0
:1062C000118287F31288DCF81800DCF81010C9037B
:1062D00003D5C3F86C88DCF81800D3F86490D2B208
:1062E000D3F86C1882F311884944D3F86C900EFBF4
:1062F00009F2121AB2FBF9F20EFB0122DAE700BF33
:1063000000ED00E0F01A00242DE9F0473A4B471E5B
:106310003A4D10264FF0E0204FF47A7C4FF0010800
:106320006A68C2F30802002A52D1EFF31182002AF0
:106330004ED15A6E8469596E8A42FAD1996E8C4256
:10634000F7D8D96E0CFB01FEAEEB040EBEFBF1FEDE
:106350000CFB02EE6A68C2F30802E2B9EFF31182A5
:10636000CAB95A6E8469596E8A42FAD1996E8C42C2
:10637000F7D8D3F86C900CFB09F1091BB1FBF9F1CC
:106380000CFB0212A2EB0E02B2F57A7FE2D3013FC0
:10639000C6D2BDE8F087EFF3118286F312888469D4
:1063A0000169C90302D5C3F86C888469D3F864A075
:1063B000D2B2D3F86C1882F31188D3F86C905144A0
:1063C0000CFB09F2121BB2FBF9F20CFB0122D9E71C
:1063D000EFF3118186F3128884690269D20302D532
:1063E000C3F86C888469D3F864E0C9B2D3F86C2828
:1063F00081F311887244A4E7F01A002400ED00E054
:10640000154C08B5D4F8B43394F8BA03ABB91420DA
:10641000FFF77AFF00BFD4F8B4335BB1196894F882
:10642000BA239B8809690B4012B91BB1FDF7B4FF71
:10643000002BFBD0FAF76AFBECE719689A880B6926
:10644000134020B1002BE2D10B691340FAE7002B77
:10645000DDD00B691340FAE7E82B00242DE98848CA
:10646000431C0A25944C4FF01008944E5FFA83FBAE
:1064700001274AF083FE4FF4FA7C4FF0E0204FF4FE
:106480007A717368C3F30803002B40F0CE80EFF3FA
:106490001183002B40F0C980D4F864E08369626EF8
:1064A0009645F9D1A26E9342F6D8D4F86C9001FBD0
:1064B00009F2D21AB2FBF9F201FB0E227368C3F3A0
:1064C0000803002B40F0D580EFF31183002B40F040
:1064D000D080D4F864E0D0F81890636E9E45F8D16F
:1064E000A36E9945F5D8D4F86CA001FB0AF3A3EB91
:1064F0000903B3FBFAF301FB0E339B1AB3F57A7F62
:10650000DCD3BCF1010CBCD158464BF009F84FF478
:106510007A7C4FF0E02061467368C3F30803002BD8
:106520003ED1EFF31183002B3AD1D4F864E08369B4
:10653000626E9645F9D1A26E9342F6D8D4F86C906B
:1065400001FB09F2D21AB2FBF9F201FB0E227368C9
:10655000C3F30803002B46D1EFF31183002B42D184
:10656000D4F864E0D0F81890636E9E45F8D1A36E1D
:106570009945F5D8D4F86CA001FB0AF3A3EB090305
:10658000B3FBFAF301FB0E339B1AB3F57A7FDED32C
:10659000BCF1010CC0D1013D7FF46BAF4BF032FC7C
:1065A000EFF3118288F31288D0F818E00369DB0357
:1065B00003D5C4F86C78D0F818E0636ED2B2D4F882
:1065C0006C9882F311884B44D4F86C9001FB09F26B
:1065D000A2EB0E02B2FBF9F201FB03227368C3F3D4
:1065E0000803002BB8D0EFF3118388F31288D0F89A
:1065F00018A0D0F810E01EF4803F03D0C4F86C78E7
:10660000D0F818A0D4F86490DBB2D4F86CE883F327
:106610001188CE44D4F86C9001FB09F3A3EB0A0374
:10662000B3FBF9F301FB0E33AEE7EFF3118288F30E
:106630001288D0F818E00369DB0303D5C4F86C783E
:10664000D0F818E0636ED2B2D4F86C9882F3118857
:106650004B44D4F86C9001FB09F2A2EB0E02B2FBA2
:10666000F9F201FB03227368C3F30803002B3FF424
:106670002BAFEFF3118388F31288D0F818A0D0F86D
:1066800010E01EF4803F03D0C4F86C78D0F818A056
:10669000D4F86490DBB2D4F86CE883F31188CE446C
:1066A000D4F86C9001FB09F3A3EB0A03B3FBF9F3F5
:1066B00001FB0E3321E700BFF01A002400ED00E0DB
:1066C0000246074B02209A4208D801335B0840007B
:1066D0009A4280B202D2FF28F8D97047704700BFB3
:1066E0007FF0FA0211F001010ED170B590F8285038
:1066F00082B00446012D08D0C368B3F1807F01D970
:106700000123037702B070BD70470B4B466AD3F884
:10671000BC03FFF7D5FFE368B080B3F1807FF1D908
:106720004FF0B70C0A4630462B4601A925778DF865
:1067300004C03FF0E5FBE5E7E82B00242DE9F0413C
:106740001F46436A94B01446064618680D4651F039
:10675000CFFB0B940022274C069204F590738DF822
:1067600020201392009304F5A0730C970193022349
:10677000CDE9092202930123CDE90E22CDE91022B1
:106780001D4A8DF80C308DF834308DF84830049265
:1067900004F58072337F05921A1D07922BB32B0EDE
:1067A00004F5817404F8013C2B0CA570DFF84C80D3
:1067B0002D0A23706570D8F8BC03FFF781FF746A57
:1067C000737FA080A3B1694620463FF0DFFB746A67
:1067D000206851F08DFBD8F8C003FFF771FF034626
:1067E0003846A38014B0BDE8F08104F20114DBE761
:1067F00005A9E9E740E60024410A0408E82B002443
:106800002DE9F0470546086888B00C464FEA902C01
:10681000BDF84080ACF5801C9DF844A0BCF1520F3F
:1068200058D819462E4B63441E7D0D2E52D806EBC8
:10683000C6032C4F06EB430307EB8307FEF718FE56
:1068400094F80590A379BAF1000F01D083F0010309
:106850005A004FF48071DB00384602F00202CDF896
:10686000088003F0080303924A46049360230193CF
:106870004FF40073CDE90613002301A905934BF0F3
:10688000F3FDA379384649469F0726D445F020FDFD
:106890004C22154B02FB063393F8892F012A10D1A5
:1068A0000221D3F84C2F83F8891F104B91680B40BD
:1068B000062B06D0B3F5803F03D0136843F00103E5
:1068C00013602168637901F1340269600021D018F6
:1068D0002860D15008B0BDE8F08745F0F9FDD7E752
:1068E00078C209083C2A0024F01A0024070001009D
:1068F00010B4284C94F8303763B3226D904234D0F2
:10690000012B27D0D4F82C21824236D0022B21D063
:10691000D4F80822904232D0032B1BD0D4F8E422C2
:1069200090422ED0042B15D0D4F8C02390422AD008
:10693000052B0FD0D4F89C24904226D0062B09D0EA
:10694000D4F87825904222D0072B03D0D4F85426CF
:10695000824210D0DC22591C02FB034284F830171B
:10696000106518465DF8044B70470023DBB25DF8F4
:10697000044B184670470723F8E70123F6E7022384
:10698000F4E70323F2E70423F0E70523EEE7062309
:10699000ECE700BFFC1000200548D0F8903723B189
:1069A000DB6A13B100F5F26018470248704700BF78
:1069B000F01A002470D1090838B51D4CD4F8C4333E
:1069C0001B8843B91B4D002384F8D33385F88837DF
:1069D000C5F8843738BDD4F8C823002AF2DDD4F8CE
:1069E000CC13012A488806D00123124DA4F8D00305
:1069F00084F8D233E7E78A880132121A9A42F3D137
:106A00000C4D0022D5F8903705F5F260C5F8BC278B
:106A10001B699847D5F890379B68002BD3D005F5B4
:106A2000F26098470028CED14BF0F4F9CBE700BFD5
:106A3000E82B0024F01A00240748D0F88C371BB14B
:106A4000064B93F8D2330BB100207047D0F8903743
:106A500000F5F2605B681847F01A0024E82B002468
:106A6000184A10B4184C92F8883744602344174CE5
:106A7000036092F8880794F8D333834218D892F8C9
:106A80008807834207D300235DF8044B1A46184653
:106A9000C1E90032704792F888071A1E5DF8044B6E
:106AA000C0F180030CBF01200220C1E90032704711
:106AB00092F88847002201201B1B5DF8044BC1E9B6
:106AC00000327047F01A002420EA0024E82B00244A
:106AD000104B114A93F8881792F8D30393F888273C
:106AE000904293F888270FD8904204D3D3F8843784
:106AF00000201844704793F88827D3F88437C2F1F0
:106B00008002104418447047801AD3F88437184420
:106B1000704700BFF01A0024E82B002438B5194D47
:106B2000194CD5F8C423937B012B08D0D4F88437B3
:106B300003F2FF736FF30A03C4F8843738BDD4F847
:106B400090375B6A63B104F5F2609847D4F89037E8
:106B50009B681BB104F5F260984778B1D5F8C4235F
:106B6000D4F884375288013B514213440B4003F25E
:106B7000FF736FF30A03C4F8843738BD4BF04AF94A
:106B8000ECE700BFE82B0024F01A0024F0B51C4C01
:106B900085B01C4B94F888271B4D0393134495F83C
:106BA000D31394F888270293914294F8883716D823
:106BB00099420CD294F888670F46C6F18006D9B97D
:106BC000334601223F2BCDE900670DD860B994F818
:106BD0008807401AB0FA80F0400905B0F0BDCB1A22
:106BE000002701221E46EDE76946002302A852F065
:106BF00049FE95F8D313EAE773180222E2E700BFD3
:106C0000F01A002420EA0024E82B00242DE9F047A4
:106C1000174684B000293ED0441E294DDFF8AC90C1
:106C20004FF0000A04EB0108264E0DE096F8883775
:106C30000846994296F888371DD2C3F1800318445C
:106C40003F281BD8A04526D095F8D30314F8013F60
:106C5000411C4844C9B280F820300B0685F8D31394
:106C6000E4D5002096F8883785F8D3A301469942E9
:106C700096F88837E1D3C01A3F28E3D996F88837C9
:106C80009942DFD0104B5B78002BDBD00020FFF760
:106C90007DFFA045D8D1694602A8FFF7E1FEDDE9F6
:106CA000003213443F2B00D910B904B0BDE8F0877F
:106CB00002463B4602A852F0E5FD04B0BDE8F0876D
:106CC000E82B0024F01A00240000002400EA00242D
:106CD00030B585B0694602A8FFF7C2FE58B9094C25
:106CE00004F5F265D4F8903728465B689847002889
:106CF000F8D005B030BD0246012302A852F0C2FD13
:106D0000EDE700BFF01A002438B50023124C134DF4
:106D1000C5F88C3749F034FFC4F8CC03FFF73CFECC
:106D2000D4F8CC33C4F8C403A3B19A885B88D21AD0
:106D3000436802FB0333C5F88C37F9F7B3FE94F8C8
:106D4000D323044695F888379A4201D0FFF7C0FF55
:106D5000C5F8844738BD00BFE82B0024F01A002492
:106D60002DE9F041104E154682180446D6F88C37AE
:106D70000F469A420D4A88BF1D1A92F8D32396F8FF
:106D800088379A4201D0FFF7A3FF002021462B4607
:106D90003A46C6F8BC07D6F89007846A0448A44669
:106DA000BDE8F041604700BFF01A0024E82B002442
:106DB000802200248C461346014662461846CFE7DF
:106DC0002DE9F04F00218BB041F69462B84854F0A1
:106DD000DBFE0420FCF75EFB01460520FCF75AFBB6
:106DE00051EA000340F05681B24B03934C2200213C
:106DF000AF48012454F0C8FE00214C22AC4854F0A6
:106E0000C3FE039BAA4AD3F86834AB4D16461471EF
:106E10001560D361136253624CF0CEFBFFF774FF31
:106E2000002108460DF0DEFFF9F73CFEB0F1000846
:106E300040F39B810024A14DDFF8A4E206F14C0948
:106E40002746A34605F5757A9D4E0294CDF804E0D9
:106E500004E00BF5006BD84540F3AD80019A536E0A
:106E6000C2F8C437F9F752FE202251465846FFF7C0
:106E700077FF12229349504654F076FF0028E8D15C
:106E8000BB4525D00299904B01EB410203EB8203F5
:106E90004A1C8E4918460293ABEB070305920493F4
:106EA00001F0DEFB029B4946059A41F84C3B049BEE
:106EB000C9F80C700292C9E90433D9F81C30C9E949
:106EC00008330123C9F80830814BC9F828308946B6
:106ED000039B5F461222D3F86834C9F81C30A91806
:106EE000335D013291F8D41399420BD00024202A4B
:106EF000F5D120375146B845384653DBFFF730FF10
:106F00000022ECE70134152CF1D1D019714F202269
:106F10003946FFF725FF384600230A2209A90997B9
:106F200001F0D2FC0746099800230A2209A9013082
:106F3000099001F0C9FC0790002309980A2209A9C9
:106F40000130099001F0C0FC0690002309980A2244
:106F500009A90130099001F0B7FC059009A9099829
:106F600000230A220130099001F0AEFC00230490B6
:106F700009980A221946013001F0A6FC97B105993B
:106F8000DDE9063243EA4212049B5B0143EAC12376
:106F9000A7F2BC7143EA600342EA412243EA02439A
:106FA000C9F81C30029B642B43D05F460BF5006B85
:106FB000D8453FF753AF029B642B1ED0BB451CD076
:106FC0000C22414C5E1C414902FB0344ABEB07051C
:106FD0003246204601F044FBD9F81C20C9F8004095
:106FE000C9F80C700296C9E908220122C9F80820E4
:106FF000374AC9E90455C9F82820029B002B03F140
:10700000010117DC4FEA4803B3F1805FC0F2AE80A4
:10701000274B9C6834B91A461B791BB11368002BA7
:1070200040F0DA80002108460BB0BDE8F04F0DF0CB
:10703000D9BE65214C261E48DFF8A8A04FF00109F3
:1070400006FB01F432460021234F0519284654F06F
:107050009BFD32460021284654F096FD1C4E1448F4
:1070600004F1100204F11803029940F804A0C5F8D5
:10707000089002312F62AE6240F802800244043070
:10708000C2F80480039AD2F86824C25003445A60BC
:107090006A62B7E74FF47A72002353F057F90F4B47
:1070A00040F2B27240F26D14B0FBF3F31EE000BF89
:1070B000803E0024000000242CB10A08E82B0024A4
:1070C00068420A0844420A08DC2F002458420A0891
:1070D000B56D0408BC2F00240068214C80510100CC
:1070E000F01A002480420A085B1A013212F00305EC
:1070F00014BF21464FF4B7718B42F5DA8749002D52
:1071000064D003910399D1F838148B42C0F29C806B
:10711000834D01245B1A55F8041F01349942F9DDAF
:107120000133A2F2BC72039D43EA44133C2443EAB8
:1071300042237C4AB0FBF2F102FB11024FF4616082
:10714000B2FBF0F100FB11221C20C5F83C04B2FB9D
:10715000F4F004FB1022521042EA401242EAC1222B
:1071600042EA0343C5F8683440E621464C266E4B9C
:10717000DFF8C091012706FB01F4324600214FF0F1
:10718000020A1D19284654F0FFFC32460021284609
:1071900054F0FAFC644B039A04F1180143F804908C
:1071A000C8F10063D2F8680404F11002BB405E4CE1
:1071B0005E4E85F805A0AF602E62A3502244536056
:1071C000231D585019444860686221E70C4603911A
:1071D0001D21C4F83C1495E75348002200232146A2
:1071E00026468464C463C0E910230246D56C02F1CC
:1071F0004C035DB398684D1E9E64A842C2E92366A5
:10720000DE630DD04D1CA84210D113F8481C002994
:107210003FF408AF1A6401461A4643F8083CE5E714
:1072200000293FF4FFAE53F80C2C014600293FF42F
:10723000F9AE81427FF4F6AE106CC56B0135C563C3
:10724000186493641A46D1E7012469E7364A022696
:10725000294613E0D36B16635B01C2E9041120D009
:1072600003F6FF7300EB133318465363C31A90639E
:1072700052F84C7F461C1D440134C7B11379701E6F
:10728000002BE7D1136916637BB103F6FF7300EBA4
:1072900013335769536337B107F6FF7700EB1730A5
:1072A000E4E73346E0E73046E0E73346F1E7DFF86E
:1072B00088E001381E4B0EF5FC62CEF81448CEF87B
:1072C00008583E243F25CEF8EC374023CEF804087A
:1072D000C2E90445CEF8F837840F8300D8B140F2F4
:1072E000FF155B1944F100045B0A43EAC45303F140
:1072F00040040D492344CEF8FC4703EBC000CEF810
:1073000000384402CEF8E807C30DCEF8E0475360DA
:10731000C2E90B1186E60123E9E700BF0000002463
:107320003804002480510100803E00240068214C74
:107330009C420A0890420A08F01A00242DE9F04302
:10734000484F93B0484DFFF737FB97F8883795F8CB
:10735000D3239A4201D0FFF7BBFC0024D7F88C67F7
:10736000C7F88447002E6DD0DFF800810AE097F857
:10737000883795F8D3239A4201D0FFF7A9FC20342F
:10738000A6421BD922464146684601F069F9684683
:1073900052F07EFB012201466846FFF737FCA3B29C
:1073A000002BE4D1D7F8C837002BE0D09A881B68AF
:1073B00059690A4218BF12049A61D8E7FFF7AEFB79
:1073C00097F8883795F8D3239A4201D0FFF780FCCD
:1073D0000023DFF8989098461C46C7F88437224669
:1073E000494609A801F03CF921220021684654F0E1
:1073F000CBFB202269462046FFF7B2FC202205463F
:1074000009A9684654F0B0FCA3B2203450B9202D2D
:1074100008D15BB1A642E2D8B8FA88F0400913B0AF
:10742000BDE8F08308F10108002BF3D1D7F8C83785
:10743000002BEFD01A689B8851690B4218BF1B04C0
:107440009361E7E7FFF76AFB97F8883795F8D3234E
:107450009A4201D0FFF73CFC00230120C7F8843793
:10746000DDE700BFF01A0024E82B0024A4420A083C
:107470000A4B93F86C241AB9094A92F8A408704789
:107480000849CA6D032AF7D10020054A4FF0010CC4
:1074900083F86C0482F8A4C8C865EEE700000024F5
:1074A000E82B00240040005808B503220E4BDA6593
:1074B00072B60E4B53E9021251EA020306D10023C1
:1074C0001A4609490A664B66FCF76EFF084B4EF6F2
:1074D000602C5B6E0CFB00F05B1842F10002C318DD
:1074E00042EBE072EDE700BF004000589834002402
:1074F000F01A002410B58C18A14215D001F1FF3EFE
:10750000013C41F2210C1EF8012F082380EA0220E1
:1075100002B24000002A8CEA420180B2B8BF88B2B1
:10752000013BF5D17445EED110BD00BF704700BFDF
:107530002DE9F047002BDDF820A0884607460CBF58
:107540004FF020094FF030095646002A144616F82D
:10755000011B23DD11B3334601E0002C05DD13F8D8
:10756000012B2546013C002AF7D1023D3CB149469A
:107570003846C047013DFAD29AF8001059B1384652
:10758000C047334616F8011B0029F8D1A4EB0A04C2
:107590001819BDE8F0872046BDE8F087002C04F1FB
:1075A000FF35E4DC00240029E9D1F4E703685A1C24
:1075B00002601970704700BF10B56FF000440246BA
:1075C000044404E0B3EB0E0015D1A24214D012F82B
:1075D000013BA3F14100192811F8010BA0F1410C66
:1075E00098BF203300F1200EBCF1190FEAD91B1A05
:1075F00004D10028E9D110BD002010BD184610BDEF
:10760000884230B54FF001043AD301FB04F4B0FBDB
:10761000F4FC8C45F9D2BCB102BB06E0A14203F8F0
:10762000015B11D81446B0FBF2FCBCF1090F0CF160
:1076300057050CF1300E04FB1C00B4FBF1F2EDDC3D
:10764000A14203F801EBEDD900221A7030BDA1422E
:1076500003F8015BF8D81446B0FBF2FCBCF1090F4B
:107660000CF137050CF1300E04FB1C00B4FBF1F2F9
:10767000EDDCA14203F801EBEDD900221A7030BD18
:107680008446002AEAD1D0E7002870B503DA2D231A
:10769000404201F8013B092886464FF0010307DD0F
:1076A00003EB83035B00B0FBF3F2092AF8D89BB12C
:1076B0000F4CA4FB030CBEFBF3F2092A4FEADC0CCF
:1076C00002F1570602F1300503FB12EE07DD092B2C
:1076D00001F8016B6346ECD800230B7070BD092BD9
:1076E00001F8015B6346E4D800230B7070BD00BF56
:1076F000CDCCCCCC0378202B03D110F8013F202B2C
:10770000FBD0092BF9D02D2B00F0A9802B2B75D0A5
:10771000B7EE000AA3F13002D1B2092977D8F2EE10
:10772000046ADFED5F7A07EE102A10F8013FB8EE29
:10773000C77AA3F13002D1B2A7EEA67A0929F0EEFA
:10774000477AF0D92E2B66D003F0DF03452B40F0AB
:10775000838010B442782D2A00F096802B2A00F006
:107760008380A2F130030130092B00F284800024D1
:10777000002303EB830302EB430310F8012FA2F174
:107780003001303B0929F4D9B3F59A7F1A46B7EE98
:10779000007A28BF4FF49A72072B09D91346DFED00
:1077A000416A083B27EE267A072BFAD802F0070237
:1077B000DAB1F2EE046A012A27EE267A15D0022AFF
:1077C00027EE267A11D0032A27EE267A0DD0042A36
:1077D00027EE267A09D0052A27EE267A05D027EE4D
:1077E000267A062A18BF27EE267A002C45D0C7EE47
:1077F000877A5DF8044B20EE270A70474378B7EE8E
:10780000000A0130A3F13002D1B2092987D92E2B09
:10781000DFED237A98D143780130A3F13002D1B261
:10782000092991D8B2EE047AF0EE475A06EE902A72
:1078300010F8013FB8EEE66AA3F13002D1B2C6EE0D
:10784000076A092927EE257A77EEA67AEED903F0A2
:10785000DF03452B3FF47DAF20EE270A70474378C6
:10786000BFEE000A013055E782780230A2F1300302
:10787000092B7FF67CAFB7EE007A67EE877A5DF86A
:10788000044B20EE270A704782780230A2F13003C1
:10789000092B01D801246BE7B7EE007AA7E700BFF8
:1078A0000000000020BCBE4CF0B5067906F0E003F5
:1078B000402B03D145794FF0FF3406E0602B4FF0A9
:1078C0000105F8D1447905FA04F40023012006F0FB
:1078D0000706AB4200D1F0BD052E0FD8DFE806F059
:1078E0000308101D242448B1C85CD75C78400FE021
:1078F00020B1C856D756C71B784278410133E8E714
:107900000028FBD031F8130032F81370784080B2B1
:1079100020420CBF01200020F0E70028EED031F912
:10792000130032F91370E6E70028E7D051F823007E
:1079300052F82370DAE7F8B50C4E054633788BB968
:10794000F8BD25B12388C3F30B039D4204D0A28860
:10795000D4E9020154F0BAF81C34BC42F1D300233C
:107960003370EDE7024C034FF7E700BF185D0024CA
:10797000CC110B08381A0B08037903F01803102BED
:107980001DD003D833B9B0F80B007047182BFAD0CC
:1079900000207047114BB0F80B0093F90030591CD0
:1079A0000BD10F4B1B7803EB430203EB820303EB7A
:1079B000C30300EB430080B27047DBB2F3E7074B31
:1079C000B0F80B0093F901305A1C04D1044B5B78DA
:1079D00000EB4310EFE7DBB2FAE700BF2405002419
:1079E0009834002420B10078B0FA80F04009704744
:1079F00001207047032870B518D80D4BC943C60045
:107A000003EBC00001F00101057A427A81EA050426
:107A1000A2420BD042683AB14D1B1068928869426D
:107A2000694109018A40826133445C7270BD00BFC4
:107A3000185D00240379062B0FD1C9B20D290AD88D
:107A4000074B59560123C2688B40134214BF0846A6
:107A50004FF0FF3070470021F4E7481C704700BF2B
:107A6000D8420A08092917D0B1FA81F35B0999B104
:107A7000013903604A0001F0030102F00802C1EB82
:107A800001119300C1EB0111A3EB92038900C3EB39
:107A9000031381809B004380704700BFB5EEC00A8E
:107AA000DFED357A0023F1EE10FA30B5C8BF30EEC5
:107AB000270A87B0D8BF30EE670ADFED307A054677
:107AC00003A9029320EE270ACDE90033FDEEC07A28
:107AD00017EE904A84EAE470A0EBE47047F0C6F930
:107AE000002C03A8B4BF2D2320238DF8003051F0C3
:107AF000CFFF01282AD0022834D003281ED003A9A2
:107B0000684654F049F8684651F0C2FF0446694699
:107B10002846033CE4B2224653F0D8FF002328460F
:107B20002B5551F0B5FF2E22431C0DEB04012A54B6
:107B3000E81854F05EF8284607B030BD302303A99A
:107B400068468DF8013054F027F8DCE743F2300244
:107B5000302303A96846ADF801208DF8033054F0B6
:107B60001BF8D0E743F2300303A96846ADF80130B3
:107B700054F012F8C7E700BF6F12033A00007A44CE
:107B80000AF07EBC38B5054658B14C1E14F8011FEA
:107B9000284619B9BDE838400AF086BC0AF070FCE6
:107BA000F4E738BD70B50546B0F8090042F0B4FB03
:107BB000054B044628461E78FFF7DEFE16B1E36843
:107BC000184470BDA368FBE7185D002438B505466E
:107BD0000C46FFF7E7FF2A7902F0070302F0E00204
:107BE000602A29D1052B0CD8DFE803F0030B0F0B1B
:107BF0001B1B6A79012393400278DBB214B1134353
:107C0000037038BD22EA0303FAE76A79012393403F
:107C100002889BB214B113430380F2E722EA030304
:107C2000FAE76B7901229A40036814B113430360A9
:107C3000E7E723EA0203FAE7052BE2D8DFE803F0DF
:107C40000303050507070470DBE70480D9E7046038
:107C5000D7E708B5202153F0AEFF034618461BB105
:107C600002780133202AF9D008BD08B5CB0701D42A
:107C7000FCF79AFB08BD2DE9F3410023124D0446A1
:107C800000EB8106114F05F8243FB44203D11048A0
:107C900002B0BDE8F081394628464FF0000853F0A5
:107CA0007BFF2146684653F0A4FF2021684653F02D
:107CB00082FF28B969462846043453F06DFFE4E793
:107CC00080F80080F1E700BF185D002425B60A089F
:107CD0003C5D00242DE9FF47914604468A461E4636
:107CE000FFF7A8FE421CBDF830700546DDF8348071
:107CF0001FD0B9F1FF3F1FD0154A3146CDE9000929
:107D000038462368C0474A465FFA8AF12079FAF775
:107D100015FA024600B10288D3B2314638460393C1
:107D2000C2F30323120B0293CDE90052094A2368E0
:107D3000C04704B0BDE8F0877B06FAD40C9031460A
:107D400023683846044AC44604B0BDE8F04760479B
:107D50002AB20A0837B20A085BB20A082DE9F043D2
:107D6000154685B0894619466A1CBDF830600D9FDE
:107D700028D04FEA101800F00F04194A304608F1D5
:107D80004008CDE900454346B847C0B1EBB2D9F849
:107D9000000099F805100F2B11D82A46FAF716FAA9
:107DA00068B103880021027830460392C3F30322AE
:107DB0001B0B02920B4ACDE900434346B84705B07E
:107DC000BDE8F0837306FAD4030900F00F00064AF9
:107DD000BC460C904033304605B0BDE8F0436047E8
:107DE0006AB20A087CB20A08A5B20A082DE9F04373
:107DF000070987B091461E46DDF83880403700F00D
:107E00000F0439B30EF0F2F9C3790546164A494614
:107E10003046CDE900433B46C047C0B12868FAF779
:107E20004DFFAA796B7912F0020F10494FEA9303C4
:107E30000F4A18BF0A46E97901330094CDE90321BE
:107E4000CDE901030B4A3B4600213046C04707B04D
:107E5000BDE8F0833B46084A49463046C4460E9486
:107E600007B0BDE8F0436047B9B20A08C3BC0A08CE
:107E7000E6BD0A08CBB20A08EDB20A08082348405A
:107E800041B240000029C0B2B8BF5040013BF7D119
:107E9000704700BF30B5056804468D4218D901F11E
:107EA000FF3E681E00231EF801CF082183EA0C0361
:107EB0004FFA83FC5B00BCF1000FDBB2B8BF53404C
:107EC0000139F5D17045EED16A1C22602B7030BDAE
:107ED00000236A1C22602B7030BD00BF9FED067A24
:107EE000F7EE007A60EE870A60EE800A30EEA70AAD
:107EF00080EE800A704700BFDB0FC94010B52DED42
:107F0000028B08EE101ADFED807ADFED800A04465E
:107F1000B8EE488A28EE008A28EE278AB0EE480A92
:107F200053F0CAF89FED7A7AF0EE407AB4EEC70AC1
:107F3000F1EE10FA40F3BD809FED746ADFED756AD3
:107F4000B0EE677A77EEC67AB4EEE67AF1EE10FA22
:107F5000F6DC9FED717AF4EEC77AF1EE10FA40F399
:107F6000C5809FED6B7A77EE677A27EEA76ADFED23
:107F70006B5ADFED6B6A9FED6B7AE6EE256A9FED3B
:107F8000660A67EE865ADFED610A38EE000AA6EE51
:107F9000267AE5EE877AB0EE678A53F08DF8DFED4A
:107FA0005C7AB4EEE70AF1EE10FA5BDDDFED576ABA
:107FB0009FED587AF0EE407A30EE660AF4EEC77A1A
:107FC000F1EE10FAF6DCDFED547AB4EEE70AF1EEEA
:107FD00010FA62DDDFED4E7A37EEC00AF7EE007A76
:107FE0009FED517A20EE004ADFED4C6ADFED4C4AFE
:107FF0000023B0EE673A9FED4B5AE4EE264AC4EDFB
:10800000097A60EE043AA361A8EE073A6361F0EEE4
:10801000675A2362F8EE006AE361A4EE245AE8EEA0
:10802000475A87EE836AA3EE850AB6EE007ABDEC66
:10803000028B77EEC07A26EE077A66EE266A27EE86
:10804000865A67EE277A25EE866A26EE807A84EDD8
:10805000015AC4ED007A84ED046AC4ED027A84ED1D
:10806000037A10BDDFED317AB4EEE70AF1EE10FAD3
:10807000A9D5DFED266A9FED2E7AF0EE407A30EE3C
:10808000260AF4EEC77AF1EE10FAF6D4DFED227A82
:10809000B4EEE70AF1EE10FA9CDCDFED267AB4EEDE
:1080A000E70AF1EE10FA99D5DFED207A37EEC00A33
:1080B00094E79FED1E7AB4EEC70AF1EE10FA7FF551
:1080C00048AF9FED126ADFED1A6AB0EE677A77EE7D
:1080D000867AB4EEE67AF1EE10FAF6D49FED0E7AD7
:1080E000F4EEC77AF1EE10FA3FF73BAF9FED117A4D
:1080F000F4EEC77AF1EE10FA7FF537AF9FED0B7A09
:1081000077EE677A31E700BF27D4D236DB0FC9405C
:10811000DB0F4940E4CB1641DB0FC93F92E741B981
:108120009730083C15A82ABEF304353FDB0F49C041
:10813000E4CB16C1DB0FC9BFDFED2D0A08B552F045
:10814000BBFFDFED2C7AB4EEE70AF1EE10FA28DD82
:10815000DFED276A9FED287AF0EE407A30EE660A6E
:10816000F4EEC77AF1EE10FAF6DCDFED247AB4EE25
:10817000E70AF1EE10FA2FDDDFED1E7A37EEC00AC6
:1081800020EE007A9FED1E6ADFED1E6ADFED1E7A9B
:10819000E7EE066A20EE076AE6EE877AA6EE270A81
:1081A00008BDDFED1A7AB4EEE70AF1EE10FADCD57D
:1081B000DFED0F6A9FED167AF0EE407A30EE260A78
:1081C000F4EEC77AF1EE10FAF6D4DFED0C7AB4EEE5
:1081D000E70AF1EE10FACFDCDFED0E7AB4EEE70A33
:1081E000F1EE10FACCD5DFED097A37EEC00AC7E719
:1081F000DB0FC940DB0F4940E4CB1641DB0FC93F21
:1082000092E741B99730083C15A82ABEDB0F49C058
:10821000E4CB16C1DB0FC9BFB0EEC07AF0EEE06A66
:10822000F0EE407AC6FE875AF5EE405AF1EE10FAAB
:108230003BD086FEC75A85EE256A9FED1D2A9FED2D
:108240001D3A9FED1D4ADFED1D4ADFED1D2AF7EEB9
:10825000005ADFED1C3A9FED1C5AA6EE423AE6EEBC
:10826000223AA6EE034AE6EE235AE6EE044AA6EECA
:10827000245A85EE250AF4EEC76AF1EE10FA03D50A
:108280009FED127A37EE400AF5EEC00AF1EE10FAD1
:1082900003D59FED0F7A37EE400AF5EEC07AF1EE86
:1082A00010FA48BFB1EE400A70479FED070AE2E7B7
:1082B00039094E3DE3B59E3E88FA163E45FE7F3FA6
:1082C00099FB243F69A2163EA7DFA834DB0FC93F04
:1082D000DB0F49402DE9F04F884689B01E461178E2
:1082E000531C0393002900F016810025144607460D
:1082F000A94609E038460135C047039C621C217835
:108300000392002900F08F802529F3D16078A31C07
:108310003028CDE9033923D0A0F130034FF0000A13
:10832000DBB2092B26D96C282AD078287FD8572889
:1083300078D9A0F15803202B79D8DFE803F0BD7875
:1083400078787878787878787882AF78787878786C
:1083500078787878AA787878789E788A7878BD0066
:10836000E31CA0784FF0010A0393A0F13003DBB2C5
:10837000092BD8D804AA03A948F0DAFB6C28D4D179
:10838000039B1A785C1C782A0394B7D8572A40F2CA
:108390008E80A2F15803202BB0D801A151F823F010
:1083A000D7840408FD820408FD820408FD820408C5
:1083B000FD820408FD820408FD820408FD82040891
:1083C000FD820408FD820408FD8204084584040837
:1083D000F3840408FD820408FD820408FD82040879
:1083E000FD820408FD820408FD820408FD82040861
:1083F000FD820408FD82040895840408FD820408B7
:10840000FD820408FD820408FD8204087D840408BE
:10841000FD82040803850408FD820408FD82040827
:10842000D784040828B9284609B0BDE8F08F039C1A
:1084300064E72528FBD1039C252138460135C04738
:108440005CE7039C56F8041B38460135C9B2C047A7
:1084500054E70DF1140B00220A2156F8040B5B4679
:10846000039CFFF7CDF85346049A41463846CDF8B1
:1084700000B0FFF75DF8054440E7039C56F8040B95
:108480000023049A414600903846FFF751F805440E
:1084900034E7039C56F8043B1D602FE70DF1140BE5
:1084A00056F8040B039C5946FFF7EEF8DBE7002A69
:1084B000B9D0252AC0D021E7A0F158020DF1140B44
:1084C000102156F8040BB2FA82F25B465209FFF70C
:1084D00097F8039CC7E7A2F158020DF1140B102185
:1084E00056F8040BB2FA82F25B465209FFF788F89D
:1084F000B9E70DF1140B56F8040B5946FFF7C4F811
:10850000B1E70DF1140B00220A2156F8040B5B466B
:10851000FFF776F8A7E70D4685E7F8B5104C074654
:108520000D461646A06CA0B10E49FFF72BFB39464D
:10853000A06CFFF727FB0C49A06CFFF723FB0B494E
:1085400033462A46A06CFFF7C5FE0949A06CFFF729
:1085500019FB94F84C3013B1012384F84D30F8BD69
:10856000185D0024FFB20A08F4CC0A08817B0408D5
:108570000CB30A080EB403B503AA52F8041B019207
:10858000FFF7CBFF044B0549986CFFF7FBFA02B0ED
:108590005DF804EB03B07047185D0024E4BD0A08E1
:1085A0000049E7E710B30A080049E3E71FB30A08E8
:1085B00007B5009313460A460249FFF7DBFF03B0F5
:1085C0005DF804FB36B30A08064B10B50446186D77
:1085D00037F042FA20B920460349BDE81040C9E708
:1085E00010BD00BF185D00244FB30A0870B5184CC9
:1085F000054694F84C307BB194F84D3063B1154981
:10860000FFF7B8FF28461449FFF7B4FF002084F8AD
:108610004C0084F84D0070BD94F85430ABB194F820
:10862000553093B90D4BA3F13C0503F120061868B2
:10863000083353F8041C2A46B34203C21546F6D148
:10864000012384F893300EF003FC0120E3E700BF20
:10865000185D002465B30A089CB30A08AC5D0024C9
:108660000EB400B584B0084905AB019001A853F8D9
:10867000042B0393FFF72EFE0022019B1A7004B017
:108680005DF804EB03B07047AD750408F7B5114E03
:10869000074600230C46304615460F49B43600F80D
:1086A000B43F04EB45050D4B002F18BF19460C4F86
:1086B00053F072FAAC4202D10A4803B0F0BD394619
:1086C00034F8022B6846FFF7CBFF6946304653F07B
:1086D00063FAEFE7185D0024C3B30A08BAB30A08C7
:1086E000CCB30A08CC5D0024F7B500230B4E04463A
:1086F00000EB41050A4F06F8E53FAC4202D10948BC
:1087000003B0F0BD394634F8022B6846FFF7A8FFE6
:108710006946304653F040FAEFE700BF185D002489
:1087200070BC0A08FD5D0024F8B54E1E054601F137
:108730001F04054F16F8012F284639460235FFF76A
:108740008FFFA642F6D1F8BDD1B30A08024608460B
:10875000531C05D1034B1A681B790A600B717047D3
:1087600001497DE765B20A0871BC0A0810B50131FC
:1087700014460DF03BFD28B9054B1A681B792260A1
:10878000237110BDC27920460249BDE8104067E759
:1087900065B20A08C6B20A0803685A1C026019705A
:1087A000090A03685A1C0260197070470268134670
:1087B000511C016013F802CB0360D31C5178036095
:1087C00093781B0443EA0123111D43EA0C03016063
:1087D000D07843EA00607047A0F13003092B07D935
:1087E00020F02000413819288CBF0020012070475C
:1087F00001207047303809288CBF002001207047C5
:10880000413819288CBF0020012070476138192891
:108810008CBF00200120704720280BD0092809D0E8
:108820000A2807D00D2805D00B3801288CBF00205E
:108830000120704701207047A0F14103192B98BF18
:1088400020307047A0F16103192B98BF2038704782
:1088500002B3844610B5841803E0981A15D1A445D4
:1088600014D01CF8013BA3F14100192811F8010BA9
:10887000A0F1410E98BF203300F12002BEF1190F84
:10888000EBD91B1A04D10028E9D110BD002010BD7E
:10889000184610BD1046704770B5044608460D4690
:1088A00051F0F6F8064602E014F8013F43B13246B3
:1088B00029462046FFF7CCFF0028F5D1204670BDA1
:1088C0001C46204670BD00BF2DE9F0430646864693
:1088D0009EF800C074460EF1010EBCF1200FF7D0D7
:1088E000BCF1090FF4D0BCF10A0FACF10B00EFD0D2
:1088F000ACF10D05B5FA85F56D09002DE8D101281B
:10890000E6D9BCF12B0F3DD0BCF12D0F39D0102A88
:108910003ED04FF0FF3E9046BEFBF2FE02FB0EF74C
:10892000FF43FFB2002014F801CBBCF1390F4CF02B
:108930002009ACF1300C0DD85FFA8CFC944510DAAC
:108940007045264602D819D1674517D21D404FF011
:10895000FF30E8E7A9F1570CB9F1600F5FFA8CFC22
:10896000ECD801B10E6003F00103D5B9002803DA99
:10897000002B18BF6FF00040BDE8F08300FB08C07B
:10898000D1E70125102A94F801C004F10104C0D1F7
:10899000BCF1300F10D06FF0704E0F274FF0100861
:1089A000C0E7B0F1004F04D91BB14FF00040BDE863
:1089B000F0834042BDE8F08360786FF0704E0F277F
:1089C0004FF01008A0F14106192E04F1010698BFDE
:1089D000203078280CBF02343446A3E701230A2252
:1089E000002171E770B50D461446FFF732F90646CF
:1089F000A0B1FFF7F3FF40F6340319229842A8BF55
:108A00001846B0F5617FB8BF4FF46170A0F561738F
:108A1000B3FBF2F32B702378013323703046FFF75A
:108A200018F90646A0B1FFF7D9FF40F63403192222
:108A30009842A8BF1846B0F5617FB8BF4FF4617087
:108A4000A0F56173B3FBF2F36B70237801332370ED
:108A5000304670BD73B50E4610490546FEF7ACFDB5
:108A600018B93070012002B070BD2C78602C8CBF1A
:108A7000613C413C082C0FD8013501230A2201A991
:108A80002846FFF721FF019BAB4205D00F2803D8F2
:108A9000013440EA0410E4E70020E4E765B20A0884
:108AA0002DE9F04116461F46404D044639463046F2
:108AB0004FF47A72002351F049FC3D4B05443D4F81
:108AC0003D4E83FB0510E9172844C1EB601183FB81
:108AD0000103C8170B44C0EB631087FB003CC317AE
:108AE000C3EBAC0386FB03764FEAE37ECEEBE61ED8
:108AF000C1EB0116A5EB860CC0EB00154FEA8E0604
:108B000084F806C0A1EB8501617103EB4301A0EB82
:108B1000C10040F2B55101FB1E332071B3F5896FDE
:108B200033DA40F2DA218B4237DCB3F5B77F234FDB
:108B3000B4BF4FF0000E4FF0010E0EEB4E01754624
:108B40004FEA4E0807EBC101C88A08EB0E0C0B2157
:108B500007EBCC0C0CF1160C01E03CF8020D98422E
:108B600010DD0139F9D1F044012137F8380006F55C
:108B7000FA6E0133A17075441B1A22812580E370BF
:108B8000BDE8F0810131C9B2F1E7032540F296500A
:108B90000A4F4FF00608AE46D7E7022540F22940BB
:108BA000064F4FF00408AE46CFE700BF80BC92C727
:108BB00089888888ABAAAA2A73B06D1624DD0908B3
:108BC0000D4B10B5D3E9004354EA03020AD1014624
:108BD000002340F2011218460B80C1F802208B716D
:108BE0000B8110BD054A1268121943F10003FFF70B
:108BF00057FF012010BD00BF90340024541B0024F7
:108C00002DE9F0410446154608469442B4FBF2F6BD
:108C100007D205FB1644134B1B5D00F8013BBDE872
:108C2000F0819642B6FBF2F70CD20E4B05FB1767AC
:108C300005FB1644DA5D1B5D00F8012B00F8013BD3
:108C4000BDE8F081BA42B7FBF2F807D905FB187806
:108C5000044B13F8082000F8012BE7E74046FFF724
:108C6000CFFFF3E7F4420A0830B56D4C83B0B4F897
:108C70003C35B3F57A7F03D94FF47A73A4F83C35C9
:108C8000B4F83E35B3F57A7F03D94FF47A73A4F87C
:108C90003E35B4F84015B1F57A7F04D94FF47A73B4
:108CA0001946A4F84035B4F84205B0F57A7F03D9E7
:108CB00000231846A4F84235B4F84435B3F57A7F5A
:108CC0004BD94FF47A73B4F846259A42A4F8443548
:108CD00048D900238842A4F8463580F08B80B4F848
:108CE0005225B4F854359A4202D90023A4F85235DB
:108CF0004C4B1B88EBB14C4DAA78062A4FD92979E9
:108D000000297AD19FED497A494A07EE903AAB792A
:108D10001178F8EEE77A06EE901AB8EEE66AC6EE3B
:108D2000276A0BB137EE077AB4EEE67AF1EE10FA65
:108D300043DC404B5978032923D83F4A02EB4112C8
:108D40001978C4F85C25032914D8EA233B4A01FBAF
:108D500003223B4B1A6003B030BDB4F84625B2F590
:108D60007A7F16D8884210D29A42B8D30023A4F84A
:108D70004435B4E70021314A1970314B1A6003B011
:108D800030BD00212C4A5970DAE70021A4F84015C3
:108D9000EAE700228842A4F84625E5D3F5E7294909
:108DA00001EB820191ED187A29790029ACD0531F8B
:108DB000032BBED9002ABCD024E067EE877ABCEE34
:108DC000E77A8DED017A9DF8043007EE103AB8EE9F
:108DD000C77AF4EEC77AF1EE10FA01DD0133DBB2A7
:108DE000E3B1102BA8BF1023DBB28B4238BF0B4678
:108DF00013709EE7A4F8403571E7053A032A98D925
:108E00009FED0A7AB7EE000A80EE070A52F086F963
:108E10002B88834228BF03462B808AE70123E3E7A0
:108E2000185D0024A01D0020B02E00246F1203380E
:108E30007436002498340024285E0024A85E0024A0
:108E40007C36002424DD09082DE9F04FA14B83B0C6
:108E50001B7800AFA3F11702022A05D99E4A12F827
:108E60003310002940F0A9829C4B0026DFF8908245
:108E700003F178059A4BA5F1780B93F8089020E060
:108E80009BF90430142B00F08E82204653F02CF80E
:108E9000A10322D5012800F08682082800F38382EE
:108EA000BAF1000F02D014EA080F06D14946204655
:108EB0004FF05AF8002800F076820BF10C0B5D455C
:108EC00011D0DBF8004014F0010AD9D02046013659
:108ED00053F00AF8A103F6B2DCD40128DDDC0BF173
:108EE0000C0B5D45EDD1731E022B00F25C8200235A
:108EF0007C4C02207C4D84F8DC3511F00BFD94F89D
:108F0000E035D5F80080022B00F0DD82002800F06B
:108F10002F83DFF8F091754B4FF47A7A94F839C6C5
:108F20004FF0000E03F56A7B6426C7F804C033F8DF
:108F3000082CB2F57A7FB3F8462088BF23F808AC36
:108F4000B2F57A7F33F8062C88BFA3F846A0B2F5B5
:108F50007A7F33F8042C88BF23F806ACB2F57A7F09
:108F600002D9002223F804EC33F8061C9142B3F82E
:108F70005A10B3F85C2098BF23F806EC914293F89E
:108F80006B2003F1650102F1FF3288BFA3F85AE0BC
:108F9000632A93F86C2002F1010288BF83F86B60AA
:108FA000D2B2092A4FF0000288BF83F86CE013F8B0
:108FB0003200013211F801CF844538BF81F800E05A
:108FC000032AF4D17A68EA33012A18BF03F864EC63
:108FD0009B45ACD1DFF830A19AF80230042B00F0A9
:108FE000A0822BB9BAF80030B3F5F07F00F2E0812F
:108FF000FFF73AFE3E4894F84C16FEF733FD10306A
:1090000094F86B16FEF72EFDB4F87A26B4F878368D
:109010001343B4F87C2613431BB213B10123A4F805
:109020007E36344B08EA0303002B00F0B08218F0C0
:10903000010F40F0588218F4804F40F0C88118F0BA
:10904000080F00F02C822C4AD9F8003008EA0208F8
:109050001340C5F80080C9F8003018F4004F00F044
:10906000018200231E4AD373D37718F4805F00F087
:10907000048294F88B36022B02D1012384F88B36BC
:10908000DFF87880434608F1780B02E006339B4511
:109090000CD01A780A2AF9D19978DA78914202D359
:1090A0005A79002AF2D00A201EF0E4FD00234FF482
:1090B000806084F8DC3511F02DFC002800F0468239
:1090C0000E490E467960707960B3317839B3434602
:1090D0001FE000BF7835002430D4090878620024EE
:1090E000B8340024185D0024F83A0024B25E00244D
:1090F0007463002409600002FE9FFFFDA863002442
:10910000BC020200B4340024B02E002406339B4578
:1091100008D01A788242F9D15A79002AF6D0084646
:109120001EF0A8FD0636B345CDD19AF802807968C5
:10913000B8F1080F00F0B98194F8393694F8392560
:10914000A3F10103032AB3FA83F34FEA531384F81C
:10915000083794F83A36A3F10103B3FA83F34FEAE0
:10916000531384F80E37D9F80030C3F3C03084F8B5
:109170000B0702D9002284F83925A64A03EA020027
:109180002B681A40A44BC9F800009B7B2A60002B77
:1091900000F0B581A14DAB88002B40F0A681A0481E
:1091A0000368B3F5000F01D30023036083689D4A71
:1091B0001A4012B140F2022383600379013B042B71
:1091C00001D901230371A8F10508974BB8F1030FEA
:1091D00093F8009040F21581B9F1000F25D00025D9
:1091E000DFF878827D604D46C146884605E0063E40
:1091F000A6EB0A06B54240F2EC804E4619F8010F84
:109200000028F4D00DF016F80028F0D082799307EA
:10921000EDD541467D6801223DB19AF8113053B930
:109220009AF80530012B00D02AB19AF8063013B114
:1092300000238AF806307D4AD38803F00F00042803
:1092400003D8C3F30313022B02D94FF42063D38056
:10925000138903F00F00042803D8C3F30313022B70
:1092600002D940F60123138194F8210794F82D27A1
:1092700094F82037904205D9002284F8212753B171
:10928000A4F8242794F82C279A4204D2002384F8C7
:109290002037A4F8243794F8222794F816389A42F5
:1092A00002D9002384F82237614DDFF8B4A105F11B
:1092B00080092B4613F8032D02EB4202524492F828
:1092C0007CC092F87D6092F87E0013F801EF9A79E5
:1092D000E645A8BFE646B242A8BF324683F800E0A2
:1092E0009A71DA788242A8BF0246AB42DA70ECD1BA
:1092F00003F120054D45DCD14E4BDA6A002A00F01F
:1093000005810025012002E006318B450ED00B7847
:109310002B2BF9D14B78043300FA03F31342F3D02B
:10932000063122EA030201258B45F0D10DB1414BF4
:10933000DA62414D6E4605F108082B4601E04345CF
:109340004BD013F8012F072AF9D9002305F8013F64
:109350000133082BFAD1B4F83226B546B4F83036CA
:109360009A4202D3354BC4F83036354BFF22354D87
:1093700003F1780084F8482813F9082C142A05D042
:1093800053F80C1C35EA010100F0C8800C339842F8
:10939000F2D12D4B5A79022A01D100225A710C3791
:1093A000BD46BDE8F08F2949294840F0CBFF9EE536
:1093B0004FF4F073AAF800301AE602EBC3025368C8
:1093C000002B7FF451AD1723224A13704CE5224A3B
:1093D0003AE641467D6800221EE788B02022FF2140
:1093E000E946484652F0D0FB134A03E0424549F8AB
:1093F0002330B0D012F8013F59F823100131F5D0D5
:10940000A3E700238AF80430B9F1000F00F0BD8013
:109410000125E5E69DD44518983400240036002443
:1094200080360024FDFDFFFF481C0020D0390024B9
:109430002D5E0024B8340024C22E0024AE014A015F
:109440008462002401000200542700247862002472
:1094500034140B0878350024F6DFFFFDB72E002406
:1094600024DD09084E4BDB7B002B7AD000234C4ACD
:1094700018F4805FD3777FF4FCAD18F0800F3FF4D1
:10948000F8AD484B1A78182A04D8474BD340DA076E
:109490003FF5EFADDFF8208108F1780B06E618F410
:1094A000005F3FF4DAAD414ACEE59AF80630002B72
:1094B0003FF442AE9AF81130012B7FF43DAE022307
:1094C0008AF8113038E600283FF423AD90F9049073
:1094D0004FF0FF0A01E080F808A048460EF060FD5A
:1094E0000028F8D115E5324AAEE5287879600CF00D
:1094F000A1FE796800287FF452AEA8804FE62D4B7C
:109500001A4303432A60C9F8003043E62B207960F0
:109510001EF0B0FB224B7968DA6AF2E684F848283C
:1095200037E7D9F8003028F4805823F48053C5F881
:109530000080C9F80030BAF82030B3F57A7FBFF464
:1095400057AD4FF47A73AAF8203051E52B6823F019
:1095500000632B60D9F8003023F00063C9F80030B5
:10956000AEE542F2010318EA030F7FF47FAF7CE51A
:10957000DFF8489028F08008D9F80030C5F800805E
:1095800023F08003C9F80030C5E44A4645E6D9F81F
:10959000003048F0080843F00803C9F8003052E5ED
:1095A000B83400247835002400410001F6BFFFFDE7
:1095B000F79FFFFD00040500A8630024B4340024D5
:1095C0007E4B2DE9F04F93F84C3883B0013B012BD3
:1095D00040F2DE807A4F7B4BFA68DFF8148202F2A9
:1095E000DC524345FA6080F0E680DFF80892012201
:1095F0009B46754D09F102060192B9F80210002947
:1096000000F0B180052906EB010240F2AC80AA42CD
:1096100080F0A980BBF800003446C0F30B000BE0DB
:10962000138814461A44002B00F09D80AA4280F053
:109630009A80052B40F2978063888342F0D163794A
:109640009B07EDD123885846DBF8081094F804A056
:10965000009340F077FEBBF80010BAEB113F00F02A
:10966000888000230193BBF804100BF11C0B5BF8FE
:10967000140CC1F30B015BF8044C46F0C7FDC34565
:109680002060BAD3514A524B1268524E524C1A6063
:10969000FFF7DAFB3278EA23504D02FB034372787E
:1096A0002B60A4F1800303EB4213C4F8CC331CF00D
:1096B000E9F94FF0FF332868494D6B6025F000FE53
:1096C0001EF01EFB04F5A06304F5AF6102E0063353
:1096D000994258D01A78002AF9D19C78D8788442D7
:1096E00002D358790028F2D0344C2A7294F8883684
:1096F000B4F88C2603EB830303EB83039B00642BFA
:10970000B8BF64237B60642303FB02F20023642A56
:109710007B61BB84B8BF642287F82630C7E9033376
:10972000BA603A622F4AC7E9063304F5CF63936201
:109730002AF07AFD94F87218B4F8700820F0DAF97B
:1097400036F028FA16F02AFC94F84C38013B012B2D
:1097500029D9254B012201981B6887F82520FB6039
:1097600003B0BDE8F08FDBF80810584640F0EAFD82
:1097700077E7009BA11D58469A1F40F019FE00286C
:109780007FF471AF6DE7F27B003A18BF0122ABE7BF
:10979000F9F70AF8154B09490222034481F86C28AD
:1097A000C1F8683816E7F8F7FFFF0223C4F8680825
:1097B00084F86C38CDE70123019363E7185D00243A
:1097C00090360024CC110B0800000408F83A00245D
:1097D000B434002498340024A85E00247C3600248D
:1097E0002405002494210020541B002460E316006B
:1097F000381A0B0800000208104B0122032810B58C
:1098000004461A7005D9601CBDE81040C0B211F0C2
:109810009FBAEA210A480B4A04FB01000A4B147064
:10982000186025F04DFD22F070FF23F051F8601C08
:10983000BDE81040C0B211F08BBA00BF6433002005
:10984000A85E0024983400247C360024044A0120B9
:109850000449136881F8740843F4001313607047D7
:1098600070360024185D0024F8B5164D6B78BE2BB9
:1098700026D1AC1C144F022229464FF6FF70FDF78B
:1098800039FE22884AB1A618BE4219D2052A17D934
:1098900021463446FDF72EFEF3E721460222FDF76E
:1098A00029FE0222A1180634FDF724FE074B641B93
:1098B000A3F8764841F60F53C31A58425841F8BDF1
:1098C0000020FCE70000020800000408185D0024E6
:1098D00070B5046886B005460E46C4F310033BBB62
:1098E00001220393CDE901332023CDE9042304F1C0
:1098F0007843B3F5801F19D3A4F10163B3F5801F3A
:1099000010D2A4F58013022203F17843694601A81E
:1099100002925B0C039341F0EBFD48B14FF0FF3036
:1099200006B070BD0520FCF799FDFBE72346EBE789
:109930003146204647F066FB18B92B6820332B6070
:10994000EEE76FF00200EBE72DE9F0416A4E90B0D0
:109950003378B12B7ED1FFF787FF80F00104E4B2AA
:10996000664B04F00104664DB3F88B30654FADF8DB
:109970000030BD4270D3002C00F0BC8028220021B2
:1099800006A852F001F9604B04969B1B05935F4BB0
:10999000DA68D40770D45D4BD3F80C21D00774D4A7
:1099A0004FF480730222694604A8ADF83C304FF0B2
:1099B000CBFA022269464FF6FF70514DFDF79AFD32
:1099C0004FF000080446BD4269D30025022201A9D8
:1099D00004A8ADF804504FF0B7FA022201A92046BE
:1099E000FDF788FD40BA022202A9C043ADF8080085
:1099F00004A84FF0A9FA0E9888B106ABC0F1200276
:109A00002946184452F0C0F89DF93C0018B906A93F
:109A100004A8FFF75DFF00238DF83C000E939DF82E
:109A20003D307BB1394BDA6842F00102DA60DA6826
:109A3000D20707D5D3F80C2142F00102C3F80C215C
:109A4000D3F80C319DF93C00B0FA80F0400910B019
:109A5000BDE8F081012483E7AB691C3535F8181C9B
:109A6000D3F8008055F8140CC1F30B0146F0CEFB7F
:109A7000804518BF01247CE7254A5A6002F18832EC
:109A80005A60DB68D90786D58AE7214AC3F80421E2
:109A900002F18832C3F80421D3F80C3180E7AE8894
:109AA00002A904A88DF80D80C6F30B061C35B31D62
:109AB000ADF8083035F81C3CC3F30B021B0BADF8B6
:109AC0000A2006228DF80C304FF03EFA062202A939
:109AD0002046FDF70FFD044655F8141C324604A835
:109AE0004FF032FA204655F8141C3246FDF702FDBD
:109AF000044668E70120AAE70000020824DD0908FF
:109B0000CC110B08381A0B08000004080020005282
:109B100023016745F8B5254DFFF796F995F84C38C0
:109B2000013B012B2FD9224E0324224FF36803F26D
:109B3000DC53F360FFF708FF58B13B78B12B08D135
:109B4000FFF792FE013C1BD040B9FFF7FDFE002855
:109B5000F3D1013CEED10520FCF780FC95F84C38A0
:109B60000022013B85F87828012B16D9124B0121E0
:109B700000221B6886F8251085F87928F360F8BD67
:109B80000028EBD1E7E7F8F70FFE0C4B0222034465
:109B900085F86C28C5F86838C5E7F8F705FE022394
:109BA000C5F8680885F86C38E0E700BF185D002448
:109BB0009036002400000208541B002460E31600C5
:109BC00010B5074A0124074B14709C73FFF7A2FFDE
:109BD000FFF7F6FC2046BDE8104011F0B9B800BF11
:109BE000643300209834002490F89230B7EE007A65
:109BF000DFED6A6A014607EE903A90F89630684ABF
:109C0000B0EE476A05EE103A90F89430F8EEE77A35
:109C100004EE903A90F89530B8EEC55A05EE903AB9
:109C200090F8983067EEA67A04EE103A25EE265AA0
:109C3000F8EEE44AF8EEE55AB8EEC44A25EE275AA3
:109C400064EEA64A65EEA65A24EE264A64EE854ADC
:109C500065EEA75A24EE274AB0EE473AF0B590F8E1
:109C6000917000F16F0602F11A050024137807EED7
:109C7000903AF8EEE77A67EE857A67EE867AFDEE3F
:109C8000E77A17EE903AFA2BA8BFFA2323EAE37398
:109C90000B72537807EE903AF8EEE77A67EEA47A03
:109CA00067EE867AFDEEE77A17EE903AFA2BA8BFB8
:109CB000FA2323EAE3734B72937803EE903AF8EEBB
:109CC000E33A63EEA57A67EE877AFDEEE77A17EE60
:109CD000903AFA2BA8BFFA2323EAE3738B72938896
:109CE00007EE903AF8EEE77A67EE847A67EE867AC6
:109CF000FDEEE77A17EE903AD5ED007AB3F57A7F6C
:109D0000F8EEE77AA8BF4FF47A7323EAE3738B8106
:109D10002B68002B3FDD90F89730B0EE436A02EEDF
:109D2000903AF8EEE22AA2EEE66A63EE863A83EE15
:109D3000A76AA2EEA66A65EEA77A013467EE877A73
:109D400067EE867AFDEEE77A17EE903AFA2BA8BF17
:109D5000FA23BC4223EAE37306F8013F00DDF0BDBD
:109D6000012C13D190F8933007EE103A90F89B3005
:109D700006EE103AB8EEC77AB8EEC66A27EE267A33
:109D800026EE266A0435083208316FE7B7EE007A0E
:109D9000B0EE476AF6E7B7EE006ACCE70AD7233C95
:109DA000B2DD090890F899306BB3B0F864308BB12C
:109DB00090F89A20642102EB8203C3EB0313B3FBF8
:109DC000F1F3A0F86430962312FB03F3B3FBF1F335
:109DD000A0F8663043884BB190F89A30642203EBC8
:109DE0008303C3EB0313B3FBF2F34380B0F85030AB
:109DF0004BB1962290F89A3013FB02F36422B3FB26
:109E0000F2F3A0F85030704790F821304BB3438BF9
:109E100083B190F82230FA22642113FB02F203EBA3
:109E20008303B2FBF1F2B3F57A7F4283A8BF4FF40C
:109E30007A738383838843B1FA2290F8223013FB2C
:109E400002F36422B3FBF2F38380C3884BB190F832
:109E5000223003EB8303B3F57A7FA8BF4FF47A7304
:109E6000C380704770B50B4C002504F56A7694F8F2
:109E7000913013B12046FFF7B7FE20460135FFF7BA
:109E800091FF3046FFF7C0FF042D04F1EA04EED144
:109E900070BD00BFA85E002410B5064C4FF4807260
:109EA000002104F67A0051F06FFE0023C4F87C39DB
:109EB00010BD00BF185D0024034BD3F8800908B122
:109EC00008F0F2BA704700BF185D002408B50B46D1
:109ED00005490246D1F8800928B10449FEF7FAF98C
:109EE000BDE80840E8E708BD185D0024817B040850
:109EF000024B0146D3F88009FDF744BE185D0024EB
:109F00000048F5E7E4BD0A080CB4C30607B500D560
:109F100061B905A904980191FFF7D8FFFFF7F0FF99
:109F2000012003B05DF804EB02B070470020F8E7B1
:109F30000FB407B504A951F8040B0191FFF7C6FF50
:109F4000FFF7DEFF03B05DF804EB04B070472DE9C6
:109F5000F74F81460846FDF745FD0E46054670B1B0
:109F6000002401A92046013444F080FF0146484600
:109F7000FFF7EDFF122CF4D103B0BDE8F08F0846D7
:109F8000FEF72CFDC4B2112C70D83D4D701CFDF7AE
:109F900060FE3C4E05EB44088346670098F884A9B0
:109FA000B0B9AAF102014B424B413D4495F88429D6
:109FB000B25C002B54D095F88539192040F2EE217F
:109FC00000FB03132146304803B0BDE8F04FAFE774
:109FD0000178304651F0EFFD80B1032C2B49A0EB06
:109FE000060394BF0022012202EB42020A4452FA05
:109FF00083F393F8B4A0BAF1030F05D1484603B038
:10A00000BDE8F04FFEF7CCBA5846FDF722FEF0B19E
:10A01000BAF1020FF2D1FEF7E1FC40F6CA0380B2BA
:10A020009842A8BF184640F2EE239842B8BF18469F
:10A030001923A0F2EE20B0FBF3F088F88509AAF10D
:10A04000020253425341EA1982F884A9ADE7BAF1FA
:10A05000020FF4D1484603B0BDE8F04FFEF7A4BAB2
:10A0600021460B4803B0BDE8F04F61E711232A46B3
:10A070000849484603B0BDE8F04FFEF799BA00BF63
:10A08000185D0024985F0A08D6B30A0824DD090881
:10A09000E6B30A08F3B30A08F8B50C4606460846C4
:10A0A000FEF79CFC20210546204651F084FD044625
:10A0B00020B93046BDE8F840FEF776BA104F0134BB
:10A0C000104E3B7832789A4201D0FCF701FE0E4BDD
:10A0D00020461D604FF0DCFC012201462046FCF7C3
:10A0E00095FD3B7832789A4201D0FCF7F1FD20468D
:10A0F0004FF0CEFC2A4601460448BDE8F84017E779
:10A1000078220024BB2F002474220024FBB30A0809
:10A11000154B1B682DE9F041044688B0F3B11A686D
:10A1200004A91846D56A6A46A847064688B104AC11
:10A130006D460027DFF83C80013735F8022B34F8F4
:10A14000021B4046FFF7F4FEBE42F5DC08B0BDE856
:10A15000F08106492046FEF70DFAF7E7044908B0FA
:10A16000BDE8F041FEF706BAC83600242BB40A0851
:10A1700043B40A0811B40A080249034801F5006112
:10A180000EC9D5E600E0F11F4AB40A082DE9F74FE1
:10A19000DFF82081834608460C464FF079FCD8F85A
:10A1A0000070064628B1024633492046FEF750FBB0
:10A1B00080B93946314844F0C9FD3149314821EA76
:10A1C000070144F0C3FD3049304803B0BDE8F04F0B
:10A1D00044F0BCBD23782D2B24D10134013E4FF037
:10A1E000010A2B4B4FF000094FF0FF3553F8041BC9
:10A1F00051B1324620460193FEF72AFB0028019B0D
:10A200000ABF4D460021012109F10109A9B9B9F19F
:10A210001D0FEBD122461F49584603B0BDE8F04F51
:10A22000FEF7A8B94FF0000ADBE73B431A49C8F82C
:10A2300000301A4B12E01A4913E00123104AAB40D8
:10A240001A40002AF7D007EA0302BAF1000FECD057
:10A2500027EA03031349C8F80030134B002A18BF3C
:10A260001946124B124803EB8503D3F8BC2003B008
:10A27000BDE8F04F5CE600BFDEC20A0889B40A08F8
:10A280009DD4451893B40A08622BBAE79FB40A0814
:10A29000E0DD0908ADB40A0881B40A087AB40A08F6
:10A2A0005EB40A086AB40A0871B40A0824DD090811
:10A2B0005BB90A08F83A002410B50446012026F0DC
:10A2C00041FC28B920460449BDE81040FEF752B9C8
:10A2D0000248BDE810402BE6BEB40A08CDB40A0817
:10A2E0002DE9FF47074608460D464FF0D1FB0828E9
:10A2F00046D105F1FF3801AE073531464246B14639
:10A3000012F8010FFEF79EFA01F8010BAA42F7D1ED
:10A310000023DFF880A08DF80C30A84518D11C4927
:10A32000484626F09BFB1A4808231A4910F8012BCF
:10A33000013B11F8014B02F110026A4402F80C4C87
:10A34000F4D101A914488DF80C30FFF7F1FD14E0A9
:10A3500018F8010FFEF776FA0446014606F8010BDD
:10A36000504651F028FC28B12146304651F023FCDC
:10A370000028D2D03846FEF713F904B0BDE8F087C4
:10A380000028D0D0384604B0BDE8F047FEF70CB93D
:10A39000B8340024885D0A08D8B40A0870B50022D1
:10A3A000124C134D134E94F85B3503F0010302B1C8
:10A3B00070BD002BFCD001212846FFF7B9FD7520A8
:10A3C0002AF0E2FB01463046FFF7B2FD1A202AF0E0
:10A3D000DBFB01460848FFF7ABFD1B202AF0D4FB4E
:10A3E00001460648FFF7A4FD0122DCE7185D0024C2
:10A3F000DFB40A08EBB40A08FEB40A0811B50A086B
:10A4000070B5054608461646FEF7E8FA0D4B041EE1
:10A410001A780EDB944205DA21460B48FFF788FDD7
:10A42000204670BD2EB1FF2C03D10848FFF780FDF8
:10A43000F6E7013A064928464FF0FF34FEF79AF84E
:10A44000EEE700BF481C002024B50A0835B50A080D
:10A4500048B50A082DE9F74307460846FDF7C2FA52
:10A460000B46044628B1384603B0BDE8F043FEF77A
:10A470009BB801AA2E491846264651F062FBA04619
:10A480000546DFF8AC905DB92A4B3246A1B2186D93
:10A4900047F068FA68BB28493846FEF76BF828E0B1
:10A4A000B8F1000F06D0B8F1010F25D03846FEF7FD
:10A4B0007BF81EE028464FF0EBFA2049064602469C
:10A4C0002846FEF7C5F950B332461D492846FEF727
:10A4D000BFF930B332461B492846FEF7B9F910B32D
:10A4E000324619492846FEF7B3F9F0B13846FEF76F
:10A4F00057F803B0BDE8F083B31E294638465A42E8
:10A500005A41FFF77DFF421C0446F2D001AA49469A
:10A51000002008F1010851F014FB0546B3E7464658
:10A52000F4E70126F2E70226F0E70426EEE700BF93
:10A5300025B60A08185D00247AB50A086EB50A081F
:10A5400071B50A0874B50A0877B50A082DE9F7430A
:10A5500080460846FDF746FA0B46054628B14046B8
:10A56000FEF722F803B0BDE8F08301AA2C49184693
:10A570002F4651F0E6FA2E460446DFF8A4907CB947
:10A58000022DECD1A7F57A73B3F57A7F21D94FF478
:10A59000FA634FF47A7223494046FEF709F8E1E77F
:10A5A0004DB1012D10D001AA49460020013551F0CE
:10A5B000C8FA0446E3E7012221464046FFF720FFA0
:10A5C000431C0646EFD1CDE72046FEF707FA0746C3
:10A5D000E9E7154BB8B21B685B689847FCEEC07A98
:10A5E000FF2E124B17EE902A0AD11149B6EEC00A7F
:10A5F0000978A1420FDC11460E48FFF799FCB1E73C
:10A6000003EB860331460C48B6EEC00A83ED000A20
:10A61000FFF78EFCA6E70134A3EC010AE9E700BFCF
:10A6200025B60A087ACA0A08C4210020C066002498
:10A63000481C0020A5B50A0898B50A08F8B50746D1
:10A640000846FDF7CFF9C8B11E4BDE68013630462B
:10A6500034460DF081FA0546E8B90134182CA8BF3C
:10A66000002420460DF078FA0546A0B9B442F4D192
:10A6700038461549BDE8F840FDF77CBF0846FEF7AF
:10A68000ADF904460DF068FA054620B921460F4899
:10A69000BDE8F8404CE40B4BDC6010F073FA2A463E
:10A6A00021460B48FFF744FC172C09D8094B0C2214
:10A6B00002FB043393F83001BDE8F84010F09EBA75
:10A6C0000020F9E724050024B4B50A08C8B50A0833
:10A6D000DEB50A0824DD090838B50446114D0846E0
:10A6E000FDF780F960B1104B93F900104B1C05D1B8
:10A6F0000E4B19780E48BDE8384019E4C9B2F9E7A5
:10A700000846FEF76BF9032804D8C0B2FFF774F8C7
:10A710002946E4E7204603220649BDE83840FDF714
:10A7200029BF00BFE6BD0A08240500249834002490
:10A73000F7B50A0807B60A0838B50446114D0846A9
:10A74000FDF750F968B1104B93F901104B1C06D17D
:10A750000E4B59780E48BDE83840FFF7E9BBC9B247
:10A76000F8E70846FEF73AF9032804D8C0B21BF010
:10A770000DFC2946E3E7204603220649BDE83840A0
:10A78000FDF7F8BEE6BD0A0824050024983400242D
:10A79000F3B50A0802B60A0808B5FFF7A9FBBDE839
:10A7A0000840FFF7ADBB10B504460348FFF7A0FB18
:10A7B0002046BDE81040EFE722B60A0808B5034678
:10A7C00010460AB9002008BDDB0601D50029FAD0E1
:10A7D000FFF7E9FFF6E72DE9F04F724C8DB0DFF897
:10A7E000D0910A4604F1B00A00218346FFF7E6FF44
:10A7F00003900025A37A99F80060AB4200F39280A1
:10A8000010345445F5D140F216200DF1180A3FF0EE
:10A8100083FD0027002E4FF015024FF00001D0E914
:10A820000245504604BF2546344651F0ADF92E7816
:10A83000002E3ED06978304605910BF0D7FC95F993
:10A840000290049009F1010253425341002C00F0A0
:10A85000A68000220599A05CB04240F09C80224472
:10A8600092F90280C14540F0948052788A4208BF34
:10A870000123012203F001030AF8072083F00101FC
:10A88000039A58460593FFF799FF059B039044B13F
:10A89000454A30460499CDE900B24246FDF75EFADA
:10A8A000059B424A30460499CDE900B24A46FDF77D
:10A8B00055FA01370335152FB9D184B3564604F143
:10A8C0003F07DFF8E480DFF8E49016F801ABBAF157
:10A8D000000F21D12078F8B194F9023001331BD058
:10A8E00061780BF083FC0546039A01215846FFF777
:10A8F00065FF94F902205346294603902078CDE95C
:10A9000000B8FDF72BFA207853464FF0FF32294666
:10A91000CDE900B9FDF722FA0334BC42D5D10DB020
:10A92000BDE8F08FE0883FF0F7FC002E627AD0E9B6
:10A930000231207A04BF1946334605FB00228F56A8
:10A9400023B39E56B742039A5846049313BF01217E
:10A9500000214FF001084FF00008FFF72FFF049B84
:10A96000039043B1104B324629462046CDE900B34F
:10A970004346FDF7AFF90D4B29463A4620460135CF
:10A98000CDE900B34346FDF7A5F933E74FF0FF36B5
:10A99000D8E700236DE703323F2A7FF45CAF4FF026
:10A9A000FF386BE7340500244DAF0408099F040805
:10A9B000185D002470B5054608460C464FF068F84F
:10A9C000024670B10D2804D12146094851F0CCF956
:10A9D00038B12846064B074A0749BDE87040FDF7E5
:10A9E000C9BD03490548BDE87040FFF7A1BA00BFE3
:10A9F00027B60A0835B60A0840B60A086AB60A0831
:10AA000070B5054608460C464FF042F8024670B154
:10AA1000042804D12146094851F0A6F938B1284646
:10AA2000064B074A0749BDE87040FDF7A3BD03493F
:10AA30000548BDE87040FFF77BBA00BF78B60A084A
:10AA40007DB60A0840B60A088DB60A082DE9F0431B
:10AA500007469BB008460C464FF01AF806462022DF
:10AA6000002101A851F090F836B3402E08D04023C1
:10AA700032463A4938461BB0BDE8F043FDF77ABD8F
:10AA800001AD04F140084FF000090222214668465A
:10AA900051F07CF90023102209A968468DF8029034
:10AAA000FDF712FF099B0DF10202934223D10234FC
:10AAB00005F8010BA045E8D109AC41220021284D41
:10AAC000204651F061F8002E3BD095F85560D6B184
:10AAD000202205F1940101A851F0AAF998B105F1DD
:10AAE00094012046FDF720FE23461E4A38461E49A3
:10AAF000FDF740FD04E01A7838461C49FDF73AFDA1
:10AB00001BB0BDE8F0832B78DBB9D6B901AB184E8A
:10AB10001A46083603CAA24246F8080C46F8041C36
:10AB20001346F5D101232046114985F85430FDF72D
:10AB3000FBFD1048FFF737FE21460F48FFF7F8F9F5
:10AB4000DEE795F854301BB995F85530002BF3D05B
:10AB500007492046FDF7E8FDEEE700BFA0B60A086A
:10AB6000185D0024DEB60A0840B60A08C2B60A0814
:10AB7000AC5D0024E8B60A08F7B60A0810B5084626
:10AB80000749FCF719FD002815BF012400240548DA
:10AB90000548FFF708FE2046BDE8104007F028B939
:10ABA00004B70A080DB70A0834B70A082DE9F04FB0
:10ABB0000C4607468BB040F216203FF0ADFB224614
:10ABC000054600213846FFF7F9FD404B06461522A1
:10ABD0001B78002104A8002BD5E9024504BF2546B7
:10ABE0001C4650F0D1FF05F13F03039395F8009008
:10ABF000B9F1000F30D095F801A0002C63D02246A7
:10AC000000231178494557D1283392F80180012259
:10AC10006B4403F8182CD0453246384613BF012147
:10AC200000214FF0010B4FF0000BFFF7C7FD064668
:10AC300054B1B8F1000F07D0254B5A46414648465B
:10AC400000933B46FDF7D2F8224B5A465146484600
:10AC500000933B46FDF7CAF80335039B9D42C5D1DF
:10AC60003CB3651C0DF110084034DFF86490DFF848
:10AC700064A018F8013BCBB915F8013CB3B116B18B
:10AC80003046FFF790FD29783B4615F8010C00226D
:10AC9000CDF800900026FDF7A9F8002215F8010C68
:10ACA0003B461146CDF800A0FDF7A0F80335A542BC
:10ACB000DFD10BB0BDE8F08F01330332152BA0D1EB
:10ACC0004FF00008A7E7A046A5E700BF185D0024E5
:10ACD0004DAF0408099F04081A4B70B55B7905460F
:10ACE000012B18D1184B1B68ABB1184E0846B6F9AA
:10ACF000C849FCF777FE90B90846FDF76FFE00F5EE
:10AD000043730446B3F5C36F09D928461049BDE81B
:10AD10007040FDF72FBC0F48BDE8704043E50E487A
:10AD2000FFF741FD0D48FFF7E3F8FFF7C5F8306D79
:10AD30000FF070FE0AF078F82046BDE87040FCF78E
:10AD4000B3BB00BF542700247C220024185D0024DC
:10AD50007DB70A0850B70A0895B70A08B5B70A08B8
:10AD60002DE9F04385B0224EFBF716FE0269838978
:10AD700000250188044602928268DFF888800192EB
:10AD80004288DFF884901B4F009242681A48FFF710
:10AD9000CFF815B91948FFF7FFFCD8F800309D42ED
:10ADA00012DA3378052B21D809EB8303D3F850222C
:10ADB000B3882946013538460093063636F8043CF8
:10ADC000FFF7B6F8062DE4D145F0DAFE4288838815
:10ADD00064689B1A03FB0444FBF77AFE02460848AA
:10ADE000214605B0BDE8F043FFF7A2B80022DFE737
:10ADF000E46600242BB80A08C1B70A081FB80A087D
:10AE00003AB80A08B02F002424DD090810B504461A
:10AE10000748FFF7C1FCFCF791FA18B10548BDE8F7
:10AE20001040B9E420460449BDE81040FDF7A2BB3C
:10AE300057B80A0861B80A0869B80A0838B50C4654
:10AE4000054615492046FCF7B7FB28B9FFF70AF875
:10AE50001248BDE838409FE411492046FCF7ACFB9E
:10AE6000A0B9104B83F8210283F8290283F80B0361
:10AE700083F8130383F8F50383F8FD0383F8DF04F5
:10AE800083F8E70483F859050748E2E72846BDE858
:10AE90003840FDF785BB00BF70B80A0876B80A08CD
:10AEA00091B80A08185D002499B80A0838B50D460B
:10AEB0000446052219492846FDF7CAFC60B9184B1B
:10AEC00093F84C2022B9012183F84D2083F84C10CF
:10AED0001448BDE838405FE4032213492846FDF7D3
:10AEE000B7FCA0B90E4D95F84C3063B195F84D30D4
:10AEF0004BB10E492046FDF73DFB002385F84C3051
:10AF000085F84D3038BD0A48FFF746FCF5E7204686
:10AF10000849BDE83840FDF72DBB00BFDCCA0A0870
:10AF2000185D0024B5B80A0827CC0A0865B30A08DA
:10AF3000CBB80A08DFB80A08034B0146D3F88009EA
:10AF400008B107F09DBA7047185D00240CB407B52E
:10AF500010F020000BD079B92320FFF7EDFF05A9F1
:10AF600004980191FEF7B2FFFEF7CAFF012003B07B
:10AF70005DF804EB02B070470020F8E72DE9F04FD0
:10AF8000914687B00C461A46002180464D46FFF791
:10AF900015FC00270646B9F1000F63D029460622AA
:10AFA000204650F045FF00283246404613BF01219D
:10AFB00000214FF0010A4FF0000AFFF7FFFB0646A1
:10AFC000287814F077FF8346F8B1687914F072FF9F
:10AFD0004FF461714FF0190CAB78EA789BF805E0FB
:10AFE0001CFB03131CFB021295F801B0297900B178
:10AFF0004079CDE90410CDE9023251463B461A4A68
:10B000004046CDE900EBFFF7A1FF207814F052FF96
:10B010008346F8B1607914F04DFF4FF461714FF041
:10B02000190CA378E2789BF805E01CFB03131CFBCA
:10B03000021294F801B0217900B14079CDE90410F1
:10B04000CDE9023251463B46074A4046CDE900EB86
:10B05000FEF75AFF013706340635142F9BD107B08F
:10B06000BDE8F08FCA46D0E7EEB80A082DE9F041F6
:10B07000054686B008460F46FCF7B4FC064638B1D4
:10B0800000235B4901201A4606B0BDE8F04175E790
:10B090000846FDF7A3FC1328044600F3A08006250C
:10B0A0008DF81760534E4543781CFCF7D2FD0746D8
:10B0B00060B1FDF793FCC0B214F016FF30B1731904
:10B0C000027983F8902601238DF817303846FCF773
:10B0D000C0FD074668B1FDF781FC0D2809D806239D
:10B0E00003FB046383F891069DF8173001338DF854
:10B0F0001730DFF8FC80A91C0DF1170238464144D7
:10B10000FDF770FCFCF7A5FD074668B1FDF766FC8E
:10B11000012809D89DF817300622013302FB04628A
:10B120008DF8173082F894063846FCF792FD80B10E
:10B13000FDF754FCC0B214F0D7FE50B19DF81730A3
:10B140000622017902FB0462013382F895168DF81C
:10B1500017309DF817200623042A2FD103FB046320
:10B160000022A3F8942606251CF0CAFD05FB046501
:10B1700095F8900614F09EFE95F8931695F8927641
:10B1800019234FF46172804695F8950613FB01264A
:10B1900013FB072714F08EFE4379214698F805200B
:10B1A000039395F8943614480097CDE9016395F818
:10B1B0009136FEF7BDFE06B0BDE8F081052A05D147
:10B1C00003FB0463002283F89526CCE7062ACAD045
:10B1D000002308EB050248F805309380C3E71323EA
:10B1E00032460649284606B0BDE8F041FDF7E0B911
:10B1F000A8630024185D0024EEB80A0807B90A08FD
:10B200002DE9F04F904689B01A460C460021814640
:10B210004546FFF7D3FA3A4E08F178030746DFF8C0
:10B22000E4B0079394F904000CF0BAFE00285CD057
:10B23000B8F1000F61D029460C22204650F0F8FDED
:10B2400000283A46484613BF012100214FF0010A69
:10B250004FF0000AFFF7B2FA074695F9040043F0F1
:10B26000EFFDEA790346514606EB82024846D2F8E2
:10B27000682204922A7A06EB8202D2F868220392AC
:10B28000AA7906EB8202D2F8682202926A7906EB6A
:10B290008202D2F8682201922A6800925A46FFF789
:10B2A00055FE94F9040043F0CBFDE2790346514684
:10B2B00006EB82024846D2F868220492227A06EB14
:10B2C0008202D2F868220392A27906EB8202D2F8B7
:10B2D00068220292627906EB8202D2F86822019219
:10B2E000226800925A46FEF70FFE0C35079B0C347D
:10B2F000AB4297D109B0BDE8F08FC246D1E700BF9D
:10B3000024DD09080DB90A082DE9F04780468CB004
:10B310000846FCF767FB054638B100235949012070
:10B320001A460CB0BDE8F0476AE7CDE909000B907A
:10B3300007A80791544950F0D7FB064643F076FC26
:10B34000431C04460CD12B460A2208A93046FDF7BF
:10B35000BBFA089B1B781BB9C4B2132C0BD944B29F
:10B3600020460CF0D1FD054640B94046FDF718F9DE
:10B370000CB0BDE8F087333464B2F1E7424907A866
:10B380008DF8284050F0B0FBB0B3002302260A220B
:10B390001946FDF799FA09900027DFF8EC90DFF8DD
:10B3A000F0A0494607A850F09FFBF8B1FDF716FB47
:10B3B000364A002352F8041B88421FD1DBB20AEB45
:10B3C0008302D2F86822904210D1022F20D0032F9E
:10B3D00023D05A1E012FD2B215D00B2A03D88DF8D4
:10B3E00029300136F6B20137042FDAD1052E1AD8EA
:10B3F0004046FDF7D9F8BBE70126CDE70133102B16
:10B40000D8D10023DBE7052AEDD88DF82A30E8E70C
:10B41000092BE8D88DF82C30E3E79A1E0D2AE2D8E4
:10B420008DF82B30DDE709AB03CB28601868696025
:10B43000A860204643F004FD154A9DF82B100346F2
:10B4400002EB8101D1F8681204919DF82C1002EBF7
:10B450008101D1F8681203919DF82A1002EB810155
:10B46000D1F8681202919DF8291002EB81020021A7
:10B47000D2F8682208460192099A0092054AFEF71E
:10B4800043FD75E77862002425B60A088CDF0908B9
:10B4900024DD09080DB90A082DE9F04F90468BB05C
:10B4A00000264FF0190A45464FF461790C461A46BA
:10B4B00000210746FFF782F90990B8F1000F49D043
:10B4C00029460A22204650F0B3FC0028099A384643
:10B4D00013BF012100214FF0010B4FF0000BFFF7CC
:10B4E0006DF92A890990334606925946EA8838460A
:10B4F00005922A790492EA780392AA781AFB0292BA
:10B5000002926A781AFB029201922A780092124AF9
:10B51000FFF71CFD2289334601365946069238460C
:10B52000E2880A35059222790492E2780392A278A1
:10B530001AFB0292029262781AFB0292019214F8AC
:10B540000A2B0092044AFEF7DFFC1E2EB5D10BB089
:10B55000BDE8F08FC346DDE72AB90A082DE9F043BC
:10B5600080468BB008460F46FCF73CFA044638B1DB
:10B5700000235E4901201A460BB0BDE8F0438BE77B
:10B580000846FDF72BFA1D28054600F3A5800A267C
:10B590008DF827404643781CFCF75BFB10B1012374
:10B5A0008DF82730FCF755FB514C074668B1FDF785
:10B5B00015FA0D2809D80A2303FB054383F8F0097F
:10B5C0009DF8273001338DF82730DFF82091711C6A
:10B5D0000DF1270238464944FDF704FAFCF739FB20
:10B5E000074668B1FDF7FAF9232809D89DF82730F6
:10B5F0000A22013302FB05428DF8273082F8F30955
:10B600003846FCF726FB074668B1FDF7E7F90D2839
:10B6100009D89DF827300A22013302FB05428DF834
:10B62000273082F8F4099DF82730062B0CD0002330
:10B6300009EB0602404649F80630536013810BB00F
:10B64000BDE8F043FCF7B0BF0A260023384606FBEE
:10B650000546A6F8F639A6F8F839FCF7FAFA0746CF
:10B6600018B1FDF7BBF9A6F8F6093846FCF7F1FA70
:10B6700030B1FDF7B3F90A2303FB0543A3F8F8093A
:10B680001C4B4FF0FF324FF461705A600A2303FBEA
:10B690000542B2F8F8390693B2F8F639059392F8F4
:10B6A000F439049392F8F3390393192392F8F219B9
:10B6B00013FB0101029192F8F11913FB0103002120
:10B6C0000193084692F8F0390B4A00932B46FEF797
:10B6D0001BFC0BB0BDE8F0831D2322460749404602
:10B6E0000BB0BDE8F043FCF763BF00BF0867002460
:10B6F000185D0024240500242AB90A0807B90A089D
:10B700002DE9F04F804691461E460C46154600270F
:10B71000DFF81CA12DED088B95B094ED008AB5EEF5
:10B72000408AF1EE10FA7BD0D4ED019A94ED029AA2
:10B73000D4ED038AB9F1000F49D0D5ED00BA95EDEB
:10B7400001BAB4EE6B8AD5ED02AA95ED03AAF1EE2B
:10B7500010FA6AD1F4EE4B9AF1EE10FA65D1B4EE1C
:10B760006A9AF1EE10FA60D1F4EE4A8AF1EE10FA1C
:10B770000CBF0121002132468B46404681F0010179
:10B78000FFF71CF8B0EE6B0A064611A8FCF786F925
:10B79000B0EE4B0A07900EA8FCF780F9B0EE6A0AEB
:10B7A00006900BA8FCF77AF9B0EE4A0A059008A8B3
:10B7B000FCF774F90599069A079B0390404602919D
:10B7C00059460192524600933B46FFF7BFFBB0EE4D
:10B7D000480A11A8FCF762F9B0EE690A83460EA880
:10B7E000FCF75CF9B0EE490A06900BA8FCF756F995
:10B7F000B0EE680A059008A8FCF750F9069B059A78
:10B800000021039040460292524610341035CDE993
:10B8100000B33B460137FEF777FB082F7FF47DAF7F
:10B8200015B0BDEC088BBDE8F08F0021A3E700BF89
:10B830004DB90A082DE9F14F06460D46DFF88CB1E7
:10B840002846FCF7CFF8074638B1002358490120B5
:10B850001A4601B0BDE8F04F52E705225549284687
:10B86000FCF7F6FF60B9524B00221A601A611A62A7
:10B870001A631A641A651A661A6701B0BDE8F08F78
:10B88000042259462846FCF7E3FF04462846002CCC
:10B8900042D1FCF7DEF907460028EED04EF0F8F86A
:10B8A000DFF82CA15FFA80F85AF8049BB9F1000F79
:10B8B00007D12A464049304601B0BDE8F04FFCF7B9
:10B8C00059BE4246494638460134FCF7C1FF84461A
:10B8D0000028E9D1364A034600211546013342F8D3
:10B8E000101B082BFAD1354B03EBC40257682FB954
:10B8F00049463348334DFEF71BFBA1E713F834E00C
:10B90000F445F5DA07EB0C1305EB0C140CF1010C04
:10B910000FCB84E80F00F3E7FDF760F80728044633
:10B920003DD82846FCF795F9074658B3FBF7E2FEE9
:10B930001F4B012503EB041383ED000A3846FCF787
:10B9400088F9074638B1FBF7D5FE194B013503EBF3
:10B95000041383ED010A3846FCF77BF9074638B13A
:10B96000FBF7C8FE124B013503EB041383ED020A0B
:10B970003846FCF76EF938B9304601B0BDE8F04FF3
:10B98000FCF712BE0546D9E7FBF7B4FE084B032DC2
:10B9900003EB041383ED030A3FF457AFECE70723EF
:10B9A0003A460949304601B0BDE8F04FFCF700BE09
:10B9B0008035002461B90A08ADB40A0830D40908FA
:10B9C0006CB90A08E6BD0A0807B90A0867B90A0887
:10B9D000CCDF09082DE9F74F92460C461A460021A4
:10B9E00081465646FEF7EAFE00258046DFF864B041
:10B9F000BAF1000F2CD031460422204650F018FA3C
:10BA000000284246484613BF012100210127002794
:10BA1000FEF7D4FE738880465A46019339463AF8B9
:10BA20002530484600932B46FFF790FA63885A4624
:10BA3000394648460193043634F8043B00932B46BC
:10BA40000135FEF761FA042DD2D103B0BDE8F08FC5
:10BA50005746EBE776B90A082DE9F3410546084653
:10BA6000FBF7C0FF0C46074638B1002333490120DD
:10BA70001A4602B0BDE8F041ACE731492046FBF779
:10BA80009BFD70B904222D4B4FF47A704FF4FA618C
:10BA9000013A1880598003F10403F9D102B0BDE8DE
:10BAA000F0812046FCF79AFF0328064641D820463D
:10BAB000FCF7CFF8074698B1FCF790FF4FF001086C
:10BAC00004463846FCF7C5F820B1FCF787FFB8F10B
:10BAD000000F09D1284602B0BDE8F041FCF764BD73
:10BAE00040F2EE248046ECE7A4F2EE2240F2DC5372
:10BAF0009A4203D8A0F2EE229A420AD940F6CA032B
:10BB000040F2EE220F49284602B0BDE8F041FCF7B2
:10BB10004FBD0D4B00210D4A03EB8603A3F81C4BD0
:10BB2000A3F81E0B3346CDE900400846FEF7ECF9BA
:10BB3000B4E703233A460649E5E700BF346800242A
:10BB400061B90A0887B90A08185D002476B90A089D
:10BB5000F3B30A082DE9F04F8FB08946174600214C
:10BB60001A4606460024FEF729FE0DF1240B054671
:10BB7000DFF86CA059F82480594602A8CDF8088057
:10BB800043F00EF94FB357F824302A463046984513
:10BB9000039313BF012100214FF001084FF000086B
:10BBA000FEF70CFE04A9054603A843F0F9F804A922
:10BBB00023465246009130464146FFF7C7F92346D7
:10BBC0000134524641463046CDF800B0FEF79CF9AC
:10BBD000402CCFD10FB0BDE8F08FB846EFE700BFE3
:10BBE00095B90A08F0B5074689B008460E46FBF736
:10BBF000F9FE054638B10023194901201A4609B05B
:10BC0000BDE8F040A6E70846FCF7E8FE3F280446FA
:10BC10001DD83046FCF71DF80146204634F00AF9DD
:10BC200078B103AE0E48314600EB840043F0B8F81B
:10BC300023460C4A294628460096FEF765F909B0C6
:10BC4000F0BD384609B0BDE8F040FCF7A9BC3F2381
:10BC50002A460549384609B0BDE8F040FCF7A8BCC3
:10BC60004468002495B90A0807B90A082DE9F04F7D
:10BC7000924685B00C461A46002181465546FEF78D
:10BC80009DFD00268046DFF86CB0BAF1000F2FD082
:10BC900029460422204650F0CBF800284246484668
:10BCA00013BF0121002101270027FEF787FDEB7854
:10BCB00080465A4602933946AB78484601932B8812
:10BCC00000933346FFF742F9E3785A46394648462F
:10BCD00002930435A378019334F8043B0093334670
:10BCE0000136FEF711F9102ECFD105B0BDE8F08F67
:10BCF0005746E9E79FB90A08F0B5074685B00846F8
:10BD00000E46FBF76FFE054638B100231C490120A3
:10BD10001A4605B0BDE8F040A8E70846FCF75EFE0D
:10BD20000F28044623DC3046FBF793FF01462046EC
:10BD300034F05AF9A8B104F14002124B29462846C2
:10BD400003EB820393F82F2B029293F82E2B019290
:10BD5000B3F82C3B0C4A00932346FEF7D5F805B008
:10BD6000F0BD384605B0BDE8F040FCF719BC0F2324
:10BD70002A460649384605B0BDE8F040FCF718BC35
:10BD800044690024185D00249FB90A0807B90A080D
:10BD90002DE9F04F85B014461A4605460291002160
:10BDA000FEF70CFD4FF00008064606234FF0000991
:10BDB00003FB08F707F5A077029B13F807B0002CE8
:10BDC0007DD0E35D324628469B45039313BF012196
:10BDD00000214FF0010A4FF0000AFEF7EFFC039B31
:10BDE0000646394A51462846CDE900934346FFF7B7
:10BDF000ADF84346344A514628460137CDE9009B09
:10BE000009F10109FEF780F8B9F1060FD4D108F164
:10BE10000108B8F1060FC8D14FF4B277029BA7F51D
:10BE2000B27913F807A0002C4BD014F807B03246B3
:10BE30002846DA450DBF4FF001084FF000080121F8
:10BE40000021FEF7BBFC062306461F4A4146284652
:10BE5000CDE9009BFFF77AF806231B4A41462846A6
:10BE60000137CDE9009AFEF74FF840F26F139F4279
:10BE7000D4D1029B93F86F71ACB194F86F813246C4
:10BE80002846474513BF0121002101240024FEF765
:10BE900095FC00230C4A2146009328460723CDF841
:10BEA0000480FFF753F80023074A214628460093F1
:10BEB00007230197FEF728F805B0BDE8F08FA246EA
:10BEC00097E7A046C8E700BFB1B90A08F0B5054634
:10BED00085B008460B46FBF785FD044638B10023C4
:10BEE0001B4901201A4605B0BDE8F04050E701AEFD
:10BEF000184F6A46174918464FF023FE88B1032CA5
:10BF000004D12846FCF750FB05B0F0BDFCF766FDF8
:10BF10006A4646F8040B3946002001344FF011FE02
:10BF2000ECE7032CEDD1039FDDE901463A463146AB
:10BF3000E0B234F093F818B92846FCF731FBE3E798
:10BF40003B46324621460448FDF7F2FFDCE700BFDE
:10BF50004468002425B60A08B1B90A082DE9F04F53
:10BF60009246002689B04FF019095546B3464FF462
:10BF700061780C461A4600210746FEF71FFC079021
:10BF8000BAF1000F27D02946062220464FF050FF75
:10BF90000028079A384613BF012100214FF0010BFA
:10BFA0004FF0000BFEF70AFC6A790790334619FB45
:10BFB00002825946384605922A7919FB0282049278
:10BFC000EA780392AA7802926A7801922A7800921B
:10BFD000104AFEF7BBFF627933460136594619FB1A
:10BFE0000282384606350592227919FB02820492B4
:10BFF000E2780392A27802926278019214F8062BFA
:10C000000092044AFDF780FF0A2EB9D109B0BDE8BD
:10C01000F08F00BFC5B90A082DE9F04F074689B077
:10C0200008468B46FBF7DEFC054638B100234C4939
:10C0300001201A4609B0BDE8F04F8FE7494B08468A
:10C0400093F82CA793F82D9793F81688FCF7C6FC65
:10C05000092804467BDC06268DF81F50404D4643D8
:10C060000BF10100FBF7F5FD834638B1FCF7B6FC98
:10C070000D2803D80123A8558DF81F305846FBF72B
:10C08000E8FD834660B1FCF7A9FC504508D80623BB
:10C0900003FB045358709DF81F3001338DF81F3097
:10C0A0005846FBF7D6FD824660B1FCF797FC484541
:10C0B00008D8062303FB045398709DF81F30013302
:10C0C0008DF81F305046FBF7C4FD814660B1FCF788
:10C0D00085FC804508D3062303FB0453D8709DF8E4
:10C0E0001F3001338DF81F30311D0DF11F024846FE
:10C0F0002944FCF777FC9DF81F30062B09D000235C
:10C10000AA193846AB51938009B0BDE8F04FFCF74F
:10C110004BBA63434FF461761921EA18507911FB49
:10C1200000600590107911FB00610491D1780391B2
:10C13000917802910021527808460192EB5C0A4AFC
:10C1400000932346FDF7E0FE09B0BDE8F08F092318
:10C150002A460649384609B0BDE8F04FFCF728BA30
:10C16000E0360024185D0024C5B90A0807B90A089A
:10C170002DE9F04F14468BB00F461A4600210646B3
:10C18000FEF71CFB0546002C00F0D78022783B7898
:10C190009A42024630460DBF4FF001084FF00008AA
:10C1A00001210021FEF70AFB237805469B4A414600
:10C1B0003046FEF7CBFE3B784146984A3046FDF7C5
:10C1C000A3FE002C00F0BB80627830467B789A4258
:10C1D0002A460DBF4FF001084FF000080121002151
:10C1E000FEF7ECFA637805468D4A41463046FEF785
:10C1F000ADFE7B7841468A4A3046FDF785FE07F161
:10C20000C90307F1020A04F1CA0B0593A31C4FF0FE
:10C2100000090693822307933B784B4500F39180F6
:10C22000002C00F0F58097F8EA30304694F8EA20C8
:10C230009A422A460DBF4FF001084FF00008012135
:10C240000021FEF7BBFA94F8EA300546754A4146EC
:10C250003046FEF77BFE97F8EA304146714A304699
:10C26000FDF752FE002C00F0D58004F1EA0307F13F
:10C27000EA0204F1FA014FF0010833F802CF32F874
:10C28000020F844518BF4FF000089942F5D188F09D
:10C2900001012A463046C9B2FEF790FA0821054648
:10C2A00004F1EC00FCF720FA5F4A034641463046B1
:10C2B000FEF74CFE97F8EA1007F1EC00FCF714FAD1
:10C2C000594A034641463046FDF71EFE002C00F059
:10C2D000A3804FF0FC094FF0010807EB090104EBC4
:10C2E0000900FBF769F909F10409002818BF4FF0AC
:10C2F0000008B9F58E7FF0D188F001012A4630465A
:10C30000C9B2FEF75BFA082104F1FC00FBF7B3FCAD
:10C31000464A034641463046FEF718FE97F8EA10B3
:10C3200007F1FC00FBF7A7FC404A034641463046B4
:10C330000BB0BDE8F04FFDF7E7BDA0463BE7A046D8
:10C3400057E7079BFB180993002C5FD0079B0998C0
:10C35000E31819460893FBF72FF9059B5A789BF8C9
:10C3600000309A424FD1B0FA80F84FEA5818069A36
:10C37000AAF102030AF10E01023A33F802CF32F8B1
:10C38000020F844518BF4FF000088B42F5D188F0AA
:10C3900001012A463046C9B2FEF710FA62780699C2
:10C3A00005469BF81800FCF771F902909BF80030E5
:10C3B00041461F4A30460193089B009309F101034F
:10C3C000FEF7C4FD059B51467A7809F10109587EB4
:10C3D0000AF1100AFCF75AF9059A0290414612F840
:10C3E000013F30460BF1010B0193099B059200932D
:10C3F0004B460F4AFDF788FD069B10330693079BBB
:10C400000933079308E74FF00008B0E7A046D9E7E3
:10C41000A04620E7A0464DE7A0467FE7DEB90A0820
:10C42000F0B90A081EBA0A0836BA0A084DBA0A084C
:10C4300005BA0A082DE9F04F8FB004460846B24904
:10C4400002AA4FF07EFB054640B903460246AF49BB
:10C450004120FFF78DFE0FB0BDE8F08FAC49FBF730
:10C46000ABF8064628BB02AAA7494FF06AFBFCF7C7
:10C47000B5FA0828054606D908233246A5492046BC
:10C48000FCF796F8E7E7A44C94F82C3783420CDCD1
:10C4900084F82C57DFE731460136384632F030FD5C
:10C4A00094F82C37B342F6DCF2E7064604F22C7718
:10C4B000F6E79A492846FBF77FF80646E0B902AA54
:10C4C00091494FF03EFBFCF789FA0828054603D94D
:10C4D000082332469249D2E78F4C94F82D37834295
:10C4E00002DC84F82D57B6E730460136294642F083
:10C4F00075FB082EF8D1F4E78A492846FBF75CF86B
:10C50000064600BB02AA80494FF01BFB0028A2D0C0
:10C51000FCF764FA0828054603D908233246824905
:10C52000ADE77D4C94F81638834209DD014604F2EC
:10C530002C7032F02BFD294604F22C7032F034FDC1
:10C5400084F8165887E779492846FBF735F80646F8
:10C5500018BB06AD704BDFF8B0910146A84610221B
:10C56000284693F816784FF00FFBBE4202AA80F2DD
:10C570000A81494600204FF0E4FA10B93A466C4966
:10C580000AE1FCF72BFA013628F8020BEDE7694CBB
:10C5900095E80F0084E80F005DE767492846FBF740
:10C5A0000BF80646C0BB5C4B06ADDFF85C9193F818
:10C5B0001678BE4202AA80F2F380494600204FF06E
:10C5C000C0FA014610B93A465C49E5E0AA464FF088
:10C5D0000008032228464FF0D9FB28464DF058FAB0
:10C5E000404502D801360435E3E79AF8000008F127
:10C5F0000108FCF727F90AF8010BEEE7B60004463C
:10C600004F4DB4423FF427AF06AB28190322191946
:10C61000043432F05FFCF4E74A492846FAF7CCFFCD
:10C620000746002840F0AC80DFF8EC8002AA3649CB
:10C6300098F82C674FF085FA00283FF40CAFFCF710
:10C64000CDF9451E01D4AE4203DC334601223E49FA
:10C6500015E72D4902AA00204FF073FA0146002881
:10C660003FF4F9AE00260DF10C09082203A88DF85D
:10C6700014604FF08BFB03A84DF00AFAB0421BD8B0
:10C6800002AA214900204FF05CFA00283FF4E3AEF3
:10C690000026037898F82DA7B1460193564502AAC3
:10C6A00019494FF0000080F285804FF04AFA834626
:10C6B00050B9524625496FE099F800000136FCF761
:10C6C000C1F809F8010BD6E7A6B99BF80030303B5A
:10C6D000092B0FD91E49FAF76FFF38B11D4958468B
:10C6E000FAF76AFF70B15A461B4955E04FF001094D
:10C6F0004FF0FF365846FCF771F9002830DA5A46F9
:10C70000164949E0B146F3E725B60A084464002417
:10C7100064BA0A086ABA0A08185D002475BA0A08D9
:10C720007EBA0A088CBA0A0898BA0A08AABA0A088D
:10C7300099BB0A0830650024D4BA0A08B9BB0A08B4
:10C7400040650024FEBA0A0803BB0A08D9BB0A08E0
:10C75000BBB30A080FBB0A0816BB0A084BBB0A0882
:10C760000EAB03EB4603013623F8200C96E7524646
:10C770001F4911E033F8022B013724F8022F30E073
:10C780002A461C4908E01C4900204FF0DAF900282D
:10C790003FF4FDAE3A4619492046FBF7EBFE5AE658
:10C7A000154900204FF0CDF900283FF427AF3A4655
:10C7B0001349F1E74FF0C5F90028D8D105EBC500C2
:10C7C000104C082203A98230204404EB051432F0F7
:10C7D00081FB0198FCF736F808EB050383F8F607B0
:10C7E00006ABBE42C6DC454485F80E9833E600BF72
:10C7F00060BB0A0883BB0A0825B60A08B6BA0A084D
:10C80000E0BA0A08446400242DE9F04F0F46904630
:10C8100089B0002187EA08080646139A0025039389
:10C82000FDF7CCFFDFF884906FEA08030446069317
:10C8300028460BF07FF9129B184230D0069BDFF898
:10C8400070B0034014BF4FF0010A4FF0000A049388
:10C8500010EA070328460CBF4A465A46059307923A
:10C860000BF07AF9039B8046079A514600903046B8
:10C87000FEF76CFB049B22463046B3FA83F149096C
:10C88000FDF79CFF059A0446039B002A0CBF5A46FD
:10C890004A4651463046CDF80080FDF735FB01355C
:10C8A000172DC5D109B0BDE8F08F00BFFEBB0A0847
:10C8B0005BB90A082DE9F04F3B4C89B00A460021CC
:10C8C0000546FDF77BFF059094F9000008F00EFB8C
:10C8D000814660883DF020FD344BD0F808B01F78C9
:10C8E00017B15F46D0F80CB0A3790026012B38BFF2
:10C8F000012306932279637906FB02331BF8038038
:10C90000002F3AD0FB5C4345059A2846079313BF96
:10C91000012100214FF0010A4FF0000AFDF74EFF00
:10C92000079B0136059053B303F00F021B095146D4
:10C930002846403302921E4ACDE900634B46FEF77B
:10C9400005FBB8F1000F24D008F00F034FEA1818C8
:10C95000174A5146029308F140032846CDE9006387
:10C960004B46FDF7D1FA069BB342C3DC0834114BAA
:10C97000A342A9D109B0BDE8F08F3B46C3E7002F21
:10C98000DFD04B460C4A514628460096FEF7DEFAA9
:10C99000D7E76B06E7D44B46074A51462846009630
:10C9A000FDF7B2FADFE700BF3CE00908185D00249C
:10C9B00005BC0A085CE109081BBC0A082DE9F04126
:10C9C0000D4688B006460846FCF708F820210446C4
:10C9D00028464FF0F0F828B9304608B0BDE8F041DD
:10C9E000FBF7E2BDFBF7FAFF224605460146104879
:10C9F000FDF79EFA85B1202D2A466946204628BFBC
:10CA00002022E846FAF7ACF900270646B74208DBD1
:10CA1000AD1B3444002EEDD1FDF772FA08B0BDE82D
:10CA2000F08118F8010B0137FEF786FAEEE700BF38
:10CA30002FBC0A080FB407B504A951F8040B0191E3
:10CA4000FDF744FA03B05DF804EB04B070472DE93C
:10CA5000F041037903F0E002402A4DD009D83ABBF7
:10CA600003F00703052B1ED8DFE803F0181D181D7F
:10CA70000910602A47D0802A41D0BDE8F081D0F863
:10CA800005102348BDE8F041FDF752BAD0F8052063
:10CA900051422048BDE8F041FDF74ABAB0F80720FE
:10CAA000B0F80510F5E7B0F90720B0F90510F0E788
:10CAB00046790024184D194805EBC605FDF718FA0C
:10CAC000012395F83C74A74203D8BDE8F041FDF777
:10CAD00017BAD5F838644FEA840856F824204AB1CA
:10CAE00013B90F48FDF704FA56F808100D48FFF780
:10CAF000A1FF00230134E6E741790B48C2E78279C0
:10CB000041790A48C6E70A48BDE8F041FDF710BA86
:10CB100047BC0A085DBC0A0824DD090874BC0A0881
:10CB200065C10A08D2C90A0885BC0A0896BC0A0869
:10CB3000ADBC0A082DE9F04F0346A1B00846FAF74C
:10CB400051FF054628B1184621B0BDE8F04FFBF76C
:10CB50002BBDFF23DFF8C09207464FF0FF388DF85A
:10CB60002830D9F850300B9093F83820ADF83000C9
:10CB70000D908DF838200F90ADF840001193099179
:10CB8000CDE90500934909A84EF0AEFF044618BB55
:10CB900001460AAC904F0B0190481A57002310F938
:10CBA000016BB24240F0D2804E1C104642F048F970
:10CBB000024631463846FDF7BBF9022E4FF001011F
:10CBC000E9D19DF938A09DF92830534540F0C58042
:10CBD0008348FDF7ADF94DE02378002BD2D0032F29
:10CBE000D4BF00260126062F00F2A980DFE807F057
:10CBF0000447509104475000042F10D07949204633
:10CC0000FBF74AFE58B14FF480600DF0A1FE0028FA
:10CC100000F0B58190F90400012306930AE07249FF
:10CC20002046FAF7C9FC70B9D9F8503093F93800AA
:10CC3000042F22D0119B119320AB03EB061606F8AC
:10CC4000580C01379EE7204641F0F0FF0028EFDA4C
:10CC500001230A2212A92046FBF736FE40B2002823
:10CC600003DB129B1B78002BE2D02246711C5F482D
:10CC7000FDF75EF921B0BDE8F08F0023DBE7204629
:10CC8000FBF7ACFE20AB03EB061646F8540CD8E7D6
:10CC900057492046FBF700FEB0F1000A55492046EF
:10CCA00018BF4FF0010AFBF7F7FD08B14AF0020A7E
:10CCB0003301DFF868C1079320AB03EB0616BCE82D
:10CCC0000F0006F850AC12AE0DF1480A0FC6BCE8D2
:10CCD0000F000FC6BCE80F000FC69CE8030086E8F3
:10CCE00003000026B346DAF8001020464FF08AF819
:10CCF00010B19AF804301E430BF1010B0AF1080A37
:10CD0000BBF1070FEFD1079B80336B4403F84F6CE7
:10CD100097E739492046FAF74FFCA0B1374920463A
:10CD2000FAF74AFC00288CD02046FBF757FE032870
:10CD3000804686D901463248FDF7FAF89AE722463E
:10CD40000821304894E7012305937AE701330A2B41
:10CD50007FF425AF01312C488AE70B9B1BB9AAF160
:10CD600014025542554100235F1CE368002B62D139
:10CD700094F900B058460BF013F9D4F8049018B1A8
:10CD80000668002E40F08B80B9F1000F237A14BFA3
:10CD90004E464FF46146666023B91C48FDF7C8F85B
:10CDA00003232372627A2AB1394619480792FDF7A4
:10CDB000BFF8079A02925846237ACDE90063002310
:10CDC0001A4619460DF043FEE06048BB394611484B
:10CDD000B2E700BF25B60A0841BD0A0823D40908F6
:10CDE0005EBD0A08E0BC0A08EBBC0A08EFBC0A08F2
:10CDF0000ABD0A08ABCB0A0861B90A08F7BE0A08DF
:10CE00000DBD0A0825BD0A084CBD0A0877BD0A08F1
:10CE100092BD0A08ADBD0A08185D002414E3090894
:10CE200058493346584A5948B9F1000F18BF0A46C5
:10CE30003946FFF7FFFD022F04F110044FF0010304
:10CE400092D1119E0D9F4DB15148FDF7A5FC33685D
:10CE50001B6A1BB13A464F4930469847059B002B49
:10CE600050D04D49474BBAF1140F18BF19464B48E3
:10CE7000FDF75EF8BAF1140F09D1059B002B43D0E2
:10CE80003368DB691BB10022454930469847069B51
:10CE9000002B43D100223146384641F0DFFEE660E8
:10CEA000B9F1000F2CD04946304602F079FE3D4AD8
:10CEB000B36839463C48FDF73BF894F80890B9F15F
:10CEC000000F0CD03279914509D04B46394637488E
:10CED000FDF72EF83368494630469B699847637AD8
:10CEE00023B1727939463248FDF722F8F36A002BF4
:10CEF000A1D039462F48FDF71BF80023F3629AE7CB
:10CF0000204AD5E71F49B2E7B8F1000FBFDB33680D
:10CF1000DB69002BBBD042462749B6E7DFF89C907F
:10CF20000025DFF89CA04FF0030B07F099FF0520C8
:10CF3000F9F7EAF99AF80030AB42ABD919F8014F8A
:10CF4000C4B1204609F076F9804698B12046F6F73C
:10CF5000B1FF0446EBB210B180F806B0C3712046B1
:10CF60000121F6F751F998F806302046DB0703D582
:10CF7000F5F77CFF0135DDE7F5F772FFFAE74FF0D3
:10CF8000FF3049E6E6BD0A08C5BC0A08C9BD0A0863
:10CF90007FBE0A08A1FB0408D3BC0A08A8BE0A0881
:10CFA0006B7C0408CEBC0A08E7BD0A080CBE0A0860
:10CFB0002FBE0A0866BE0A08F5790408B72E0024B9
:10CFC000481C0020194B1B682DE9F0415BB300257C
:10CFD000174FDFF868801748FDF7DEFBFCF76CFFA2
:10CFE000F9F7EAFCF9F728FD044648B113200DF0E3
:10CFF00005FEFCF785FF1048BDE8F041FDF7CCBB0E
:10D000003B78012BF2D040466E1CFFF713FD792DC3
:10D0100002D12646FCF774FFFCF74EFF642035462C
:10D02000F9F772F9DEE7BDE8F08100BF7C22002449
:10D03000BA2F0024CBBE0A08E5BE0A0816CD0A089E
:10D040002DE9F74F019008460E46174698464CF0DA
:10D050001FFD0446E8B9404D4048FFF7EBFC204671
:10D060000AF068FD3B68184206D020460AF074FDBD
:10D0700001462846FFF7DEFC0134172CEFD13B6850
:10D0800013B93748FCF734FF03B0BDE8F04FFCF7A5
:10D0900037BF024633493046FBF7DAFB0546A8B9ED
:10D0A0002C46314D3148FCF723FF20460AF042FD63
:10D0B00010EA080F06D020460AF04EFD0146284629
:10D0C000FFF7B8FC0134182CEFD1DDE733782D2BB6
:10D0D00029D10136013C01254FF0000948F4000B2D
:10D0E00048460AF039FD2246824601463046FBF7A3
:10D0F000AFFB18BB48460AF01DFD1BEA000F1DD010
:10D100009DB1B9F1170F02D03B6840EA03081848F7
:10D11000C7F80080FCF7ECFE5146134803B0BDE8A9
:10D12000F04FFCF705BF0025D6E7B9F1170F02D085
:10D130003D6825EA00050F483D60EBE709F101096C
:10D14000B9F1180FCCD132460B49019803B0BDE8B4
:10D15000F04FFBF70FBA00BF8EC10A08EBBE0A08FA
:10D16000F5BE0A08DEC20A088FC10A08FCBE0A081A
:10D1700071B40A0881B40A08ADB40A0840F2022367
:10D18000004A5DE788360024014B024A58E700BF99
:10D19000FFFF7F00803600242DE9F04F074691B055
:10D1A00082480E46824DFCF7C3FE0023814940248D
:10D1B000062285F8A03C304601230978C5F89CDC9E
:10D1C00085F8A14C05F02AF90A20F9F79DF895F8A1
:10D1D000A03C0C2BDAB240F2E4809DF80C60FE2EED
:10D1E0002CD0FF2E15BF0F241524002501259442B5
:10D1F00040F0D780611E6846C9B238F01DFB04F1CB
:10D2000040030DEB030414F8413C834240F0C4801A
:10D210006A1E9DF80D30012A12D903F01F075C0920
:10D2200061376548FCF764FE022D39D0013C042CBF
:10D2300034D8DFE804F00B2D2F3331000225D6E778
:10D240009DF80E701E469DF80F40EAE75B486C465D
:10D250004FF00008DFF8BC91FDF79EFADFF8B8A1A7
:10D26000DFF8B8B15648FCF743FE08F1010814F89E
:10D27000011B4846FFF7DEFBB8F10C0F16D00AFB86
:10D2800008F3B3F1553FF0D85846FCF731FEECE710
:10D290004C48DCE74C48DAE74C48D8E74C48D6E73E
:10D2A00000230DF11F008DF83F30D0E7FCF728FE7A
:10D2B000022D3AD064223B464648B6FBF2F102FB0F
:10D2C0001162C9B2D2B2FCF733FE85F001035B42B2
:10D2D000DBB2012B59D8404A404B9DF81010404812
:10D2E00000290CBF114619463E4EFCF721FE9DF861
:10D2F00011103D4B3D4800290CBF31461946FCF743
:10D3000017FE022D41D19DF812403948FCF7F0FD7F
:10D310008CB1FF2C1FD00A233648B4FBF3F103FB7A
:10D320001142D2B2FCF704FE08E03A4631463248D8
:10D33000FCF7FEFDCFE73046FDF72EFA9DF81340CF
:10D340002E48FCF7D5FD44B1FF2C21D021462C48B6
:10D35000FCF7EEFD04E02B48EEE72248FDF71CFA4F
:10D360000DF1130500241F4E1F4FDFF8988015F8AC
:10D37000013F7BB1FF2B14BF3A46424621460134A0
:10D380002148FCF7D5FD042CF1D111B0BDE8F08F98
:10D390001C48E3E73246F1E71C493846FBF7EAF858
:10D3A000F3E71B48FDF7F8F9EFE700BF27BF0A08CE
:10D3B000185D0024481C002038BF0A0843BF0A0833
:10D3C00071BF0A084ABF0A0852BF0A085ABF0A08B2
:10D3D00069BF0A0883BF0A0810BF0A0807BF0A0806
:10D3E000BABF0A0817BF0A087ECB0A08D1BF0A08CD
:10D3F000D8BF0A08ECBF0A089FBF0A08F4BF0A0892
:10D4000071BC0A081BBF0A0804C00A080FC00A083A
:10D410001FC00A08D1B30A08ABAAAAAAEFCD0A080E
:10D420002DE9F74F05460846FAF7DCFA0B460446A5
:10D4300018B9334A92F8A27C2FB9284603B0BDE848
:10D44000F04FFBF7ADB82646DFF8C890DFF8C8A06C
:10D4500001AA2C4918464EF074FB10B907F00CFDD8
:10D4600008E056B9012201462846FCF7C9FF421CD4
:10D4700004461AD103B0BDE8F08FFBF7AFFA2F28AE
:10D48000834636D80FB107F0EBFCBBF1060F13D083
:10D490001D4901235FFA8BF20978E0B204F0BEFF68
:10D4A000002759464846FCF743FD01AA15490020CC
:10D4B00001364EF046FBD0E7DAF800301B0114D5F8
:10D4C000FF2C0ED0E1B22846FFF766FEE8E70137F1
:10D4D0002846FFF761FEF9B298F800208A42F6D894
:10D4E000DEE70027DFF82080F5E70848FDF754F96C
:10D4F000D6E72F2206492846FBF73CF8D5E700BFC0
:10D50000185D002425B60A08481C0020BEB40A088D
:10D5100039C00A0828C00A08B43400242DE9F843A9
:10D5200007460C46DFF8A09020464CF0B1FA0646BC
:10D5300058B91D4B1D481A781D4B03EB8203D3F8D5
:10D54000A412BDE8F843FCF7F3BC02464946204666
:10D55000FBF77EF960B1DFF86080002558F8041B06
:10D56000B1B9224638461349BDE8F843FBF702B883
:10D57000114C124D1248FCF7BBFC54F8041B19B1B6
:10D580002846FFF757FAF8E7BDE8F843FCF7B8BCC0
:10D59000324620460135FBF75BF90028DED1024B0D
:10D5A000084C1D70C0E700BF7835002459C00A0838
:10D5B00024DD0908ADB40A08CCDF09088FC10A08C8
:10D5C000FCBE0A08E6BD0A08DEC20A08B04B42F2F9
:10D5D00001011A68B1EB124F4FEA12432DE9F047EF
:10D5E00090B000F0508142F20302934200F04D816E
:10D5F00041F20302991A4B424B41A64A4FF00008F0
:10D60000A54D1168464605EBC303A44AA44CA548A2
:10D61000A54FB1FBF2F2D3F82C16FFF70BFAB4F8D2
:10D62000A42C4FF47A730A20B2FBF3F103FB11220E
:10D63000B4F9A63C92B2B2FBF0F29C48FCF778FC3D
:10D640009B4A9C499C48FFF7F5F9FCF759FC9B4B1A
:10D650009B4A997B9B4B05EB81019B48D31AB4F8FD
:10D660007628D1F84816FCF763FCFCF749FC97488C
:10D67000FCF73EFC94F8A81C9548FFF7DBF99548A9
:10D68000FCF736FC944B94F8A91C1A88934892B284
:10D69000FFF7D0F9FCF734FC91499248FFF7CAF93B
:10D6A000DFF8B49294F8573503F00103B8F1000F96
:10D6B00000F05681002E40F087818B48FDF76CF812
:10D6C0008A4F0126D4F8B08CDFF8909207F1180A3F
:10D6D0000123B34013EA080F15D019F8062057F8B4
:10D6E00026305AF8261053F822208148FFF7A2F975
:10D6F000012E06D17F4B93F8211011B17E48FFF720
:10D7000099F9FCF7FDFB0136062EE1D17B48FCF7C9
:10D71000EFFB7B4B1B681B0640F18A8194F8D03CE1
:10D72000032B8CBF77487848FCF7E2FB94F8E03590
:10D73000022B40F04C817548FCF7DAFB94F8D03CA2
:10D74000042B00F26C817248FCF7D2FB94F8E03CA9
:10D75000002B00F06B8105EBC303D3F8E4166D4892
:10D76000FFF768F9FCF7CCFB6B4B6C481E686C4B01
:10D770001B7805EB8303D3F81817FFF75BF926B185
:10D78000327A717A6748FFF755F9FCF7B9FBF9F778
:10D7900003F9016921B182686348120DFCF7C8FBE7
:10D7A000FCF7AEFB614B624819684FF47A73B1FB2A
:10D7B000F3F1FFF73FF905A8FBF702FA38B105A925
:10D7C00008A84BF091FF08A95A48FFF733F9FCF776
:10D7D00097FBD4F86C7D002F00F02E8107EE907A35
:10D7E000DFED556AB8EEE77AC6EE877AFDEEE77AA6
:10D7F00017EE903A514E96F86C0330B1504A0393AD
:10D8000092ED320A4DF08AFC039BD4F8EC4C5CB1EB
:10D8100007EE904ADFED486AF8EEE77A86EEA77ADF
:10D82000FDEEC77A17EE904A324AB2F870103A46C7
:10D830006429CDE90004A8BF64214248FCF778FBC5
:10D84000B6F8702364234048B2FBF3F103FB1122C6
:10D8500096F8813305EB830592B2D5F82C37012574
:10D86000009396F88033FCF763FB3848FCF740FBE5
:10D87000374B384E1C68002C40F0E080FCF740FB32
:10D8800010B0BDE8F0870223B7E60323B5E600BF7A
:10D890000010005C0004002424DD090840420F0051
:10D8A000185D002463C00A08A01D002075C00A0886
:10D8B000F8FF01200008000097C00A0898340024EF
:10D8C0000000040800000208A9C00A08C0C00A0835
:10D8D000D2C00A08DAC00A0848250024DCC00A08B9
:10D8E000F0C00A08F5C00A0814C10A08D4E3090800
:10D8F0006EC60A086433002019C10A081DC10A084F
:10D90000B434002423C10A082FC10A083FC10A0801
:10D910001FCE0A0883C10A08483A00249FC10A089A
:10D92000443A0024A8C10A08B2C10A08541B0024C2
:10D93000CDC10A08E7C10A0800247449106E00240A
:10D9400024050024FAC10A0840C20A0865C20A0870
:10D95000703600248FC10A0865C10A08E405002456
:10D96000002B3FF4A7AE16B14846FCF7C1FA0121DF
:10D970003A48FFF75FF894F8AC3C394805EB83036D
:10D98000D3F85016FFF756F897F8CE33DA0702D5DA
:10D990003448FFF74FF897F81831032B09D0324875
:10D9A000FFF748F897F81831012B02D12F48FFF7FD
:10D9B00041F8FB6C01265B7BB046B3427FF672AE4A
:10D9C0002B48FFF737F86BE6FCF79AFA78E6022067
:10D9D0000CF0BEFF064608B92648ADE690F90400F3
:10D9E00041F02EFA074632F0BFF805EB80003946C9
:10D9F000D0F868222048FFF71DF894F8E335012B92
:10DA000004D11E48FCF774FA1D4895E6B3791D4809
:10DA100005EB8303D3F86812FFF70CF8F4E794F8EA
:10DA2000E2350BB918488FE618488DE6184996E696
:10DA30001848FCF75DFA95E63B46DBE694FAA4F05D
:10DA4000B0FA80F005FA00F024EA00040AF05AF86F
:10DA500001463046FEF7EEFF0DE700BFFAC00A08A8
:10DA60008FC10A08C0C90A08FFC00A0807C10A080E
:10DA70000CC10A0845C10A084FC10A085FC10A085B
:10DA800064C10A0826B90A0868C10A0878C10A08E8
:10DA900069BF0A0893C10A082DE9F04FDFF86C81CD
:10DAA00099B098F80330002B00F093804E48002581
:10DAB0004E4EDFF85CB1FCF76FFE2F46DFF8549155
:10DAC000DFF854A10BA9E8B214F02CFB9DF8343018
:10DAD000002B53D0139C54B107EE904A9FED440A9B
:10DAE000F8EE677A80EE270A4DF018FB04460B9A91
:10DAF00029465846FEF79EFF109A002A6BD002FB7B
:10DB000004F04FF47A73B0FBF3F30993DDF848C0E7
:10DB1000BCF1000F61D00CFB04F142F21073B1FBB9
:10DB2000F3F1082D98F8033018BF7F18002B56D05A
:10DB300017984FF47A7E0A23079015980690169846
:10DB400005901198B0FBFEFECDF810E00998B1FBEE
:10DB5000F3FE03FB1E11CDE902E10999B1FBF3F1DC
:10DB600003FB1100BCFBF3F3CDE900102146504646
:10DB7000FCF7DEF90023B362C6E90D330135403608
:10DB80001E2D9FD198F8033003B31A4C4FF47A73CB
:10DB90001948D4E9E112B1FBF3F3D208D4F88C139D
:10DBA000FCF7C6F90A22154897FBF2F102FB117245
:10DBB000FCF7BEF9124B1B78432B04D11148D4E972
:10DBC000E421FCF7B5F90023C4F88C3319B0BDE8A3
:10DBD000F08F0D486BE7099298E76146A1E721466F
:10DBE0004846FCF7A5F9C5E77BC20A08FC69002492
:10DBF0008096184B106E002422C30A0842C30A08FC
:10DC00009F26002466C30A08D9C20A089834002453
:10DC1000E3C20A086EC90A08F2C20A0810B5114B1D
:10DC200086B0114904460493104B11480393114BDD
:10DC3000114A0293114B0193114B0093114BFEF7C4
:10DC4000F9FEFCF75DF910491048FCF771F93CB199
:10DC50000F4A1049104806B0BDE81040FCF768B9FB
:10DC600006B010BDD0C30A089AC30A08D5C30A0873
:10DC7000A5C30A08DFC30A0890C30A08E8C30A0854
:10DC8000F4C30A089F340024FEC30A0806C40A0825
:10DC900027B60A0878B60A0817C40A080120BDE7A3
:10DCA000234870B5FCF724F9224B93F86C33002B12
:10DCB00038D0214B93ED320A4DF030FA01461F481F
:10DCC000FCF736F91E4C1F48FCF712F91E4B94F86E
:10DCD00021001E4A00280CBF10461846FCF75CFDC8
:10DCE00094F8213013B31A4C1A48B4F80611FEF711
:10DCF000A1FE194E94F80401184D00280CBF3046BF
:10DD00002846FCF749FDB4F808111548FEF792FEC5
:10DD100094F8050100280CBF30462846BDE8704045
:10DD2000FCF73ABD0F48FCF737FDCBE770BD00BFED
:10DD300054C40A08106E0024240500246EC40A0886
:10DD4000B83400247DC40A08C2BC0A08EBD20A0811
:10DD5000643300208EC40A084DC40A0844C40A086B
:10DD6000B5C40A0873C40A0838B50B4D0C4605EB58
:10DD7000C00595F9180307F0B9F801460748FEF702
:10DD800059FE95F81E3333B1611C0548C9B2BDE890
:10DD90003840FEF74FBE38BD24DD0908D2C90A0855
:10DDA00070BC0A082DE9F04F80468BB008460D463E
:10DDB0004BF06EFE0246A8B3A5492846FAF748FD87
:10DDC000044678BBFCF79CF8A24DA348A34EFCF791
:10DDD000E3FCA34F1420DFF8CC8240F013FFE110E6
:10DDE000304604F007020131FEF724FE95F81D903D
:10DDF00095F91C00B9F1000F0DD007F077F84A46ED
:10DE000001464046FCF794F801342435102CE6D145
:10DE10000BB0BDE8F08F07F069F801463846FCF713
:10DE200087F8F1E7284605AA8E494DF08AFE054697
:10DE300020B901464120FCF7CEFCE9E78A49F9F711
:10DE4000BBFB20B989494046FAF794FBE0E7884ECE
:10DE50000B27002431682846F9F7AEFB002808BFDD
:10DE60003446013F06F11006F4D154B981492846E1
:10DE7000F9F7A2FB28B12A467F494046FAF77AFB18
:10DE8000C6E7002005AA77498DF813004DF059FE2A
:10DE90000646002C4DD0002849D0FAF79FFD031EFE
:10DEA00042DB2279062A3AD10121E26801FA03F025
:10DEB000104239D0DBB2714840FA03F2D20733D5B1
:10DEC0009940013908404EF00FF80546E0880027D8
:10DED0003CF022FA6A4903970978D0E90223002925
:10DEE00018BF1A46217A637A05FB0133D11812F95B
:10DEF0000390029105AA5B4900204DF022FE834663
:10DF000000283FD101235F499CB3029A204692F931
:10DF10000020CDE900312946F9F7DCFE78E75D1EE7
:10DF200013B1A37A9D42D1DB32465749A5E7574E3C
:10DF3000FAE768B10DF11301FAF78CFD28B19DF8ED
:10DF400013502846F5F7B6FF20B93246504994E7FA
:10DF50004E4EFAE72846F4F71DF98146284608F0A8
:10DF600031F903902846254608F064F902940746E3
:10DF7000C0E7CDE900314A4639469DF81300F9F76C
:10DF8000EDFE45E73849F9F717FB064600282FD183
:10DF9000ACB1EDB23F4F72B229462079F4F7CEF81A
:10DFA00000283FF435AF0288314603783846013601
:10DFB0000093C2F30323120BFBF7BAFFEBE73868B9
:10DFC0007979344C72B2F4F701F900283FF420AFAC
:10DFD000028831460378013620460093C2F30323BA
:10DFE000120BFBF7A5FF102E38687979EAD10FE7FD
:10DFF00029495846F9F7E0FA002876D05846FAF74A
:10E00000EDFC824642B29CB1E9B22079F4F796F871
:10E0100000284DD1266829462046F9F70BFD3246E7
:10E0200003461E49CDF800B04046FAF7A3FAEFE6E2
:10E030005FFA8AF6386879790F2E35D99DF8133052
:10E0400017491A09CDF800B003F00F034032EBE78F
:10E05000D5C40A083C010024DAC40A08F0C40A083E
:10E060008FC10A0825B60A08DEC20A0801C50A08D7
:10E070003405002431C80A0815C50A08FEF103005A
:10E08000185D0024099F040824C50A08E6BD0A0893
:10E0900034C50A0846C50A08F7BE0A0867C50A0853
:10E0A0008AC50A085FC60A08F4F790F80028C5D0A8
:10E0B00006AE50463146FAF749FB08A94846FAF73A
:10E0C00045FBCA4520D04FFA8AF38CB1029A294603
:10E0D000204613702768F9F7ADFC08AB02463946B5
:10E0E00014480096FBF724FF92E64FF0FF3ADFE773
:10E0F000039A1148937008AB9DF8132000961109FC
:10E1000002F00F024031EDE75CB126682946204657
:10E11000F9F790FC08AB024631460848FBF708FFC8
:10E1200076E69DF8132008AB0548110902F00F02AE
:10E130004031F3E7B2C50A08D5C50A08FDC50A088B
:10E1400018C60A082DE9F04F07468DB008460D465F
:10E150004BF09EFC044630B9014601200DB0BDE8ED
:10E16000F04FFCF723BD0246A5492846FAF770FB9D
:10E1700030B9A44938460DB0BDE8F04FFAF7FAB906
:10E180002246A1492846FAF763FB002854D1FBF741
:10E19000B7FEDFF8B8A29D480E27DFF8B4B2FCF74F
:10E1A000FBFA172040F02EFD1AF9018BB8F1000F91
:10E1B00036D00025414658462E46FEF73BFCB100BE
:10E1C0004046013689B208F06BF8814608F0F0F855
:10E1D00090F900300446CBB10DB9FBF791FE99F8E8
:10E1E0000630657803F0020394F90000884A894CF0
:10E1F000002B18BF1446B5B106F078FE2246034640
:10E20000314685480095FBF793FE0125042ED6D1B3
:10E2100015B98248FCF7C0FA013F17F0FF07C3D1D8
:10E220000DB0BDE8F08F06F061FE22460346314690
:10E230007B48FBF77DFEE8E7002407AA75492846DE
:10E240008DF81B404DF07DFC18B93846FAF7A8F957
:10E25000E6E70DF11B01FAF7FDFB81460028F4D03B
:10E260009DF81B502846F5F725FE20B96D49384624
:10E27000FAF780F9D4E72346DFF8D8814FF0FF346E
:10E2800003EB430218F8022095420BD0002C02DA6F
:10E29000002A08BF1C460133152BF1D1002C16DAD9
:10E2A0006149E4E71C4607AA5A4900204DF049FCA1
:10E2B0000646002800F097805149F9F77DF938BBF0
:10E2C00004465A4FDFF84881DFF88C9117E04FF091
:10E2D0000009E8E73068F4F7F1FCB1797379024698
:10E2E00011F0020F96F807A04FEA930348460CBFBF
:10E2F00039464146013300915146FBF719FE01347E
:10E300002846214607F072FF06460028E2D187E73B
:10E310004FEA151A0222464930460AF1400A05F032
:10E320000F0BFAF795FA002845D10390B01CFAF7C5
:10E3300055FB039902460491013128460592039149
:10E3400007F054FF059ADDE9031338B95B465246DE
:10E35000384900963846FAF70DF961E7C0799042DE
:10E36000E9D11F466300B9F1000F31D01A194244B8
:10E370005678013E7A1C23440AAC284614BF29462D
:10E38000002108EB030208F803107B1C3946537088
:10E39000FF2393702246FAF7E9F908AA3146284686
:10E3A000FAF7E4F9B74216D108AB5A46514622486B
:10E3B000FBF7BEFD34E721493046F9F7FDF820B1FF
:10E3C0005B4652461E490096C4E74FF0FF37C9E747
:10E3D0004FF0FF36CEE708AB5A4651461948009435
:10E3E000FBF7A6FD1CE704EB4404174B0246284646
:10E3F000A0440093012398F80110F9F7F7FC0FE708
:10E40000DEC20A0801C50A08D5C40A0834C60A08CB
:10E41000C3BC0A0825B60A0854C60A0875C60A0805
:10E4200066C60A087BC60A0892C60A08E6BD0A083C
:10E43000BBC60A08BEC60A0810C70A08F7BE0A0803
:10E44000EAC60A082EC70A08099F0408D8420A0823
:10E450004DC60A084C250024A6C60A082DE9F04F2F
:10E4600089B0074608469C4905AA4DF06AFB054657
:10E4700030B901464120FEF71DFA09B0BDE8F08F22
:10E480009649F9F799F8044600283BD19448954DF0
:10E49000FCF782F9944E1420DFF88C8240F0B2FB36
:10E4A00095F9060006F022FD2968AA88034601F1C5
:10E4B00027413046B2FA82F201F57E01C2F11F0215
:10E4C000890A4131FEF7B6FAE97911B14046FEF703
:10E4D000B1FA0134FBF714FD0835902CE0D17E49E8
:10E4E00005AA00204DF02DFB8049F9F765F80028BA
:10E4F000C3D138467949FFF725FE78493846FFF7FA
:10E5000051FCBAE70024DFF8F89119F9340006F05D
:10E51000EDFC804601462846F9F74EF840B101343B
:10E52000242CF2D12A4672493846FAF723F8A4E798
:10E5300005AA69494DF005FB064690B3FAF74EFA75
:10E5400005466C4B4FEAC40A03EBC40393F81E3331
:10E550004BBB002D29DC09EB0A03588893F8049083
:10E5600093F805A03BF0D8FEEBB2D0F808B003FB5F
:10E5700009AA0093002E00F09A803378002B00F057
:10E58000968006A93046FAF765FA002800F08C80DC
:10E590009DF818500DBB58480BF80A50FCF7FCF8D2
:10E5A0006BE70546CDE7002D05DD012B1A4638BF88
:10E5B0000122954209DD012B4FF001024F493846F7
:10E5C00038BF0123F9F7F4FF57E705AA42490020B5
:10E5D000013D4DF0B6FA0646BDE72846F5F76AFC60
:10E5E000814600285CD02B09454F4FF000080BF8FE
:10E5F0000A504033029305F00F030393BB790026C2
:10E60000012B38BF0123019397F804B097F805A0B8
:10E6100078883BF081FE06FB0BA38268D15CA9429F
:10E6200022D1444504D10099B1421DD00021D154DA
:10E630005FFA86FB33485FFA88FADDE90212FEF7DB
:10E64000F9F959465046FFF78FFB444509D12E484A
:10E65000FEF7F0F950465946FFF786FB2B48FEF7C8
:10E66000E9F92B48FCF798F80136019BB342CBDC63
:10E6700008F101080837B8F1240FBFD1D9F800100C
:10E68000B9F8042001F127412248B2FA82F201F5DB
:10E690007E01C2F11F02890A4131FBF749FCECE619
:10E6A0003846F9F77DFFE8E632461B493CE71BF8A0
:10E6B0000A30013573B11A09184903F00F0306A88F
:10E6C0004032F9F7CDFF06AB2A4641461448FBF726
:10E6D0002FFCD2E6134BF7E725B60A08D5C40A0883
:10E6E00054C70A08601B002492C70A089DC70A087D
:10E6F000A1C70A0824DD0908BDC70A0807B90A0826
:10E700003CE00908CFC70A08E2BE0A08F3C70A08B6
:10E7100016CD0A08FDC70A0819C80A0814BC0A0859
:10E7200035C80A0865B20A0870BC0A086B4B1B782A
:10E730002DE9F04F87B0002B00F0CA80684D4FF0F4
:10E7400000086848A968FBF7F3FB69686648FBF7AF
:10E75000EFFB664B6648D3E90031C91A654B1A686E
:10E76000B1FBF2F2FBF7E4FBFBF7CAFB6248FCF7F4
:10E7700013F86248FCF710F8614B5FFA88F41B78D5
:10E78000A34221D85F4D00245F4EFBF7B9FB013453
:10E7900055F8041F3046FEF74DF9162CF7D15B4DA6
:10E7A0000124594EFBF7ACFB2B4669680134304617
:10E7B0001B680435C91AFEF73DF9162CF4D107B0D1
:10E7C000BDE8F04FFBF79CBB514B14264FF03C0BC0
:10E7D000671C03EB840306FB045693ED450A4CF0DB
:10E7E0009DFC96F81EA081B2B6F80E901AF0010FAB
:10E7F00080B20CBF2D2252221AF0020F049045481D
:10E800000CBF2D2354231AF0040FB1FBFBF10CBFF6
:10E810004FF02D0C4FF0560C1AF0080F05914FF0E9
:10E8200064010CBF4FF02D0E4FF0430E1AF0800F15
:10E8300001FB09F10CBF4FF02D0A4FF0530ACDE94F
:10E8400000CECDE902A13946FEF7F4F8B37FDB072D
:10E850003AD55C23304A6343D118D05891ED010A70
:10E8600070B1B8EE400ADFED2D7A20EE270A07EEF0
:10E87000900AF8EE677A80EE270A4CF04FFC00B25F
:10E88000642290FBF2F102FB11022548FEF7D2F858
:10E890001421244808F1010801FB075701FB045427
:10E8A000F988628A0491218B02F003039208039194
:10E8B000E18A0291A18B0191A18A009119214B4318
:10E8C000218AFBF735FB57E71748FBF711FBDFE71A
:10E8D000164807B0BDE8F04FFBF75EBF040000200C
:10E8E000101B002049C80A0859C80A083C1C00200F
:10E8F00070C80A085C1B00249DC80A08F9C80A08E9
:10E90000481C0020B81B0020A9C90A08BC1B002015
:10E910006433002055C90A083018002000401C4606
:10E9200072C90A0887C90A087EC90A08ADC90A0857
:10E930002DE9F84F002607460C461D4DB046DFF87E
:10E940007890DFF878A02046F9F74CF8D5F800B0B9
:10E9500048B921465846F9F79FFF20B92146686813
:10E96000F9F79AFF80B15846FBF7C2FA696811B10E
:10E970005046FEF75FF8A96811B14846FEF75AF80D
:10E980004FF00108FBF7BCFA01361035382EDAD10A
:10E990002046F9F727F848B9B8F1000F06D122460A
:10E9A00038460449BDE8F84FF9F7E4BDBDE8F88FF3
:10E9B00064E40908D5C90A08CFC90A08C9C90A0800
:10E9C0000EB403B503AA52F8041B0192F9F7A5FD92
:10E9D000064BD3F880291AB90549986CF9F7D2F893
:10E9E00002B05DF804EB03B0704700BF185D00246F
:10E9F000E4BD0A082DE9F04798460B7981460F4699
:10EA000003F0E0051646402D32D10024634DDFF8B7
:10EA1000A881DFF8B09116E03B7903F00703013BD2
:10EA2000042B04D8DFE803F014171A1D2100315D10
:10EA30005A48FDF7FFFF7B79013BA34202DD4846C0
:10EA4000FBF756FA01347B79A342E5DCBDE8F08799
:10EA500031572846EDE736F81410FAE736F9141066
:10EA6000F7E756F824104046E3E756F82410F0E79D
:10EA700003F00703052B57D8DFE803F0031F27290E
:10EA80002C3E3478602D55D02CD8002D75D1B7F898
:10EA90000550B7F8076021464048FDF7CBFFAC4270
:10EAA00039DBB44237DCB8F1000FCFD0324629460B
:10EAB0003B48BDE8F047FDF7BDBF96F90040602D2B
:10EAC00038D00FD8002D58D151E03488DAE7B6F9A4
:10EAD0000040F4E7D6F800A0202D54464DD034D99C
:10EAE000602D27D0802DB1D132782E4B2E48002AB0
:10EAF00014BF3146194635E0202D34683DD0EFD89B
:10EB000021462648FDF796FFD7F80510A14202DB03
:10EB10004B42A34221DDFBF7F3F923463A6848460E
:10EB20002249BDE8F0474BE7202D25D01ED9602DA6
:10EB3000D8D100247B7944FA03F3DB07BDE8F04722
:10EB40004CBF1B481B48FDF775BF51461A48FDF7DF
:10EB500071FFD7F805108A45DDD8B8F1000F3FF4F2
:10EB600075AF1648BDE8F047FDF764BF0024B7F95C
:10EB70000550B7F907608EE700247A79104B03EB54
:10EB8000C20393F83C24A242C5DDD3F8383453F8CD
:10EB90002400BDE8F047FBF7ABB900BF71BC0A0821
:10EBA00030B20A08EFCD0A08D2C90A08EFC90A082C
:10EBB000C2BC0A08EBD20A085ABC0A08E9C90A080A
:10EBC00024DD0908DAC00A082DE9F04F164685B0A1
:10EBD000334C1A464FF00009A246CDE9010100214D
:10EBE0003046FBF7EBFD06F0100300900393FBF7B4
:10EBF00063F92379029A03F01803934203D0002AA1
:10EC000044D1182B42D14FF00D0B0BFB09A3B3F8E5
:10EC100009003BF081FB80462046F8F7ADFE074631
:10EC2000D8E90221024401442046F8F73DFE80F075
:10EC300001010546009AC9B23046FBF7BFFD039BB0
:10EC4000009003B115BB0BFB09FBB3065AF80BB0E0
:10EC50000ED56DB959461348FDF7ECFED8F80820DB
:10EC60002B4621463A440198FFF7C4FEFBF748F9CA
:10EC700059460D48FDF7DEFED8F80C20002321464A
:10EC80003A440198FFF7B6FEFBF73AF909F101099A
:10EC90000D34B9F5187FAAD105B0BDE8F08F00BFDB
:10ECA000BCED090809CA0A080ACA0A080329F0B50E
:10ECB000054685B00C46164614D80B4F3970FBF745
:10ECC0001FF90A492846FBF707FD2246084901A813
:10ECD000F9F7C6FC01AB324608212846FFF774FF5E
:10ECE000FF233B7005B0F0BD24050024E6BD0A08F3
:10ECF000F7B50A080329F0B5054685B00C46164657
:10ED000014D80B4F7970FBF7FBF80A492846FBF73C
:10ED100013FD224608496846F9F7A2FC6B463246C5
:10ED200010212846FFF750FFFF237B7005B0F0BD90
:10ED300024050024E6BD0A08F3B50A0870B5164696
:10ED400005460C460846F8F72DFF33460246214695
:10ED50002846BDE870404DE6444B2DE9F74FDFF8FB
:10ED6000289105461A785B78009189F80130404B6C
:10ED700089F800201B780BB903F056F800263D4CAB
:10ED80003BF004FBB0460D233A4A0099734352F816
:10ED900003A05046F9F780FD002841D0B8F1000FDC
:10EDA00001DDFBF7ADF851463348FDF743FE002285
:10EDB00021462846FFF7C2FFFBF7A2F8237903F0AC
:10EDC0001803082B44D0102B47D02046FDF73FFEF8
:10EDD0000D22284B02FB0633B3F809003BF09CFAE6
:10EDE0008346D8B12046F8F7C7FD0746DBE9022184
:10EDF000024401442046F8F757FD78B95146019086
:10EE00001E48FDF717FEDBF80810019A2846134646
:10EE1000CA192146FFF7EEFDFBF772F808F1010869
:10EE200001360D34B6F5187FADD10020F8F783FD1B
:10EE3000FF2389F8003089F80130B8F1000F11D1B3
:10EE4000009A28460E4903B0BDE8F04FF9F792BB8F
:10EE50000C492846FBF740FCB7E70A492846FBF770
:10EE60006BFCB2E703B0BDE8F08F00BF983400241C
:10EE7000185D0024BCED09080ECA0A0814CA0A0865
:10EE8000ADB40A08E6BD0A08240500242DE9F74FB1
:10EE9000804608460F464AF0FBFD044620B1012893
:10EEA00023D13B782A2B20D1A64E00254FF00D0A06
:10EEB000A54FB14604F00104A448FBF76DFC0AFB22
:10EEC00005F33846013559F80310FDF7B3FD314617
:10EED00022464046FFF732FF0D36FBF711F8B5F535
:10EEE000187FECD103B0BDE8F08F3D2138464CF0DF
:10EEF00062FE002800F0208103469A4613F8012D97
:10EF0000202AFAD0AAEB070A0130054610F8013B87
:10EF1000202BFAD05FFA8AFA4FF000094FF00D0B60
:10EF20000BFB09F3874A3846D158D4185246019151
:10EF3000F9F78EFC064680BB019908464AF0A8FD09
:10EF400082452AD1277907F0E001402900F0898025
:10EF500014D879B366797E4B002703EBC606BA4610
:10EF6000BB4696F83C340193019BBB4202D9BAF1EF
:10EF7000000F64D0BBF1000F05D02CE06029EAD06F
:10EF8000802900F0A18040467249F9F7F3FA204643
:10EF900003B0BDE8F04FFDF75ABD09F10109B9F51D
:10EFA000187FBDD13A466C49404603B0BDE8F04FEA
:10EFB000F9F7E0BA07F00703042B1CD10B460A222D
:10EFC0002846F9F781FCD4F8053001468342DAD3AC
:10EFD0002046F8F7FBFD0D23604803FB09F9594B68
:10EFE00053F80910FDF726FD00222146404603B0E4
:10EFF000BDE8F04FA2E6052B0DD101230A222846D9
:10F00000F9F762FCD4F8053001468342BBDB5B4272
:10F010008342B8DCDCE72846F9F7E0FC17F0050F7F
:10F02000014607D1B4F80520B4F807309142AADBB5
:10F030009942EEE7B4F90520B4F90730F6E7D6F8BF
:10F04000382452F8270050B12946F8F7B5FA30B9FC
:10F050004FF0010A39462046D346F8F7B7FD01378D
:10F0600082E707F0070794F805B0013FB345B2DD2A
:10F07000AA4615F8013B202BFAD02046F8F792FD5E
:10F080000546042F04D8DFE807F0030E0E141D0018
:10F090005046F9F7A3FCA8552C2150464CF08BFDA7
:10F0A0000136451CE2E75046F9F798FC25F81600B2
:10F0B000F2E700230A2200215046F9F705FC45F843
:10F0C0002600E9E70123F5E728464AF0E1FCE37969
:10F0D000064694F805A0DB07A7790AD52046F8F77D
:10F0E00061FD0378014623B1324628464CF03CFED0
:10F0F000E0B9DEB1B74219D32046F8F753FD3A46DE
:10F1000000214CF041FDB2453FF665AF324614494F
:10F1100028464CF029FE00283FF45DAF2046F8F762
:10F1200041FD324629464CF0D1FC54E73A460D49A0
:10F130004046F9F71FFA26E73946404603B0BDE8D6
:10F14000F04F09E6BCED09080ECA0A0824CA0A08ED
:10F1500024DD090872CA0A08ADB40A0867CA0A0899
:10F16000EFCD0A0837CA0A0870B504460E460846AD
:10F170004AF08EFC3146054602462046F9F768FB08
:10F1800068B9635D1846F9F747FB00B933B9013533
:10F190002C44204601340378202BFAD070BD002087
:10F1A000FCE72DE9F04F0E4693B082469E4930466B
:10F1B0001746FFF7D9FF0546002840F01F819B49FD
:10F1C0003046FFF7D1FF0546002840F019819849E5
:10F1D0003046FFF7C9FF0546002840F013819549E6
:10F1E0003046FFF7C1FF0546002840F00D819249E7
:10F1F0003046FFF7B9FF002805460ABF012408245E
:10F2000035467F428D49284607F010073C43FFF7FB
:10F21000ABFF002800F0FA8044F02004884B1B78F4
:10F220000BB902F001FE3BF0B1F814F0090F00F049
:10F2300029838448FBF7B7FA0020FEF7EFFC14F4AB
:10F240008073059340F0EC807F48FBF7ACFA7F4871
:10F25000FBF7A2FA04F01803182B05D17C48FBF742
:10F26000A2FA7C48FBF798FA01230493FAF748FEC8
:10F2700079497A48FAF75CFE79497A48FAF758FEF4
:10F2800004F48473082B07D177495046FAF774FFCA
:10F2900075495046FBF7DAFB14F0800307930ED153
:10F2A000724B204693F8982303F56673002A704A40
:10F2B00006BF0121134600216E4AFAF725FE6E496A
:10F2C0002046FDF7F7FA6D492046FBF76FFC6C49C5
:10F2D0002046FBF780FA6B4B1D686B4B1E6814F0E1
:10F2E0001003039340F09E806848FBF75CFA039B91
:10F2F00002934FF00008664B9946069365EA0603B1
:10F30000099359F804BBBBF1000F21D00127099BD9
:10F31000029A204607FA08F73B400CBF0121002162
:10F320000893FBF74BFA66EA05035A4A0290204617
:10F330003B425B4614BF01210021FBF707FE089901
:10F340005B46544A0039204618BF0121FAF7DCFD1C
:10F3500008F10108B8F11D0FD3D166EA05034FF09B
:10F360000008DFF84C910893069B53F804BB069302
:10F37000BBF1000F23D0012707FA08F73E420AD05D
:10F3800065EA06034A4620463B425B4614BF01211C
:10F390000021FBF7DBFD3D4211D0089B2046029A7D
:10F3A0001F400CBF01210021FBF708FA391E029013
:10F3B0005B464A4618BF01212046FAF7A5FD08F131
:10F3C0000108B8F11D0FCFD1334B2046334A3449E1
:10F3D000FBF716FF079B002B6CD0134B224618211E
:10F3E0005046FFF7F1FB049B002B00F0AE812D4847
:10F3F000FBF7D9F92C48FBF7CFF9A6E1012400E788
:10F400000224FEE60424FCE68124FAE62749284685
:10F41000FFF7AAFE00283FF401AF44F48074FDE634
:10F42000002322E7194B63E793CA0A089ACA0A081D
:10F43000A2CA0A08A8CA0A089DC70A0874CC0A0802
:10F44000185D0024B6CA0A08BECA0A08D6CA0A0845
:10F45000E2CA0A080ACB0A0827B60A086AB60A08E6
:10F4600078B60A088DB60A08E6BD0A08106E0024B0
:10F47000EFCD0A081ACB0A0827CB0A0831CB0A08B5
:10F4800008C10A08F83C0024F83A002480CA0A0897
:10F49000E0DD090837CB0A084ECB0A087862002461
:10F4A000107200240BCC0A0821CC0A08B1CA0A0841
:10F4B00043CB0A08DFF8A8832046DFF8A89398F822
:10F4C000002099F80030B34D9A42B34A13BF01218E
:10F4D000002101270027FBF771F999F80030064653
:10F4E000AE4A05EB830339462046D3F8A432FBF736
:10F4F0002DFD98F800303946A84A05EB83052046D3
:10F50000D5F8A432A64DFAF7FFFCA64A2046D5ED61
:10F51000007AF5EE407AF1EE10FA0CBF01210021DD
:10F52000FAF7F2FC33462A469F4920469F4EFCF7E5
:10F53000E7F89F4D9F4B20469F4A01930092326807
:10F540002968FDF761F99D4B40F2022220460193A4
:10F550000092B268A968FDF757F9039B002B40F0B1
:10F56000FA809748FBF71FF9039A964E01259648B3
:10F570000021964F16F8013B10F801EB03F1480CFF
:10F58000EC440CF820EC17F801CB0CF14808E844E7
:10F5900008F810EC002D00F0E080A3EB0C056B42A6
:10F5A0006B4101311D460829E4D1002683F0010199
:10F5B00020468DF83060FBF701F90EAB844A2946EE
:10F5C00020468DF84060FBF7C1FC0AAB804A294613
:10F5D0002046FAF799FC7F4B7F4A20467F49FCF78B
:10F5E000B9FA7F4B7F4A20467F49FCF73FFB7F4BB0
:10F5F000794A20467949FCF7CBFB7D4B7D4A204672
:10F600007D49FBF7BBFC7D4B7D4A20467D49FBF7DE
:10F6100043FF7D4B7D4A20467D49FCF7DBF97D4B5E
:10F620007D4A20467D49FCF7A3FD7D4B7D4A20465F
:10F630007D49FCF793FC039B002B40F090807B48B6
:10F64000FBF7B1F8DDF80CB0794E0025794FDFF803
:10F6500018823946022230464CF0EAFB0028337803
:10F660005A4614BF0121002120460CBF4FF001096A
:10F670004FF000090293FBF7A1F8029B8346022B8F
:10F6800070D17B78192240F2EE21204612FB031341
:10F69000694A494601933B7818F8033000932B469A
:10F6A000FBF754FC7378192240F2EE21204612FB3E
:10F6B0000313614A49460193337818F803300093E5
:10F6C0002B46FAF721FC013502360237122DC0D144
:10F6D00000215A4B22465046FFF776FA210740F1A7
:10F6E000C5800025E9B2013522465046FFF7DEFA13
:10F6F000042DF7D1524F534D3B782B70059B33B9F6
:10F700005148FBF750F851495046FAF7E5FFFF23FF
:10F7100000262B70F1B2013622465046FFF7EAFA76
:10F72000042EF7D17B786B70059B83BB4848FBF7B1
:10F730003AF846495046FAF7FFFF4648FBF733F8D8
:10F740004548FAF7D5FBFF236B70002013B0BDE8E6
:10F75000F04FF8F7F0B81A4A07E72B4621E7DFF831
:10F76000CCB071E73B7849463C4A204618F8033054
:10F7700000932B46FBF7EAFB3378384A494618F8E2
:10F780000330204600932B46FAF7BEFB9BE7FF238E
:10F790006B7028E624DD090855CB0A085BCB0A0804
:10F7A0008035002464CB0A08003B00248036002406
:10F7B000143D002473CB0A08FFFF7F007ACB0A08B0
:10F7C00088CA0A08A03B0024885D0A08B8340024CF
:10F7D000D8B40A0885B40A08446800248C7200244E
:10F7E00086CB0A08446900248C73002481CB0A0864
:10F7F0008CCB0A08A8630024FC73002490CB0A0871
:10F80000086700247474002499CB0A083468002423
:10F81000A0750024A1CB0A0844640024B07500241C
:10F82000AACB0A08E0360024043C00248CCA0A084B
:10F83000CC7600249C660024D6B30A0893CA0A0832
:10F84000F03B002424050024AECB0A08E6BD0A08DC
:10F85000D1CB0A08F8CB0A0815CB0A08E6B30A0888
:10F86000003D002478350024985F0A080F4D224699
:10F8700050462978FFF71AFA224669785046FFF772
:10F8800039FAB0E5A20706D5084B2246504619784A
:10F89000FFF70CFA59E763077FF557AF034B224692
:10F8A00050465978FFF726FA4FE700BFF03B002497
:10F8B000002276E4012274E408B504460848FAF709
:10F8C00017FBFAF7F9FA074B186D0BF0A3F805F0E0
:10F8D000ABFA012C01D142F095FAF4F765FD00BFB7
:10F8E000B5B70A08185D002410B5044608460B4653
:10F8F000F8F778F828B9032208491846F8F7A8FF5E
:10F9000028B90748FAF74FFF0120FFF7D5FF204637
:10F910000449BDE81040F8F72DBE00BF2BCC0A0803
:10F920002FCC0A08DFB80A082DE9F74F4FF0000B7B
:10F93000064601AA08462D495D464CF002F901270A
:10F940000446DFF8B880DFF8B890DFF8A0A014BB59
:10F95000BBF1000F27D1264C002D43D02946254866
:10F96000FAF7E6FA23780BB902F05EFA3AF00EFDE8
:10F97000002384F84D30FAF775FA15B12846F7F7E9
:10F98000DAFF9FB13046F8F731FE78B1FAF7C2F8E6
:10F990000020FFF791FFBBF1000F0AD02046F9F7D6
:10F9A0001DF885B2C5B93046F8F7FAFD03B0BDE8D9
:10F9B000F08F41462046F8F76FFF80B94946204650
:10F9C000F8F76AFF0028EED05F4601AA51460020F2
:10F9D0004CF0B7F80446BAE74FF0000BF5E74FF0EC
:10F9E000010BF2E70448FAF7DEFEBFE725B60A0886
:10F9F000185D00245ACC0A087DCC0A0851CC0A08AC
:10FA000013CB0A0810B50C46F8F7F0FD78B1084B97
:10FA100001229A73FAF77EF80648FAF7C4FE0649FF
:10FA20002046F7F7C9FD10B10020FFF745FF10BDD4
:10FA30009834002493CC0A0804B70A08224BB0F586
:10FA4000FA6F1A680346A8BF4FF4FA63B3F57A7FDA
:10FA5000B8BF4FF47A73D20416D540F2DC5290420C
:10FA600015D040F2DB5207EE903A9042F8EE677AFA
:10FA70001FD8DFED166A9FED167A77EEE67A9FEDD6
:10FA8000150AA7EE870A7047B0F57A7F02D89FED76
:10FA9000120A704707EE903ADFED106A9FED107A78
:10FAA000F8EE677A9FED0F0A77EEE67AA7EE870AFF
:10FAB0007047DFED0D6A9FED0D7A77EEE67A9FEDE8
:10FAC0000C0AA7EE870A7047B434002400007A4479
:10FAD000D62000C000E082440000000000407A44CC
:10FAE000661000400000404200A0BB44D620004009
:10FAF000000083444FF4EB720023084910B4084C13
:10FB0000C280084AC0F8024003705DF8044B0381CC
:10FB1000C0F80A10C0F80E2043827047C2010E01DF
:10FB20004A01B40096004400704700BF704700BF10
:10FB30000020704701207047704700BF704700BF2A
:10FB4000704700BF704700BF9FED010A704700BFBC
:10FB50000000000000207047064B1B78834206D946
:10FB600000EB4000044B03EBC003586970470020D2
:10FB7000704700BF000600203C05002000EB40005D
:10FB8000024B03EBC003587C704700BF3C050020CC
:10FB9000024B1878003818BF01207047000600207B
:10FBA00003681B6903B11847704700BF70B5094C63
:10FBB000236873B10546002606E099681A681E732B
:10FBC00021609047236823B15A681846AA1A002A70
:10FBD000F3DA70BD5C7D00240B4B1A79D20700D597
:10FBE00070479A68002AFBD04FF47A7101FB02F249
:10FBF0009042F5D3054A12781AB9054A91681269FC
:10FC00000A6000229A6070475C7D0024443600241C
:10FC100058360024F8B5354C2368002B53D00A28F9
:10FC200001D00D284DD1324D2B7B0BB1FAF768F97D
:10FC3000304E232130464BF0BEFF08B1801B2060C0
:10FC4000236800226BB902B12360FAF725F92B7BF8
:10FC5000EBB12948BDE8F840FAF74AB901220B4652
:10FC6000F0E7591E705C2028F8D08AB90022234C96
:10FC7000204FF2543926013E0CD13146204B9C4294
:10FC800011D2E368206898476B7B002BDDD1F8BD6B
:10FC90002360EBE721683846FFF766FA0146002843
:10FCA000ECD11034E7E72B7B23B116491648FEF759
:10FCB00087FECAE71548FAF71BF90E48FAF76CFDFC
:10FCC000C3E7FF2BE3D8A0F120025E2ADFD80BB9EF
:10FCD0002028DCD05A1C2260064AD054044B1B7BDF
:10FCE000002BD4D0BDE8F840FBF726B99466002479
:10FCF0005C7D00249265002422B60A0864E40908A9
:10FD0000E4E70908C8CC0A08E4CC0A08EACC0A08E7
:10FD100008B5294B1B68DB041ED5B5EE400AF1EE91
:10FD200010FA26D0DFED257AB4EEE70AF1EE10FAEC
:10FD30001FD49FED237AB4EEC70AF1EE10FA2AD849
:10FD400070EE677A9FED1F7A9FED1F0AA7EE870A74
:10FD50004BF0E4F980B208BDDFED187AB4EEE70AA3
:10FD6000F1EE10FA0BDA9FED190A4BF0D7F980B2D9
:10FD700008BD9FED170A4BF0D1F980B208BD70EEB7
:10FD8000677A9FED147A9FED140AA7EE870A4BF06D
:10FD9000C5F980B208BDDFED117ADFED116A70EEB2
:10FDA000677A9FED107AA7EEA67AB0EE470A4BF07D
:10FDB000B5F980B208BD00BFB43400240000404251
:10FDC00000E0824466BEFFBE0060BB4400007A448F
:10FDD0000080BB4438DFFF3E00407A44000083448B
:10FDE00066BEFF3E00A0BB44F8B5CA4B1B6813F0CB
:10FDF00004052DED048B40F0D6809FEDC78AC74CDB
:10FE000013F0200304D094F8DC3013F0020343D144
:10FE10002279DFEDC38A12F0010294F81C114FD150
:10FE2000A9BBD4ED487A9FEDBF6ADFEDBF6A67EEEC
:10FE3000867A94ED4A7A38EE477AE8EE267A84EDAF
:10FE4000497AC4ED487A63B1012194F83021D4F89D
:10FE5000E0308A4284F81D11C4F82C3118BFC4F870
:10FE60002431B24B1E780D2E0BD1D4ED387A9FED94
:10FE7000B07AB04B67EE877AFDEEE77A17EE902AFC
:10FE80009A80B0EE489A00259FEDA37A36E084F878
:10FE90001D2184F81C21C4E7D4ED3B7AB4F8F0307E
:10FEA000F8EEE77AC4ED387A002B40F0EE80DFED13
:10FEB0009C8A2279012394F81C1112F00102AFD020
:10FEC000002900F0CB80D4ED4A9A984A38EE699A1E
:10FED00094F81D711678002B6AD0012F02D0002DE6
:10FEE00040F0EB80002F40F003810D2E00F00581E3
:10FEF000002D40F0BB8094ED4E7A0125D4ED507A70
:10FF0000D4ED516A37EE677A94ED4F8AE6EE877A40
:10FF100037EEC87AC4ED507AA6EE878A84ED4F8A10
:10FF200084ED4E8A0DB184ED498AD4ED547A94ED76
:10FF3000527AB0EE676ADFED805A38EE477AD4ED38
:10FF4000556A94ED530A84ED528A97EE256AE6EEDF
:10FF5000867A37EEC07AC4ED547AA6EE870A84ED2D
:10FF6000530A84ED560A4BF0D9F802B282EAE273E2
:10FF7000A3EBE2739BB2092B6ED9002AACBF0A38FF
:10FF80000A3005B20D2EA4F85C5150D0242E41D079
:10FF9000382E05D1B0EE480A4BF0C0F8654B98807A
:10FFA000BDEC048BF8BD5D4C012594ED348A27E748
:10FFB0000D2E77D0DFED588A002F99D094F830318C
:10FFC000002B5CD194ED4E7A002D96D077EE487AD6
:10FFD00094F831319FED596A06EE903A77EEA97A9E
:10FFE000F8EEE66AF0EEE77A67EEA67AF4EEC67A05
:10FFF000F1EE10FA03DD28EE866AC6EE278AF7EEE8
:020000040805ED
:10000000007A77EEE87A67EE897AE8EE877AB0EEE2
:10001000677A73E7DFED4A7A94ED490A20EE270A02
:100020004BF07CF8434BBDEC048B5880F8BDDFED02
:10003000427A9FED430A68EEA77A3E4C29EE000A09
:10004000FDEEE77A17EE903A23804BF067F8E580F3
:100050006080BDEC048BF8BD002593E7D4ED489A91
:100060000122C4ED4A9A84F81C212EE794F830311D
:10007000012B94BFB0EE497A94ED4E7A3EE7022B05
:100080003FF439AF002DF1D135E707EE903ADFEDBF
:100090002A6A9FED2C7AF8EEE77AC6EEA78AC8FEA8
:1000A000C78A06E7DFED267A94ED4E0A20EE270A8E
:1000B0004BF034F81F4B98807CE794ED380A01230D
:1000C00070EE487A84F81D3177EEA97AC4ED4B7A48
:1000D00030EE670A0D2E84ED4E0A7FF46FAFDFED30
:1000E000187A20EE270A4BF019F8124B988065E732
:1000F00094ED380AD4ED4B7AEAE7DFED117A94ED0E
:100100004E0A20EE270A4BF009F80A4B9880002D82
:10011000ACD1F0E6C8690024000000005C7D00243A
:100120009A99993ECDCC4C3FCDCC4C3E9F26002495
:100130000AD7233CA02600240000C84200401C46E9
:10014000CDCCCC3D6666663F70B5254C2378012B3F
:1001500000D070BD234B1B68002BFAD0224D2B68BA
:1001600028465B6898470028F3D0204B204E1A6839
:10017000338892889A421FD31E4900222846096874
:100180004968EA622A6803FB01F1D36898472B6843
:100190009B6813B128469847F8B13388164A013353
:1001A00052683380002AD4D0116893884A69134278
:1001B00018BF1B048B6170BD0F4A00210F4B5268A2
:1001C0001B782170002AC4D0C3F3400391881268C1
:1001D0001B0101FA03F3936170BD41F01BFEDCE7E4
:1001E000BA2F00247C22002480220024B42F002473
:1001F000B82F0024AC2F0024B8220024C4220024ED
:100200002DE9F84FB14C8046B14B2DED028B227990
:1002100094F85E51D2071F885DD5AE4E012D94ED46
:100220005C8A00F09080022D49D0ADB9B4F86431F9
:100230009F42A94B00F2B5801A68F37DD4F874117F
:1002400003EB8303521A03EB8303B2EB830FC0F279
:100250002381012584F85E51F37B33B1B38923B147
:100260009E4B1B78002B40F0908094F85F21AA42AF
:1002700038BF2A46337A632B07D8022D94F86811C9
:1002800000F0DA80002940F0EB80954B9FED957AE5
:100290001A70B17BD4E96030C4F884311B1A07FBB3
:1002A00003F307EE903AF8EEE77AA7EE878A84ED3B
:1002B0005C8A00293BD1BDEC028BBDE8F88FB4F815
:1002C0006231BB42C8D2844B01251B6884F85E5161
:1002D000C4F87431C0E7EA1E012A44D918897D4E5A
:1002E000C0F30B004BF000FE092897DDB6F806902E
:1002F000B94502D83388BB4290D2B7EB490F8DDCA9
:100300000323DFED797A754A84F85E31B0EE678AAF
:1003100084F85F310023C4ED5C7A1370A4F8603177
:10032000A4F86231A4F86431A4F866312BE0012A04
:1003300000F0A080022ABED10720BDEC028BBDE8F0
:10034000F84F0AF05BBCB4F86631BB422ED2B4F869
:100350006031BB4202D2002584F85E515E4B1B68BF
:10036000C4F8743178E75B4EB6F80690B94502D808
:100370003288BA422CD2B7EB490F29DC032D40F06A
:10038000988094ED5C8A032566E712F0C5F8002892
:1003900077D102232A469D4284F85F3138BF1A463E
:1003A00068E71B680025C4F8743155E74A4BD4F858
:1003B00074111A68337E521A03EB830303EB830331
:1003C000B2EB830FFFF648AF022584F85E5143E796
:1003D0001889C0F30B004BF087FD09285EDD002271
:1003E000317D84F85E2184F85F21002900F082804D
:1003F0003A4B1970B388728813FB01F312FB01F2B8
:10040000717C9BB292B28B42A4F86031A4F8622155
:100410005AD95B1A9BB28A42A4F8643152D9521A53
:1004200092B2A4F86621642294ED5C8A84F8692172
:100430000022C4F86C21FBE691B90120C4F86C815C
:1004400084F86801C3F1640301FB03F0274B83FBCD
:100450000013C017A0EBA350643084F8690114E7BF
:10046000D4F86C112248A8EB01018142EADB84F840
:1004700069310AE7BDEC028B0820BDE8F84F0AF0AD
:10048000BDBB337C83420FD301232A469D4284F8AF
:100490005F3138BF1A46EDE60025DDE6032D3FF457
:1004A00070AF94ED5C8AD7E600232A4684F85F316A
:1004B000E0E61889C0F30B004BF016FD09283FF762
:1004C00017AFEEE70022ACE70023A4E75C7D002431
:1004D0008071002448630024541B00249071002480
:1004E00091710024ACC52737000000006BCA5F6B18
:1004F000809698003588B7FBF5F50135082D39DC75
:10050000E9B2204ADFF88890126889F8001092F961
:100510007620AA423FF46EAF002A3FF46BAF1A4A2E
:1005200092F800E00EF1010202F0030296453FF45A
:1005300061AF4FF0FF30DFF85CB04FF0EA0A0AE03D
:10054000002803DABCF1000F08BF1046013202F0A8
:100550000302964511D00AFB02BC9CF976C0AC455B
:10056000EED11046C0B2F9F747F9084B99F80010E0
:100570001F883FE708252946C3E70028FFF63AAF62
:10058000F0E700BF7C3600249834002480710024FA
:1005900090710024A85E00242DE9F843A84C2DEDAD
:1005A000048BA36820469847002800F0BB80B4F96C
:1005B0000E30A17D06EE903AB4F91030092907EE0D
:1005C000103AB4F91230F8EEE66A07EE903AB8EE57
:1005D000C77AF8EEE77AC4ED126A84ED137AC4EDB7
:1005E000147A00F0A380974E04F1480023F0BAFE7D
:1005F000B28DB36A002A40F0A580934A934D1268E9
:10060000520700F1E880B3F90020D4ED147A06EE29
:10061000102AB3F90220B3F9043006EE902AB8EE9E
:10062000C66A07EE103A8A4BF8EEE66A94ED128A33
:10063000B8EEC77A93F8D273864B38EE468AD4ED7B
:10064000138A93F8008037EEC79AB4F8443078EEF6
:10065000E68A84ED128A07EE903A3388C4ED138A55
:10066000F8EEE79A84ED149A002B40F0FF80B8F181
:10067000040F00F0D881D5ED6D7AD5ED6E6A95ED59
:100680006F7A78EEE66A85ED6D8A39EE477AC5EDC8
:100690006E8A38EE678A85ED6F9A66EEA96A27EE54
:1006A000297A28EE298AC4ED166A84ED177A84ED3A
:1006B000158A94ED137AB8F1040FD4ED167A27EE6B
:1006C000077AD4ED124A67EEA77A94ED155AD4ED65
:1006D000145AA4EEA47A94ED176AE5EE057AD4EDE7
:1006E000006AA5EEA57AE6EE067AB1EEC70AB1EE8B
:1006F000E77A26EE800A84ED180A26EE878A84EDD2
:10070000198A0CD1DFED548A544D20EE280A4AF0A4
:1007100005FD28EE280AA8804AF000FD2881012363
:1007200084F86830BDEC048BBDE8F883454E04F1D5
:10073000200104F1480023F0ADFDB28DB36A002A18
:100740003FF45BAFB2F5C87F00F051813F4D4FF0F1
:10075000000E94ED127A4FF0000CD5ED626A012A7A
:10076000D4ED137AF8EEE66A94ED146AC4F848E022
:10077000A3F800C076EE876A95ED637AC4F84CE082
:10078000B8EEC77AA3F802C0FDEEE66AC4F850E0FE
:10079000A3F804C037EE277AD5ED647A16EE907A86
:1007A000C5ED626AF8EEE77ABDEEC77A77EE867A33
:1007B00017EE100A85ED637AFDEEE77A17EE901AD0
:1007C000C5ED647A00F01682013AB2851E4A1268BD
:1007D00052077FF518AFB5F89471322F00F0C18041
:1007E000002F40F0828195F8B221002A3FF40BAF30
:1007F00005F5D270DFF86CC0B4F80CE0002707C82C
:100800008CFB0298D21785F8B271C2EB2812A2EBCA
:100810000E029A808CFB00E2C017C0EB22108CFB0A
:10082000012CC91701221880C1EB2C1159800C4BE7
:10083000DF81C3F80A20F9F7C3F9B36AE3E600BF22
:100840006833002094210020B43400245C7D00240F
:10085000A01D00209F26002400007A44A02600242A
:100860008C6300241F85EB510AD7233C002F00F036
:10087000B380D6ED027AD6ED036A38EE678A96ED3C
:10088000010A95ED6D7AE8EE267A37EEC06AC6ED7C
:10089000027AA6EE260A30EE478A86ED010A84ED3A
:1008A000120A85ED6D0A28EE298A84ED158A002F3B
:1008B0007FD0012F00F07981D6ED057A012F96EDDA
:1008C000067A78EEE78A96ED040A95ED6E8AE8EEF0
:1008D000877A77EEC06AC6ED057AA6EE870A30EE13
:1008E000488A86ED040A84ED130A85ED6E0A28EE27
:1008F000298A84ED168A00F03A81022F00F04A819D
:1009000096ED087A022FD6ED096A79EE477A96EDD0
:10091000070A95ED6F8AA6EEA77A77EE407A86ED04
:10092000087AA6EEA70A30EE488A86ED070A84ED1B
:10093000140A85ED6F0A28EE298A84ED178A7FF460
:10094000B8AEB8F1040F7FF4B4AE4AF0E7FB1FED88
:100950003A0ABB4D28EE000A68804AF0DFFBE880C7
:10096000A7E6B84A0021D4ED126AD26894ED137A52
:10097000FDEEE66AC5F8A0211A68BDEEC77AD4ED8F
:10098000147AC5F898219A88FDEEE77AA164A5F853
:100990009C210022C5ED696A1A8085ED6A7AE164BE
:1009A000C5ED6B7A5A8021659A80013FA5F8947154
:1009B00019E7B8F1040F7FF47FAF4AF0AFFB9FED6A
:1009C000A20ADFF87C9228EE000AA9F802004AF099
:1009D000A5FBA9F806006FE7B8F1040F7FF449AF53
:1009E000B0EE480A4AF09AFB954B188041E7D4EDE7
:1009F000126A002094ED137A0021D4ED147AFDEEF2
:100A0000E66ABDEEC77A914DFDEEE77AA064C5EDCA
:100A1000626A198085ED637AE064C5ED647A598075
:100A200020659980D0E697B3D5ED6D7A012F85EDDD
:100A30006D8A38EE678A28EE298A84ED158A00F0DF
:100A4000BF80D5ED6E7A022FC5ED6E8A78EEE77A1B
:100A500067EEA97AC4ED167A3CD1B0EE490A784E19
:100A60004AF05CFBD5ED6F7A9FED770A00B279EE24
:100A7000677A85ED6F9A3080708067EEA97A27EEED
:100A8000800AC4ED177A4AF049FBF08011E6B0EE17
:100A9000480A6B4E4AF042FBD5ED6D7A9FED6A0A2B
:100AA00000B278EE677A85ED6D8A3080708067EEEF
:100AB000A97A27EE800AC4ED157A4AF02FFBD5ED0E
:100AC0006E7AF08078EEE77AC5ED6E8A67EEA97AE5
:100AD000C4ED167AD5ED6F7A85ED6F9A79EE677A67
:100AE00067EEA97AC4ED177AE3E5D5ED696A0021CE
:100AF00094ED127A0022F8EEE66AD4ED137A94EDC2
:100B0000146A012FA16476EE876A95ED6A7A1A80DD
:100B1000B8EEC77AE164FDEEE66A5A80216537EEE9
:100B2000277AD5ED6B7AC5ED696AF8EEE77A9A8097
:100B3000BDEEC77A77EE867A85ED6A7AFDEEE77AC2
:100B4000C5ED6B7A7FF431AF0B2085F8B02185F8C5
:100B5000B1710AF053F8B36AD5F89821D5F8A0110D
:100B60001A60B5F89C219A80364AD1601DE7B8F129
:100B7000040F7FF4C5AE4AF0D1FA9FED330ADFF8D7
:100B8000C09028EE000AA9F802004AF0C7FAA9F8B6
:100B90000600B5E6B8F1040F7FF4B2AEB0EE490A34
:100BA0004AF0BCFA264B1880AAE6B8F1040F7FF48D
:100BB00083AEB0EE680A4AF0B1FA214B18807BE6AA
:100BC000B0EE680A1E4E4AF0A9FAD5ED6E7A9FED96
:100BD0001E0A00B278EEE77AC5ED6E8A308070802A
:100BE00067EEA97A27EE800AC4ED167A4AF096FAE3
:100BF000F0806FE7DFF858E0C831C837C8304FEAF7
:100C0000E1788EFB0191C8EBE111B4F80C80A1EB07
:100C1000080199808EFB0781FF17C7EBE1178EFB58
:100C2000001EC0171F80C0EBEE105880054BC3F8A4
:100C30000A20A3F80EC0F8F7C3FFB28DB36AC3E56C
:100C4000A02600248C6300240AD7233C5C7D00246A
:100C50001F85EB514B4B1B68190700D470472DE9DA
:100C6000F047494F0546494C2DED108B3978D4F8A3
:100C7000D0315829D4F8C021C4F8C001187800F048
:100C8000F881012800F0A6824149D4F8C831A1F5C5
:100C90008070984797F8008080F00100B8F1580FF5
:100CA000C0B265D0002840F0B682B4F9C43294F8DE
:100CB000901206EE903AB4F9C632092907EE103ABE
:100CC000B4F9C832F8EEE66A07EE903AB8EEC77AA1
:100CD0004FF00103F8EEE77AC4EDB46A84EDB57A1B
:100CE00084F8CC32C4EDB67A45D02A4823F03AFBDA
:100CF00094F8DC92B9F1000F58D1DFF8ACA0264E81
:100D0000B6F90830B8F1570F94EDB49A07EE903A5F
:100D1000B6F90A3094EDB58AF8EEE77A07EE103AA4
:100D2000B6F90C30B8EEC77AD4EDB68A39EE679AC8
:100D300007EE903AF8EEE77A38EE478A84EDB49AF7
:100D400078EEE78A84EDB58AC4EDB68A00F09A8120
:100D5000B8F1580F00F01F82104B01221B688AF86F
:100D60000020002B40F05D82BDEC108BBDE8F087C9
:100D70000B4B588196E70B4901F13C0023F08AFAAE
:100D8000B6E700BFC86900249F2600245C7D0024CC
:100D9000208000242C80002464630024F0050024BB
:100DA000A0260024F07F00249C340020D4F8E032F8
:100DB00094F8DD225B1B002B40F3C081DFF878A3A1
:100DC0009FEDD46ADAED027ADAED016A67EEA77A6E
:100DD0009AED037AE6EEA67AE7EE077AF4EE467A23
:100DE000F1EE10FA40F34081012A00F03D810D2020
:100DF000C94E09F003FF0023B360B381012384F8D7
:100E0000DD32F1F7D1FCC54B97F800800344C4F8FC
:100E1000E032C34B1A6852B1C24B91881B781268FA
:100E2000DB4303F001031B0101FA03F3936194ED2B
:100E3000B50AD4EDB43A60EE006AD4EDB60A94ED8A
:100E4000C28A94EDBA5AE3EEA36AD4EDD27AB0EE38
:100E500045AA94EDC7FA94EDC32A23EE8F7AD4ED18
:100E6000CCFAD4EDC81A60EE2F5A94EDC44AE0EEE5
:100E7000A06AD4EDCDDA94EDC9DAE3EEA15A94ED8F
:100E8000D13A94EDD4EA20EE833A94EDC5CAD4ED7C
:100E9000C08A26EE886AD4EDD5EAA6EE827A94ED71
:100EA000BF9AE6EE845AD4EDBE9A66EE272AA6EEE5
:100EB00022AA65EE8E4AF0EE64BA87EE8A6AF0EEF8
:100EC0004AAA60EE2D7AE3EE8D7A73EE277A84EDEE
:100ED000D26A94EDD36AE6EE8C7A27EE061A87EE94
:100EE0000A6AE7EE01AAB0EE427AA6EE627AB0EEA6
:100EF000626AA2EE016AB0EE412A84EDC37A27EE5F
:100F0000017AA1EEA42AA8EE227A85EEAA8AF0EE52
:100F10006A2AE5EEA42AF0EE445AC7EEA2CAE8EE29
:100F2000465AE8EE411A20EE288AA4EE246AB0EE72
:100F3000454AA3EE898AA5EEA47AC4EDC45A67EEA9
:100F4000AE5AC4EDC81AB0EE62BAA3EE254AB7EEA7
:100F5000003AA7EEA5BAE5EEADBA73EE487A94ED85
:100F6000C18AE0EEC87AF0EE6D0AECEEE40AE6EE35
:100F7000E97AC4EDCD0A65EEA00A67EEABBAEFEEF2
:100F8000A40AA0EE204AB0EE4C0AF0EE4D0AACEEF8
:100F9000C60AECEEC20AA5EE8C6AA5EE8D2AA5EE75
:100FA000807A84EDC50AC4EDC90A65EEA00A27EE71
:100FB000866A27EE822AEFEE010A67EEA57AA6EE90
:100FC000874A83EE0B7AE1EEA40A25EE0BBAA3EE74
:100FD000A04AE7EE069A82EE8B6A65EE222AC5EEFB
:100FE000046A2AEE855ACAEEA24AA7EE278AA7EE1D
:100FF000029AEBEE878A8AEE057A83EE294A24EE7E
:101000008E5AD4EDD34A26EE2E6AFEEE007A84ED97
:10101000D45A66EEA66A84EDD56A69EE275A27EEA1
:10102000247A28EEA76A68EE277A84EDD37A94EDC5
:10103000B97A65EE845AC4EDBE9A33EE473A84ED30
:10104000BF9A26EE046AC4EDC08A67EE847A84ED06
:10105000C18AA3EE267AC4EDBB5A84EDBC6AC4ED06
:10106000BD7A84EDBA7A4BE62B4E002A3FF448AEA7
:10107000CFE6AA1A2C4E0128B28100F0D6800023B8
:10108000338101E6284EB0EE490A4AF047F894ED64
:10109000BB0A30804AF042F8B0EE480A30814AF08C
:1010A0003DF894EDBC0A70804AF038F8B0EE680A5A
:1010B00070814AF033F894EDBD0AB0804AF02EF802
:1010C00028EE080AB081A9EE090AA8EEA80AB1EE36
:1010D000C00A4AF023F8F080B9F1000F13D094F859
:1010E000DD3283B1D4EDB96A9FED107A9FED106ABD
:1010F00037EE667AD4EDBA7A77EEE67A86EE070AAC
:1011000020EE270A01E09FED0B0A4AF007F8F08174
:1011100022E600BFFF41EF476463002480C3C9019A
:10112000B8220024C4220024A02600240800803F06
:101130000000FA44000000009C340020002A65D022
:1011400094EDBB0A4FF00108414E49F0E7FF94EDE2
:10115000BC0A308149F0E2FF94EDBD0A708149F08C
:10116000DDFFB081012009F049FD3A4B83F8008092
:10117000394B83F80E80F8F7CDFCF8F721FA40469A
:1011800009F0E6FD4FF0000997F80080DFF8D8A0DD
:1011900084F8DC92B4E5D4F85863C4F85853F1F7F6
:1011A00003FB3B78582B7FF4D7ADAE1BDFED2B6AEA
:1011B0002B4B282207EE906A401B1A80B8EEE77A84
:1011C0009E80D880C6EE877AFCEEE77A17EE902AEA
:1011D0005A80C1E593F904206421224B01FB0233BC
:1011E00093F85920202A04D19B699B691B047FF541
:1011F0004BAD1D4A01214FF4FA7311701B4A12685E
:10120000BDEC108B12681361BDE8F0870C20104E06
:1012100009F0F4FCB6E7144A01214FF47A73117017
:10122000ECE70A2BB8BF0A23E8E793F9042064210E
:101230000C4B01FB023393F85920202A02D00123E2
:101240003381D6E79B699B691A04F8D417E700BF7E
:10125000646300246433002098340024002474491B
:10126000A0260024B42300249C34002098340020BD
:10127000C24BDB79022B40F021812DE9F047C04CB5
:10128000B4F85C33B4F85E239A422DED028B82B041
:1012900000F00981A4F85E330126B4F8603313F43A
:1012A000006300F0078194F86473002F00F00A8255
:1012B000DFF8008394ED4E8A98F80050B4F9DCA36F
:1012C0004A2D00F04C81492D12D10023B4F870C38F
:1012D000B4F872131A46B4F80E016CF30F036AF3F4
:1012E0000F0260F31F4361F31F42A649C1E90032B8
:1012F000B4F9DE23DFF8C092AAEB0203DFEDA26AA5
:10130000DFEDA27A07EE103A99F81C30B8EEC77AF2
:10131000A3F10503B3FA83F3B4EEE67A5B0967EE53
:10132000277AF1EE10FA84F8743300F20B819FED06
:10133000987A77EE877AF0EEE78A4A2DA4F872233E
:10134000C4EDDE7AC4EDE38A00F0CF80002E63D0D6
:10135000D4EDF87A4C2D94EDF90AF8EE677A8D4ABF
:101360009FED8D7A516830EE670AC4EDDA7A67EE48
:10137000876AC4EDF97AD2ED027AB4F80C3120EE26
:10138000270AC4F87C13C4EDDB6AB4F8EE1384EDCD
:10139000E00AA4F8703300F04581A1B307EE903A5B
:1013A00094F80534B1EE006AF8EEE77A77EEC07A89
:1013B000F0EEE77A67EE877A07EE103A774BB8EEF1
:1013C000C77AC7EE876A36EE867AC6EE077AC4ED2C
:1013D000F37AD3ED017AF5EEC07AF1EE10FA40F32C
:1013E00091819FED6F6AB0EE007A67EE867AC7FE54
:1013F000C77A042F05D1B0EE0C7AC6FEC76A76EE26
:10140000A77AC4EDE47A482D00F057814A2D03D124
:1014100049F084FE5B4B1880F1F7C6F999F81C304F
:10142000052B40F0CB8094F8DC3013F0010200F083
:10143000DF80D4F808245B49821A8A4240F3E982AB
:1014400003F0020394F81021C4F80804002B15BF20
:101450000023012301210021032A84F80C3494F98C
:101460000E348CBF4FF0FF3201221344022B1A4678
:10147000A8BF0222012B22EAE27284F80E2400F3B4
:10148000D082002384F80D3484F8D413082F3FD879
:10149000DFE817F03B017A02C4018C010502EC0180
:1014A000300033007501B4F86033002613F4006394
:1014B0007FF4F9AE1F4684F86433F9E63A4B03F142
:1014C000780102E0063399420ED01A780A2AF9D13F
:1014D0009878DA789042FFF4D0AE5A79002A7FF4F7
:1014E000CCAE06339942F0D17047264BA3F808A042
:1014F0005A812BE7304618F0C1F92C4BD4EDEF7A26
:1015000093ED187AB4EEE77AF1EE10FA00F3E58085
:1015100098F800304A2B29D0242B09D1DFED1B7A13
:1015200094EDE50A20EE270A49F0F8FD154B1880E6
:1015300018F04CF8304602B0BDEC028BBDE8F04725
:1015400017F064BDDFED1A6AB4EEE67AF1EE10FA38
:101550007FF7F1AE9FED0E7A77EEC77AEBE6B0EE4D
:10156000480A49F0DBFD074B9880C1E694EDE70A95
:1015700049F0D4FD034BD880DAE700BF9C63002418
:101580005C7D0024A02600240000E1C4CDCCCC3D2D
:101590000000B443F00500240AD7233C80810024D6
:1015A0003EC3AE393F420F00A863002468330020D9
:1015B0000000E1449F260024CC690024002384F825
:1015C000D433082FA4D801A353F827F00B1705082C
:1015D000031A05081D180508AD1705089F1805080A
:1015E0006D180508F5140508FB1405087F17050894
:1015F00084F8D423082F8BD801A353F827F000BF19
:101600000B1705080B1A05081D180508AD17050866
:101610009F1805086D180508F5140508FB14050842
:101620007F170508FDEEC07ACD4D17EE900A288190
:1016300000293FF4F1AE07EE903A94F80534F1EE4C
:10164000005ADFEDC86AF8EEE77A77EEC07AF0EE7E
:10165000E77A67EE877A07EE103AC34BB8EEC77A9F
:1016600087EE876A36EE255A66EE267A85EE857A0B
:10167000FDEEE77A84EDF37A93ED017A17EE903A76
:10168000B5EEC07A6B81F1EE10FA40F3E381DFED45
:10169000B75AF0EE007A27EE257A87FE677A67EE72
:1016A000267AFDEEE77A17EE903A1BB2042FAB8153
:1016B00000F0D48184EDE47AAEE649F02FFDA84B2A
:1016C0009880A9E60123384684F8643317F09EFC1D
:1016D00017F07CFF94F86473EAE5A54A136843F0B9
:1016E000805313602379D90708D594F8222412B9BE
:1016F00043F002032371072011F010F8002384F84F
:10170000643305E7DFED9B7A73E62379DD0704D4C4
:10171000994B1B7A002B00F0BA81D4EDE57AC8FE14
:10172000277AC4EDE57A002E3FF4F2AEB4F8EC333C
:10173000F6EE005AD4EDDB6A06EE103A94F8FB336D
:1017400066EEA56AB4F80024B8EE466A012B07EEEF
:10175000102A84EDE78AC6FEC66AC4EDEC6A00F082
:10176000DD81B8EEC77ADFED7F6A022B27EE267A9D
:1017700000F0CD8177EE877AC4EDE67AC8E67C4A40
:10178000136843F0805313602379DA0708D594F87F
:10179000222412B943F002032371012010F0BEFF8E
:1017A000002384F8B43384F86433B1E6B7EE007AEA
:1017B000D4EDEE7AF4EEC77AF1EE10FA05D59FED8E
:1017C0006F7A77EE877AC4EDEE7AF3EE0E7AF4EE66
:1017D000E78AF1EE10FA0DD5B4F8E83307EE903A47
:1017E0000423F8EE677A84F864330023C4EDEA7AC0
:1017F00084F8B433B4F8EE3394EDE07A07EE903A1F
:101800005F4B84EDE97AF8EEE77AB4EEE77AF1EE31
:1018100010FA4CBF012200225A7379E694EDE67A61
:10182000574BB4EEC87A1A7BF1EE10FACCBF012305
:101830000023934200F0FA80B4F8F633D4EDDB6A6B
:1018400007EE903A002384EDE77AF8EEE77AC4F8E1
:10185000A033F4EEE76AF1EE10FA02DD032384F818
:101860006433D4F88033C4F8A43351E694F81034C8
:101870009FED3C7A07EE903AF8EEE77A67EE877ACA
:10188000B4EEE78AF1EE10FA05D50622002384F8BB
:10189000642384F8B433304617F0F0FF38E6384A52
:1018A000B7EE007AD4EDEE7AF4EEC77AF1EE10FAE4
:1018B00005D59FED327A77EE877AC4EDEE7AB4F8EB
:1018C000EE3394EDE97A07EE903A537BF8EEE77A3F
:1018D000F4EEC77AF1EE10FACCBF012200229A4250
:1018E00007D177EEC77ADFED256AA7EEA67A84EDF9
:1018F000E97AF7EE006AD4EDF47A9FED226AB0EE51
:10190000007A76EEE76AE6EE867A37EE677AC4ED1D
:10191000F47A84EDF27A002E3FF4FAADB4F8E833AD
:10192000B6EE007AD4EDDB5A06EE903A94EDEC6A0E
:10193000F8EE666AF4EEC65A26EE877AC4EDEA6AD5
:10194000F1EE10FA67EE277AC4EDEB7A3FF6E0ADE0
:101950000522002384F8642384F8B433D8E500BF5B
